:100000000C947A370C94AB370C94AB370C94AB3719
:100010000C94AB370C94AB370C94AB370C94AB37D8
:100020000C94AB370C94AB370C94AB370C94AB37C8
:100030000C94AB370D94E2A70C94AB370C94AB3710
:100040000C94AB370C94FDF10C94AB370C94AB379C
:100050000C94AB370C94AB370C94C4EE0D9498A76A
:100060000C94AB370D942C7F0D94227F0C94AB37FE
:100070000C94AB370C94AB370C94AB370C94AB3778
:100080000D94234F0C94AB370C94AB370C94AB37D7
:100090000C94AB370C94AB370C94AB370C94AB3758
:1000A0000C94AB370C94AB370D94F54E0C94AB37E6
:1000B0000C94AB370C94AB370C94AB370C94AB3738
:1000C0000C94AB370C94AB370C94AB370C94AB3728
:1000D0000C94AB370C94AB370C94AB370C94AB3718
:1000E0000C94AB37084AD73B3BCE016E84BCBFFDB6
:1000F000C12F3D6C74319ABD56833DDA3D00C77FF8
:1001000011BED9E4BB4C3E916BAAAABE0000008090
:100110003F05A84CCDB2D44EB93836A9020C50B91F
:10012000918688083CA6AAAA2ABE000000803F0744
:10013000634236B79BD8A71A39685618AEBAAB5582
:100140008C1D3CB7CC5763BD6DEDFD753EF6177247
:1001500031BF000000803F08000000BE9224491219
:100160003EABAAAA2ABECDCCCC4C3E00000080BE3D
:10017000ABAAAAAA3E00000000BF000000803F001A
:1001800000000000084178D3BB4387D1133D190E0E
:100190003CC3BD4282AD2B3E68EC8276BED98FE176
:1001A000A93E4C80EFFFBE01C4FF7F3F000000006E
:1001B00000000C9468910C9484430C941C9C0D9446
:1001C00046B10D94A44E0C94FF9B0C94619D0C942D
:1001D000B1C70D9484A20D947C7D0C94AB910C94CA
:1001E0000BA10D9415A20C948EE00C942C9D0D94F3
:1001F000DEA00C94D28D0C94A2A30C944B960C947C
:1002000018A50C94B5920D9491500D9434A10C94B2
:1002100057960C9475960C94DD8D0C94A3C70D9491
:100220000EA10C94BAC70C94CBB00C94269B0C94E2
:1002300078580C949C920C94C4370D94FDA00D94A6
:1002400026A10C946CB00D94C67F0D940AA10D9458
:1002500029A20C9403920C94CDCC0C946F960C9420
:10026000C3C70C949F9D0C94BA900C947B960C94ED
:1002700044C80C9478B90D94E3A00C94DB460D941B
:100280005FA10C94DE370C94BDC70C942D960D9491
:100290006C7D0C943AC20C94CDE00C94F6A70C94AF
:1002A000529D0C94C1B40C94C6A70C94ECCD0C9444
:1002B000C0C70D943B7C0D94F17A0D94FEA10D9472
:1002C00022A10C9410990C942AA90C942EAC0C9495
:1002D0003BA40C94BFB00C940ABE0C94DE960D9413
:1002E000BF4E0D9404A10C9411390C94B4C70C9416
:1002F000F7370C9490DC0C94579D0C94BAA70C948F
:10030000ADD10C945C470C94149C0C946A920C94A0
:1003100041990C94CED50C94155D0C944CA90D9478
:10032000437B0C9451960C94D6CE0D9439A20D9427
:100330007AA20D94BA7F0C940A590C9408C80C94B4
:100340001C970C9459910C9439960C94B8A00C9469
:10035000CEA70C9453C80C94E09D0D94DC7F0C94B4
:100360005EB00C9486CA0C9417380C9460B00C9450
:100370009B9A0C9402AA0D9463800C9452B30C9433
:1003800077C70C9469960C941C8E0C94B1DF0D9475
:1003900018A10C9417470D941FA20C942B9B0D943D
:1003A000A9A10C9403A30D94B7B10C9494CF0C9411
:1003B00051900D94AFA10C946D440D94894E0C9402
:1003C00067A00C9471B00C9483920D9498A20C9435
:1003D00073390C9470D70C94129C0C94CE920D949B
:1003E0006A500D9414A10C9447BC0C941E9E0C945E
:1003F0005AC40C94D2A70C949A390C942E920C9453
:10040000DB370C9483900C94F5DF0D9457A20C9479
:10041000B6A70C94448E0D944A490C940EDC0C94AF
:10042000F15A0D948EA20C94A0E00C94FBDE0C9477
:1004300010E00D94C27F0C94B6440C945AC10C94F5
:10044000809D0C94AEA70C9466B00C945C9D0C94AB
:10045000BEA70C94D4CB0C94AD370C9490DF0D94C4
:1004600099B10D948D7F0C94FF9D0D94BE7F0C94DB
:10047000CAC70C94A9A00C9491DC0C943E8E0C94E9
:10048000CD900C94E4DD0D94B27F0C9480430C94D9
:1004900040910C94AF8D0C94DBA70C94CDC70C94B9
:1004A000C8C70C9436920D94B67F0C94219C0C9482
:1004B0006EB00C9453AA0C94D8A70D9498A10C94E8
:1004C0005D960D9401A10C94D9920D94C4A10D9444
:1004D000647F0C94CAA70C94C4C30C94FB900C9436
:1004E00068B00C946A900C94A0930D94493E0D94BE
:1004F0002AA10C945CAA0D94F87A0C9434A90C945B
:10050000AAA70C94D2B50C94AEC70D9470A20C940B
:10051000E0900D944DA20D94E47F0C9414910C94F2
:1005200044AA0C9497E10D9466A20D94D17F0C948B
:1005300082D30D94B2800C9444A20C94319B0C9401
:1005400063960C94169C0D949C7F0C94FA910C94D9
:1005500012B10D9444A10C9418DF0C94C2A70C9412
:1005600092900C9445960C9433960C9464B00D9430
:1005700043A20C9445940C947B910D940BA20C9483
:10058000258E0C9462B00C94B2A70D94CA7F0C9483
:1005900014A10D9430A10C942BBB0C9477990C945E
:1005A000E8380D94F5A00D94DA4E0C9488430C9421
:1005B00094910D94757D0C946AB00C9471A00C9478
:1005C0006CA00C94AB900D941CA10C94C8A90C9435
:1005D0000F920C944D9D0C947C9B0C9427910D9440
:1005E00090800D94F9A00C94A1B70C947CDE0C942F
:1005F000D5A70D9431A20D9406A20D945B400D94E5
:10060000AB7F0C94B7C70D94B9A10D949DA10C9428
:10061000219B0C9439A20C943F960C942DAF0C9412
:10062000A5B84E414E494E495459494E46CDCCCCC1
:100630003D0AD7233C17B7D13877CC2B329595E6B6
:10064000241FB14F0A000020410000C84200401C96
:100650004620BCBE4CCA1B0E5AAEC59D7400407AE3
:1006600010F35A00A0724E18090010A5D4E800003B
:10067000E87648170000E40B54020000CA9A3B00D9
:100680000000E1F505000080969800000040420F50
:10069000000000A08601000000102700000000E814
:1006A00003000000006400000000000A00000000D9
:1006B000000100000000002C76D888DC674F08237A
:1006C000DFC1DFAE59E1B1B796E5E3E453C63AE6E0
:1006D00051997696E8E6C28426EB898C9B62ED40C0
:1006E0007C6FFCEFBC9C9F40F2BAA56FA5F490050F
:1006F0005A2AF75C936B6CF9676DC11BFCE0E40D43
:1007000047FEF520E6B500D0ED902E030094357736
:10071000050080841E080000204E0A000000C80C5E
:10072000333333330F986E12831141EF8D211489C7
:100730003BE65516CFFEE6DB18D1844B381BF77C21
:100740001D901DA4BBE424203284725E228100C966
:10075000F124ECA1E53D27434F4D4D554E49434112
:1007600054494F4E0044525952554E004552524F33
:10077000525300494E464F004543484F00473236DA
:100780002048656174696E67204E6F7A7A6C6500E7
:100790004732362048656174696E6720426564009F
:1007A00057616974696E6720666F7220686561744D
:1007B00075702E0A004669786564204C656E677412
:1007C00068205072696D6500446F6E6520507269D3
:1007D0006D696E67004D616E75616C207072696D38
:1007E000696E672E2E2E004C656176696E67204714
:1007F0003236003F53706563696669656420582C22
:100800005920636F6F7264696E617465206F7574CF
:10081000206F6620626F756E64732E0A003F285247
:100820002965706561742076616C7565206E6F74E2
:1008300020706C61757369626C653B206D757374B3
:10084000206265206174206C6561737420312E0A0A
:10085000003F537065636966696564206E6F7A7ADC
:100860006C652074656D7065726174757265206E5B
:100870006F7420706C61757369626C652E0A003F3D
:100880005370656369666965642066696C616D654E
:100890006E742073697A65206E6F7420706C617558
:1008A0007369626C652E0A003F53706563696669FF
:1008B0006564207072696D65206C656E6774682070
:1008C0006E6F7420706C61757369626C652E0A00BE
:1008D0003F537065636966696564206E6F7A7A6CF0
:1008E000652073697A65206E6F7420706C61757312
:1008F00069626C652E0A003F5265747261637469A7
:100900006F6E204D756C7469706C696572206D75C1
:100910007374206265207370656369666965642E0F
:100920000A003F53706563696669656420526574A7
:1009300072616374696F6E204D756C7469706C6957
:100940006572206E6F7420706C61757369626C657E
:100950002E0A003F537065636966696564206C61A7
:1009600079657220686569676874206E6F7420709D
:100970006C61757369626C652E0A0043292E0A004A
:100980003F537065636966696564206265642074BD
:10099000656D7065726174757265206E6F7420701C
:1009A0006C61757369626C65202834302D004732A4
:1009B00036207374617274696E672E2E2E0A004F92
:1009C00046460A0046616465204865696768742088
:1009D00000426564204C6576656C696E6720004650
:1009E00061696C656420746F20656E61626C65205E
:1009F000426564204C6576656C696E670A00496ED5
:100A000076616C6964206D6573682E0A0076616C8E
:100A100069640A53746F7261676520736C6F743A0E
:100A20002000696E004D65736820697320003F5592
:100A30007365203020746F20003F496E76616C69C9
:100A4000642073746F7261676520736C6F742E0A13
:100A5000003F454550524F4D2073746F726167657A
:100A6000206E6F7420617661696C61626C652E0A1C
:100A7000004D65736820706F696E74206F75742007
:100A80006F662072616E67650A004D3432312069ED
:100A90006E636F727265637420706172616D6574EC
:100AA00065722075736167650A00446576696174D3
:100AB000696F6E0025533A2025730046696E69738D
:100AC000686564210A003A207A3A2000206F662087
:100AD00000476F696E6720746F3A20580043570AC9
:100AE00000206469723A0020616E676C653A0053B9
:100AF00074617274207261646975733A004D3438A0
:100B000020506F696E740025533A2025642F2564A8
:100B100000506F736974696F6E696E6720746865E1
:100B20002070726F62652E2E2E0A003F4C6567732F
:100B3000206F66206D6F76656D656E7420696D70CF
:100B40006C61757369626C652028302D3135292EF2
:100B50000A003F2028582C5929206F7574206F6691
:100B600020626F756E64732E0A0050726F6265208A
:100B70006F7574206F6620626F756E6473003F53EB
:100B8000616D706C652073697A65206E6F7420707A
:100B90006C61757369626C652028342D3530292E9F
:100BA0000A004D3438205A2D50726F62652052650C
:100BB000706561746162696C6974792054657374DD
:100BC0000A003F2856296572626F7365206C65764E
:100BD000656C20696D706C61757369626C65202845
:100BE000302D34292E0A005374616E6461726420C2
:100BF000446576696174696F6E3A20002052616EB7
:100C000067653A2000204D61783A2000204D696EDA
:100C10003A2000205369676D613A20004D65616E8E
:100C20003A20005741524E494E4721204C6F7720C1
:100C30005A204A65726B206D6179206C6561642071
:100C4000746F20756E77616E746564207061757362
:100C500065732E0A0020204D61783A200020002084
:100C6000204D696E3A2000536F667420656E647380
:100C7000746F70733A20004D32342053256C642019
:100C800054256C64004739322E39204525730047BE
:100C90003120462564004739322E39205A25730009
:100CA0004731205A30204632303000473120582515
:100CB0007320592573204633303030004D343230A4
:100CC00020532569205A2573004D31303620502598
:100CD0006920532569004D32303020442573004788
:100CE000323852305859004739322E392045302099
:100CF0005A300A47315A2573004D31303920532577
:100D000069004D31393020532569004D343230208F
:100D10005330205A300020496E76616C696420653A
:100D200078747275646572200047322F47332062F1
:100D3000616420706172616D65746572730A00533D
:100D40006C6565702E2E2E005A2050726F626520E1
:100D500050617374204265640A005A2050726F62B9
:100D60006520506173742042656400205A3A200067
:100D700020593A200042656420583A20004D65739E
:100D80006820706F696E74206F7574206F662072B2
:100D9000616E67650A004D302053746F70004D31ED
:100DA0002053746F7000436C69636B20746F205222
:100DB0006573756D652E2E2E004E6F204D6F766516
:100DC0002E00456E642066696C65206C6973740A38
:100DD00000426567696E2066696C65206C69737492
:100DE0000A004E6F206D656469610A005265737573
:100DF0006D696E6720534400286E6F2066696C65CC
:100E0000290043757272656E742066696C653A20BC
:100E1000005072696E742074696D653A20000A533F
:100E2000746174733A2046696C616D656E742075E7
:100E30007365643A20002C204C6F6E6765737420D4
:100E40006A6F623A2000546F74616C2074696D653A
:100E50003A200053746174733A20002C2046616973
:100E60006C65643A20002C2046696E69736865647D
:100E70003A20005072696E74733A200053746174A2
:100E8000733A2000436F6F6C696E672E2E2E0048F8
:100E9000656174696E672E2E2E0045202553006F04
:100EA0006B006F666600780773076C076507570766
:100EB00044454255473A004D313133205300426595
:100EC0006420436F6F6C696E672E2E2E004265643E
:100ED0002048656174696E672E2E2E00537550652B
:100EE000522043522D3230204F46462E002F2F00E5
:100EF0004D31343520533C696E6465783E206F7502
:100F000074206F662072616E67652028302D31294C
:100F10000A00205200416363656C65726174696FF9
:100F20006E3A2050004D32303620580046523A007A
:100F300020466C6F773A20003A2000205365727685
:100F40006F2000206F7574206F662072616E676578
:100F50000A00536572766F200020643A0020693AD7
:100F60000020703A00496E76616C6964206578747F
:100F700072756465720A0020643A0020693A0020A4
:100F8000703A004C434420436F6E74726173743A3C
:100F9000200064697300656E0043290A0061626C79
:100FA000656420286D696E2074656D702000436F44
:100FB0006C64206578747275646573206172652055
:100FC000004F666673657473204170706C69656468
:100FD000004572723A20546F6F206661722100548E
:100FE0006F6F206661722066726F6D207265666534
:100FF00072656E636520706F696E740A00454550B6
:10100000524F4D204F4B0A002E0A002028302D3120
:101010003029002076616C7565206F7574206F66CD
:101020002072616E676500416476616E6365204B76
:101030003D004F4646004F4E00506F7765722D6C55
:101040006F7373207265636F7665727920004D3817
:101050003400446F6E65207072696E74696E67202B
:1010600066696C650A004D3737004D3331004361C6
:10107000703A004D4541545041434B00434F4F4C53
:1010800045525F54454D50455241545552450043D9
:1010900048414D4245525F54454D5045524154558B
:1010A000524500424142595354455050494E470021
:1010B00041524353004D4F54494F4E5F4D4F4445AD
:1010C0005300544845524D414C5F50524F54454394
:1010D00054494F4E004C4F4E475F46494C454E4198
:1010E0004D45004155544F5245504F52545F534463
:1010F0005F5354415455530053445F57524954452C
:10110000005245504541540053444341524400501D
:10111000524F4D50545F535550504F525400454D0F
:10112000455247454E43595F504152534552004343
:101130004153455F4C494748545F425249474854E0
:101140004E45535300544F47474C455F4C49474821
:10115000545300534F4654574152455F504F5745E3
:1011600052004255494C445F50455243454E54004D
:101170004C4556454C494E475F44415441005A5FE7
:1011800050524F42450052554E4F55540041555410
:101190004F4C4556454C005052494E545F4A4F42C1
:1011A0000050524F4752455353004155544F5245FA
:1011B000504F52545F54454D5000564F4C554D457D
:1011C0005452494300454550524F4D0042494E410B
:1011D00052595F46494C455F5452414E5346455221
:1011E0000053455249414C5F584F4E5F584F464659
:1011F000004649524D574152455F4E414D453A4D8B
:1012000061726C696E20322E302E375F4457372E54
:101210003320544D33442032534D4442552028410D
:10122000707220323420323032312032313A323151
:101230003A34332920534F555243455F434F444579
:101240005F55524C3A68747470733A2F2F67697403
:101250006875622E636F6D2F496E73616E69747964
:101260004175746F6D6174696F6E2F4D61726C6939
:101270006E2F747265652F437265616C6974794471
:1012800077696E5F322E302050524F544F434F4C8F
:101290005F56455253494F4E3A312E30204D41430F
:1012A00048494E455F545950453A53755065522050
:1012B00043522D32302045585452554445525F43D5
:1012C0004F554E543A3120555549443A636564654B
:1012D000326132662D343161322D343734382D3954
:1012E0006231322D633535633632663336376666A2
:1012F0000A0050726F6265204F6666736574205AEB
:101300000050726F6265204F6666736574205A00E4
:10131000290A0020746F20003F5A206F7574206FD7
:10132000662072616E6765202800290A0020746FAC
:1013300020003F59206F7574206F662072616E67C0
:101340006520282D00290A0020746F20003F5820B6
:101350006F7574206F662072616E676520282D009E
:1013600050726F6265204F66667365742058004343
:10137000616E6E6F74206F70656E20737562646944
:101380007220002569730025696D20256973002589
:1013900069682025696D2025697300256964202509
:1013A00069682025696D20256973002569792025E4
:1013B0006964202569682025696D202569730023EB
:1013C000646566696E652044454641554C545F002E
:1013D000626564004B6420004B6920004B70200064
:1013E000504944204175746F74756E652066696E4E
:1013F0006973686564212050757420746865206C79
:10140000617374204B702C204B6920616E64204BFB
:101410006420636F6E7374616E74732066726F6D97
:101420002062656C6F7720696E746F20436F6E6603
:10143000696775726174696F6E2E680A005049445D
:10144000204175746F74756E65206661696C6564A2
:10145000212074696D656F75740A005049442041FC
:1014600075746F74756E65206661696C65642120A2
:1014700054656D706572617475726520746F6F204C
:10148000686967680A00204B643A2000204B693A7B
:101490002000204B703A200020436C617373696315
:1014A00020504944200A00204E6F206F76657273E9
:1014B000686F6F740A002054753A2000204B753A0B
:1014C0002000206D61783A2000206D696E3A20007E
:1014D00020643A200020626961733A200050494438
:1014E000204175746F74756E652073746172740A2F
:1014F00000504944204175746F74756E65206661B3
:10150000696C6564212054656D70657261747572D3
:101510006520746F6F20686967680A00504944202D
:101520004175746F74756E6500504944204175743F
:101530006F74756E65206661696C65642120426117
:1015400064206865617465722069640A004572727E
:101550003A207574663820666F6E74206E6F742042
:10156000696E697469616C697A65642E004572728E
:101570003A207574663820666F6E74206E6F742022
:10158000696E697469616C697A65642E004572726E
:101590003A207574663820666F6E74206E6F742002
:1015A000696E697469616C697A65642E0000FE0079
:1015B00003FF8007C7C00701E00000E00000F00063
:1015C00000700400700E00701F00703F80F00E006D
:1015D000E00F01E007C7C003FF8000FE0000FE002F
:1015E00003FF8007C7C00F01E00E00E03F80F01F3F
:1015F00000700E00700400700000700000F0000029
:10160000E00701E007C7C003FF8000FE000E000EE8
:10161000000E000E000E000E000E000E007FC03FF8
:10162000801F000E00040004000E001F003F807F9A
:10163000C00E000E000E000E000E000E000E000E7A
:1016400000FFFFFF7F80FFC0FFC0FFC07F807F8063
:10165000FFC0FFC0FFC03F001E000C00FFE0FFD135
:1016600040A0C8A6A22FF80023AC00AF10FFFEFFD9
:1016700005FFD0FFE0FFC1FFD1E240A0C8A6A22F26
:10168000F800238127AC00AFFFD0FF64FFD1A5FF96
:10169000D0FF64FF64FFD1A4FFD0FF16FFFE4265B8
:1016A0006400456E636C6F73757265002568753AEA
:1016B00025303268750025303268753A2530326839
:1016C0007500202020202020200020202020001F26
:1016D000E0201020102010102010202010201030AA
:1016E000300840048003001FE03FF03FF03FF01F50
:1016F000E01FE03FF03FF03FF00FC0078003003FE6
:10170000FFF038007030FC3020FC102078102030C2
:10171000102C00D02E31D02F7BD02F7BD02E31D06B
:101720002C00D020301020781020FC1030FC3038F5
:1017300000703FFFF03FFFF03800703186302387A4
:10174000102787902F87D02F03D0203010207810BB
:101750002078102030102F03D02F87D02787902398
:1017600087103186303800703FFFF01FFFF81FFFF1
:10177000F8041040020820020820041040082080CD
:101780001041001041000820800410400000001F9C
:10179000FFF81FFFF8FFFFFF8000018E00E19F01AF
:1017A000F19381399F81F99F81F99FB9F98F28F1D0
:1017B0008038018000019FFFF99174999B06A99BD5
:1017C00054A99B56A99B54999FFFF9FFFFFF53759E
:1017D0005065522043522D32302052656164792E7B
:1017E000005072696E74696E672E2E2E006E6F74D3
:1017F000696669636174696F6E200063616E636519
:101800006C005072696E742041626F72746564007E
:101810004469736D6973730055492041626F727436
:101820006564004D323520500A4D323400507269E3
:101830006E742050617573656400526573756D65D3
:101840000055492050617573650050617573696E6C
:10185000672E2E2E00726573756D65004D32340053
:1018600050726F6265205A204F6666736574004C33
:101870006F6164206D6D00556E6C6F6164206D6DDD
:101880000046696C2E204469612E004520696E2057
:101890006D6D5E3300416476616E6365204B004D73
:1018A0003330332055312045256920532569000008
:1018B0000C0F00FE07022503BB017FFE08FE08FE99
:1018C00005080806000040F0C888889878100508C8
:1018D00008060000C0F88888888888F8050505068D
:1018E00000012030F830200508080600002070F8BC
:1018F00020202020E00509090600FF2070A8A8B8D4
:1019000088887020070505070001D86C366CD8055B
:1019100009090600FFF8A88888888888A8F8050AB9
:101920000A0600FE205050505088A8A88870030373
:101930000306000340A040FFFFFFFFFFFFFFFFFF84
:10194000FFFFFFFFFFFFFFFFFFFFFFFFFF000000A4
:101950000605FF0107070602008080808080008066
:10196000030303060105A0A0A0050606060000501B
:10197000F85050F8500509090600FF2070A8A07023
:1019800028A87020050707060000C8C81020409846
:101990009805070706000040A0A040A89068010332
:1019A000030602058080800309090601FF204040EC
:1019B0008080804040200309090601FF80404020CC
:1019C000202040408005070706000020A8702070F6
:1019D000A8200505050600012020F82020020303A9
:1019E0000601FFC04080050101060003F802020263
:1019F000060100C0C00507070600000810102040BF
:101A00004080050707060000708898A8C888700302
:101A1000070706010040C040404040E005070706B8
:101A20000000708808102040F8050707060000F83D
:101A30000810300888700507070600001030509025
:101A4000F81010050707060000F880F008088870F5
:101A5000050707060000304080F0888870050707FA
:101A6000060000F8081010202020050707060000D7
:101A7000708888708888700507070600007088885D
:101A800078081060020505060100C0C000C0C00251
:101A900006060601FFC0C000C04080030505060120
:101AA000012040804020050303060002F800F803EF
:101AB000050506010180402040800507070600005B
:101AC000708810202000200507070600007088B8E5
:101AD000A8B88070050707060000708888F8888815
:101AE00088050707060000F04848704848F00507D9
:101AF0000706000070888080808870050707060050
:101B000000F04848484848F0050707060000F880FC
:101B100080F08080F8050707060000F88080F080DC
:101B2000808005070706000070888080988870050F
:101B30000707060000888888F88888880307070652
:101B40000100E04040404040E00507070600003843
:101B50001010101090600507070600008890A0C0C4
:101B6000A09088050707060000808080808080F8AC
:101B700005070706000088D8A88888888805070711
:101B80000600008888C8A89888880507070600000E
:101B900070888888888870050707060000F08888A4
:101BA000F080808005070706000070888888A8906C
:101BB00068050707060000F08888F0A090880507F0
:101BC0000706000070888070088870050707060007
:101BD00000F8202020202020050707060000888824
:101BE00088888888700507070600008888888850DC
:101BF000502005070706000088888888A8A8500597
:101C000007070600008888502050888805070706C7
:101C1000000088885020202020050707060000F8D3
:101C20000810204080F80309090601FFE080808049
:101C300080808080E005070706000080404020107B
:101C400010080309090601FFE020202020202020A1
:101C5000E00503030600052050880501010600FE8B
:101C6000F803030306010580402005050506000072
:101C700070087888780507070600008080F088885B
:101C800088F005050506000070808088700507074C
:101C90000600000808788888887805050506000091
:101CA0007088F08070050707060000304840E0406B
:101CB00040400507070600FE708888887808700590
:101CC00007070600008080F08888888803070706D9
:101CD00001004000C0404040E00409090601FE1038
:101CE000003010101010906005070706000080807B
:101CF0008890E09088030707060100C040404040FC
:101D000040E0050505060000D0A8A8A8A80505051F
:101D1000060000B0C88888880505050600007088A0
:101D20008888700507070600FEF0888888F08080A4
:101D30000507070600FE78888888780808050505E5
:101D4000060000B0C8808080050505060000788088
:101D50007008F00507070600002020F82020201852
:101D600005050506000088888898680505050600B1
:101D70000088888850200505050600008888A8A8E6
:101D80005005050506000088502050880507070605
:101D900000FE88888850204080050505060000F870
:101DA000102040F80309090601FF20404040804010
:101DB0004040200109090602FF80808080808080E9
:101DC00080800309090601FF8040404020404040D8
:101DD0008005030306000248A890FF554E4C4F4172
:101DE000442046494C414D454E54004C4F414420FF
:101DF00046494C414D454E540046494C414D454E97
:101E000054204348414E4745005049442041757491
:101E10006F74756E65202A005049442D44202A00B5
:101E20005049442D49202A005049442D50202A0071
:101E300020082046616374002008204D617800204E
:101E400008204D696E004F6666004F6E0041757444
:101E50006F74656D70005654726176204D696E0026
:101E6000566D696E00566D6178204500566D61783B
:101E7000205A00566D6178205900566D61782058BF
:101E800000416D6178204500416D6178205A004124
:101E90006D6178205900416D6178205800412D54C2
:101EA000726176656C00412D5265747261637400D5
:101EB000416363656C0056652D4A65726B00565A26
:101EC0002D4A65726B0056592D4A65726B00565843
:101ED0002D4A65726B0050726F6265205A204F6602
:101EE000667365740050726F62652059204F666694
:101EF0007365740050726F62652058204F66667378
:101F0000657400452073746570732F6D6D005A20E1
:101F100053746570732F6D6D005920537465707321
:101F20002F6D6D00582053746570732F6D6D0041D7
:101F30006476616E6365642053657474696E67735B
:101F4000003F0043616E63656C00496E6974004D2B
:101F500034323800496E697469616C697A6520456C
:101F60004550524F4D0046696C616D656E7400546A
:101F7000656D706572617475726500537465707318
:101F80002F6D6D0050726F6265204F6666736574C9
:101F900073004A65726B00416363656C65726174BE
:101FA000696F6E0056656C6F636974790053657470
:101FB00020486F6D65204F66667365747300436FCC
:101FC0006E66696775726174696F6E003F004E6579
:101FD000787420506F696E7400446F6E65004E65B2
:101FE0007874003F0043616E63656C204F626A65E0
:101FF0006374004E4F005945530043616E63656C36
:10200000204F626A656374203D004D61696E005324
:10201000746F770053572D4D6F6465004465706C85
:102020006F790053656C662D546573740052657347
:10203000657400426564004E6F7A7A6C6500466193
:102040006E20537065656400436F6E6669677572D4
:102050006174696F6E004C6F6164205365747469BC
:102060006E67730053746F72652053657474696E84
:10207000677300526573746F72652044656661759D
:102080006C74730050726568656174202420436F1E
:102090006E66004F6666004F6E00506F7765722067
:1020A0004F7574616765004C434420436F6E7472D2
:1020B00061737400424C546F7563680050726F62B4
:1020C00065205A204F666673657400416476616EC0
:1020D0006365642053657474696E6773004D61694C
:1020E0006E004D37303220542564004D363030209C
:1020F000423020542564004D373032203B256400A7
:102100004D37303120542564004D373032004D3783
:102110003031004D363030204230004D61696E0064
:10212000436F6E74696E7565005075726765206DDA
:102130006F726500524553554D45204F5054494FDD
:102140004E533A005052494E542050415553454445
:102150000020204E6F7A7A6C653A20005061726BD5
:10216000696E672E2E2E0000005761697420666F1D
:10217000720066696C616D656E74206368616E677C
:102180006500746F20737461727400576169742004
:10219000666F720066696C616D656E7420756E6C39
:1021A0006F616400004E6F7A7A6C652068656174B7
:1021B000696E6700506C6561736520776169742E84
:1021C0002E2E0000507265737320627574746F6EEA
:1021D00000746F2068656174206E6F7A7A6C650098
:1021E00000496E736572742066696C616D656E740A
:1021F00000616E6420707265737320627574746F11
:102200006E00746F20636F6E74696E756500576140
:10221000697420666F720066696C616D656E74200A
:102220006C6F616400005072657373204275747442
:102230006F6E00746F20726573756D6520707269C2
:102240006E7400005761697420666F722070726945
:102250006E7400746F20726573756D652E2E2E007E
:10226000005761697420666F720066696C616D6504
:102270006E7420707572676500003E2000256C64E6
:102280002E25696D00457874727564656420546FFD
:1022900074616C003E20004C6F6E67657374204A59
:1022A0006F622054696D65003E2000546F74616C4C
:1022B000205072696E742054696D6500436F6D70B3
:1022C0006C65746564003A20005072696E74204336
:1022D0006F756E74003A200031353000350042458C
:1022E000443A204154432031303447542D32005277
:1022F000756E617761792057617463683A204F4E3B
:10230000004D61782054656D7000333135004D69A2
:102310006E2054656D7000350045313A20455043BC
:102320004F53203130304B005053550047656E6598
:102330007269630050726F746F636F6C00312E307E
:1023400000426175640032353030303000437265D0
:10235000616C69747933442052414D505300556E7D
:10236000696669656420426564204C6576656C69C0
:102370006E6700457874727564657273003100741D
:10238000696E796D616368696E657333642E636F1E
:102390006D0053755065522043522D32300032305B
:1023A00032312D30342D313800322E302E375F440B
:1023B00057372E33004D61726C696E005072696E32
:1023C00074657220537461747300546865726D692A
:1023D00073746F727300426F61726420496E666F2E
:1023E000005072696E74657220496E666F004D61AF
:1023F000696E004D313030300053746F7020507270
:10240000696E7400526573756D65205072696E74E3
:1024100000506F776572204F7574616765004D31AC
:1024200039305335350A4732380A47323950310A84
:1024300047323950330A47323953310A4732395318
:10244000300A47323946302E300A473239410A4D78
:10245000313034533231350A4732380A4D31303950
:10246000533231350A4731583135305931353046DC
:10247000353030300A47315A300A4D3530300A4D48
:102480003430300A4D31313720536574205A204F93
:102490006666736574004D313036533132380A4DFB
:1024A0003330334338533231354530550A4D3530AA
:1024B000300A4D313137205049442054756E652023
:1024C000446F6E65004D3139305335350A4D31302A
:1024D00034533231350A4732380A4732394C310ADF
:1024E0004731205831303059313030463530303076
:1024F0000A47315A30004D3530300A4D31313720DE
:1025000053657474696E67732053746F72656400E9
:102510005072657020666F72205A2041646A75732C
:1025200074005049442054756E650053746F726591
:102530002053657474696E67730053657475700019
:102540004D61696E003F004261636B0053746F70B0
:10255000005072696E742066726F6D204D656469FB
:1025600061004368616E6765204D65646961004D77
:1025700032310041626F7574205072696E746572F9
:10258000004368616E67652046696C616D656E74B5
:10259000004C6576656C696E6720546F6F6C7300D4
:1025A000436F6E66696775726174696F6E0054651A
:1025B0006D7065726174757265004D6F74696F6ED0
:1025C00000486F73742053746172740052657375A0
:1025D0006D65205072696E740043616E63656C2096
:1025E0004F626A6563740054756E650053746F7052
:1025F000205072696E740050617573652050726965
:102600006E74004E6F204D6564696100496E666F9F
:102610002053637265656E003F00537461727420CD
:102620005072696E740043616E63656C005072692C
:102630006E740043616E6E6F7420656E74657220F7
:102640007375626469723A2000022E2E004D616932
:102650006E002100486F74656E6420746F6F206394
:102660006F6C64004261636B0050726F63656564F8
:10267000004F6666004F6E00536F667420456E64AF
:1026800073746F7073004D6F74696F6E004469737B
:1026900061626C65205374657070657273004D38AB
:1026A00034004D34382050726F6265205465737465
:1026B000004732384F0A4D343820503130004C65D5
:1026C00076656C20436F726E65727300556E696635
:1026D00069656420426564204C6576656C696E6747
:1026E00000486F6D65205A004732385A00486F6DB8
:1026F000652059004732385900486F6D65205800F1
:1027000047323858004175746F20486F6D65004D31
:1027100061696E0050726568656174202420456EA1
:10272000640050726568656174202420426564000D
:1027300054656D706572617475726500436F6F6C7E
:10274000646F776E0050726568656174202400467E
:10275000616E205370656564207E00426564004EA2
:102760006F7A7A6C65004D61696E0050726F6265B8
:10277000205A204F666673657400416476616E630B
:1027800065204B00466C6F770046616E2053706584
:102790006564207E00426564004E6F7A7A6C650045
:1027A0005370656564004D61696E005A2056616C16
:1027B0007565004732380A4D313930205325690A92
:1027C0004D313039205325690A47323920503100C4
:1027D0004265642054656D7000486F74656E6420B6
:1027E00054656D70002E2569004732395036432DEF
:1027F0000048656967687420416D6F756E740041AB
:10280000646A757374204D657368204865696768EC
:10281000740046696E652054756E6520436C6F7355
:10282000657374004732395034540046696E652030
:1028300054756E6520416C6C004732395034523902
:10284000393954004732380A4732364350482569EF
:102850004225690056616C69646174652043757333
:10286000746F6D204D657368004732380A47323601
:10287000435049310056616C6964617465204D654F
:10288000736820282429004732380A4732364350DB
:102890004930004732394A2569004C6576656C201D
:1028A0004D657368005369646520506F696E747379
:1028B0000047726964204D657368204C6576656CCD
:1028C000696E6700332D506F696E74204C657665B4
:1028D0006C696E67004732394A30004732395033ED
:1028E00052432E2569004D616E75616C2046696CFE
:1028F0006C2D696E00473239503242543000536DAE
:102900006172742046696C6C2D696E0047323950D3
:102910003354300046696C6C2D696E20416D6F75C3
:102920006E74004D65736820696E76616C696461D0
:102930007465642E0A00496E666F20536372656584
:102940006E00496E76616C696461746520436C6FDA
:1029500073657374004732394900496E76616C695A
:102960006461746520416C6C00436F6E74696E75B0
:102970006520426564204D657368004732395031E7
:10298000430046696C6C2D696E204D65736800428A
:1029900075696C6420436F6C64204D6573680047F3
:1029A00032394E5031004275696C6420437573743E
:1029B0006F6D204D657368004732380A4D313930EC
:1029C00049310A4D31303949310A47323950310ADB
:1029D0004D31303453300A4D31343053300042756C
:1029E000696C64204D6573682028242900473238BB
:1029F0000A4D31393049300A4D31303949300A47B2
:102A0000323950310A4D31303453300A4D3134307F
:102A1000533000473239256325690A4D313137205B
:102A2000004D657368202569204C6F616465640002
:102A30004D65736820256920536176656400536194
:102A4000766520426564204D657368004C6F616453
:102A500020426564204D657368004D656D6F727925
:102A600020536C6F74004E6F2053746F72616765F2
:102A7000004732395034582573592573522569005F
:102A8000202D2D2D2D2D005A3A00593A00486F6DFA
:102A9000696E672058595A00473238004F666620E1
:102AA0005072696E746572204261636B7570004785
:102AB0003239532D31004F757470757420666F7202
:102AC00020435356004732395431004F75747075A6
:102AD0007420666F7220486F737400473239543027
:102AE000004D657368204C6576656C696E670045BE
:102AF000646974204D6573680056616C6964617423
:102B000065204D657368004D616E75616C6C792050
:102B10004275696C64204D657368004732394939E4
:102B200039390A4732395032425430004275696CA3
:102B300064204D65736800372E205361766520420E
:102B40006564204D65736800362E2046696E6520E9
:102B500054756E6520416C6C0047323950345239DF
:102B600039395400352E2056616C696461746520D2
:102B70004D65736800342E2046696E652054756E6D
:102B80006520416C6C004732395034523939395420
:102B900000332E2056616C6964617465204D657345
:102BA0006800322E20536D6172742046696C6C2D62
:102BB000696E004732395033543000312E2042754F
:102BC000696C6420436F6C64204D65736800473204
:102BD000394E503100556E696669656420426564FE
:102BE000204C6576656C696E6700466164652048B7
:102BF0006569676874004F75747075742055424C30
:102C000020496E666F00473239570055424C2054B8
:102C10006F6F6C73004F7574707574204D657368B9
:102C2000204D6170004D6573682053746F72616749
:102C300065004D6573682045646974005374657060
:102C40002D42792D537465702055424C00416374B8
:102C500069766174652055424C0047323941004421
:102C60006561637469766174652055424C00473232
:102C70003944004D6F74696F6E00486F6D696E67FF
:102C8000204661696C6564006F70656E005452493E
:102C9000474745524544003A20007A5F6D696E000F
:102CA000795F6D696E00785F6D696E005265706F57
:102CB0007274696E6720656E6473746F70207374CC
:102CC000617475730A0020746F6F206C6F6E6720DB
:102CD000657874727573696F6E2070726576656E53
:102CE0007465640A0020636F6C6420657874727583
:102CF00073696F6E2070726576656E7465640A0024
:102D0000486F6D652025732573257320466972739E
:102D100074005761726E696E673A20486F6D696E14
:102D2000672042756D702044697669736F72203C2C
:102D300020310A0002020400000000000000000030
:102D4000000000000070430000704300007A430060
:102D50000000410000004100000040FFFFFF0000B4
:102D600000010000000100008000555555000000E2
:102D7000400033333300AAAA2A00499224000000FD
:102D80002000C7711C0099991900D14517005555AD
:102D900015003BB11300244912001111110000006D
:102DA00010000F0F0F00E3380E0043790D00CCCC5C
:102DB0000C00C3300C00E8A20B0064210B00AAAA8F
:102DC0000A00703D0A009DD80900427B0900922448
:102DD0000900DCD3080088880800104208000000C1
:102DE0000800F0C107008787070075500700711CB5
:102DF00007003EEB0600A1BC06006990060066666F
:102E00000600703E06006118060017F4050074D134
:102E100005005BB00500B2900500627205005555D3
:102E2000050078390500B81E0500050505004EECC3
:102E3000040087D40400A1BD040090A704004992B7
:102E40000400C17D0400EE690400C7560400444438
:102E500004005C320400082104004110040000005A
:102E600004003FF00300F8E0030026D20300C3C3D0
:102E70000300CCB503003AA803000A9B0300388E78
:102E80000300C08103009F750300D0690300505EFA
:102E900003001D53030034480300913D0300333306
:102EA000030016290300381F030097150300300C98
:102EB0000300030303000BFA020049F10200BAE821
:102EC00002005CE002002DD802002DD0020059C89B
:102ED0000200B0C0020031B90200DAB10200AAAAB1
:102EE0000200A0A30200BC9C0200FA9502005C8FC5
:102EF0000200DF88020082820200457C0200277601
:102F0000020027700200436A02007C640200D05E67
:102F100002003F590200C8530200FFFDFCFAF8F618
:102F2000F4F2F0EEECEAE9E7E5E3E1E0DEDCDAD941
:102F3000D7D5D4D2D0CFCDCBCAC8C7C5C3C2C0BFE6
:102F4000BDBCBAB9B7B6B4B3B2B0AFADACAAA9A85C
:102F5000A6A5A4A2A1A09E9D9C9A999897959493AA
:102F600092908F8E8D8B8A898887868483828180D8
:102F70007F7E7D7B7A797877767574737271706FE6
:102F80006E6D6C6B6A696867666564636261605FD9
:102F90005E5D5C5B5A5958585756555453525150C0
:102FA000504F4E4D4C4B4A4A49484746464544438C
:102FB000424241403F3E3E3D3C3B3B3A3938383748
:102FC000363535343332323130302F2E2E2D2C2BF6
:102FD0002B2A292928272726252524232322212196
:102FE00020201F1E1E1D1C1C1B1B1A191918181728
:102FF0001616151514131312121111100F0F0E0EB1
:103000000D0D0C0C0B0A0A0909080807070606052E
:1030100005040403030202010000000070430000E5
:10302000704300007A430000000000000000000030
:10303000000053657474696E67732053746F726512
:103040006400454550524F4D20496E697469616C6A
:10305000697A65640A003F556E61626C6520746F21
:103060002073617665206D65736820646174612EDC
:103070000A003F556E61626C6520746F206C6F6151
:1030800064206D65736820646174612E0A00556E5A
:10309000696669656420426564204C6576656C6983
:1030A0006E67003B20003A0A0020204D3630332066
:1030B000002055004C0046696C616D656E74206C93
:1030C0006F61642F756E6C6F6164206C656E6774E0
:1030D00068733A0020204D393030204B004C696E27
:1030E00065617220416476616E63653A0020204D0F
:1030F0003835312058005A2D50726F6265204F6666
:10310000667365740020204D343133205300506FB6
:103110007765722D4C6F7373205265636F7665729D
:10312000793A0020204D3235302043004C43442072
:10313000436F6E74726173743A002044002049003A
:1031400020204D33303420500020440020490020FE
:10315000204D333031205000504944207365747441
:10316000696E67733A0020460020480020204D31E8
:1031700034352053004D6174657269616C20686557
:103180006174757020706172616D65746572733AF7
:1031900000206D65736865732E0A0A00454550521C
:1031A0004F4D2063616E20686F6C64200041637432
:1031B000697665204D65736820536C6F743A200002
:1031C00020204D34323020530020204D3230362024
:1031D0005800486F6D65206F66667365743A00200D
:1031E000580020530020204D3230352042004164E9
:1031F00076616E6365643A20423C6D696E5F73650B
:10320000676D656E745F74696D655F75733E20539D
:103210003C6D696E5F66656564726174653E2054DD
:103220003C6D696E5F74726176656C5F666565643E
:10323000726174653E20583C6D61785F785F6A65A5
:10324000726B3E20593C6D61785F795F6A65726B85
:103250003E205A3C6D61785F7A5F6A65726B3E20F2
:10326000453C6D61785F655F6A65726B3E00205416
:103270000020520020204D32303420500041636342
:10328000656C65726174696F6E2028756E69747300
:103290002F7332293A20503C7072696E745F6163FB
:1032A00063656C3E20523C726574726163745F6149
:1032B0006363656C3E20543C74726176656C5F613B
:1032C0006363656C3E0020204D3230312058004D44
:1032D0006178696D756D20416363656C65726174B9
:1032E000696F6E2028756E6974732F7332293A00E6
:1032F00020204D3230332058004D6178696D756D56
:10330000206665656472617465732028756E6974E2
:10331000732F73293A00537465707320706572209F
:10332000756E69743A0020440020204D3230302000
:1033300053002044697361626C65640A0046696CDD
:10334000616D656E742073657474696E67733A009D
:1033500020204D3134392043203B20556E69747351
:1033600020696E2043656C736975730A0020286DAF
:103370006D29002020473231202020203B20556E2F
:1033800069747320696E206D6D003F4D6573682010
:10339000746F6F2062696720666F722045455052D6
:1033A0004F4D2E0A0000803B4400803B440000202B
:1033B00041000096420000A0420000A0420000C868
:1033C000430000BE42D0070000D0070000640000A8
:1033D000004B00000024F4D43050C38E20C2A24021
:1033E00017828B7011127A910D816CD90AA861E154
:1033F00008C7586607615143061E4B5D05C145A7C6
:10340000041A411104093D9803713931034036DB38
:103410000265339102D4305402802E1D02632CEEDB
:1034200001752AC501B028A001102781018F2564EC
:10343000012B244B01E0223401AC211F018D200D12
:1034400001801FFC00841EED00971DDF00B81CD218
:1034500000E61BC600201BBC00641AB200B219A80B
:10346000000A19A0006A189900D117910040178B23
:1034700000B516840031167E00B31579003A157335
:1034800000C7146F0058146A00EE136600881363B7
:103490000025135E00C7125B006C12570015125412
:1034A00000C111510070114F0021114B00D610497D
:1034B000008D1047004610440002104200C00F402B
:1034C00000800F3E00420F3C00060F3B00CB0E3841
:1034D00000930E37005C0E3500270E3400F30D32DA
:1034E00000C10D3100900D3000600D2E00320D2D09
:1034F00000050D2C00D90C2B00AE0C2900850C29E1
:10350000005C0C2700350C27000E0C2600E80B246D
:1035100000C40B2400A00B23007D0B23005A0B21B9
:1035200000390B2100180B2000F80A1F00D90A1ED1
:1035300000BB0A1E009D0A1D00800A1D00630A1CB4
:1035400000470A1B002C0A1B00110A1A00F7091A6F
:1035500000DD091900C4091900AB09190092091707
:10356000007B091800630917004C0916003609167C
:1035700000200916000A091500F5081500E00814D6
:1035800000CC081400B8081400A408140090081314
:10359000007D0812006B081300580812004608123C
:1035A000003408110023081100120811000108114D
:1035B00000F0071000E0071000D0071000C007104F
:1035C00000B0070F00A107100091070E0083070F3E
:1035D0000074070F0065070E0057070E0049070E1D
:1035E000003B070D002E070E0020070D0013070DEE
:1035F0000006070D00F9060C00ED060D00E0060CB4
:1036000000D4060C00C8060C00BC060C00B0060C6A
:1036100000A4060B0099060C008D060B0082060B19
:103620000077060B006C060B0061060A0057060BBC
:10363000004C060A0042060A0038060A002E060A56
:103640000024060A001A060A001006090007060AE6
:1036500000FD050900F4050900EB050900E2050974
:1036600000D9050900D0050900C7050900BE0509F4
:1036700000B5050800AD050800A50509009C050872
:1036800000940508008C050800840508007C0508E6
:1036900000740508006C050700650508005D050756
:1036A00000560508004E05070047050700400508BD
:1036B0000038050700310507002A05070023050724
:1036C000001C050600160507000F05070008050683
:1036D0000002050700FB040600F5040700EE0406DF
:1036E00000E8040600E2040700DB040600D5040637
:1036F00000CF040600C9040600C3040600BD04068A
:1037000000B7040600B1040500AC040600A60406D8
:1037100000A00405009B0406009504050090040623
:10372000008A04050085040500800406007A04056B
:103730000075040500700405006B040500660405AF
:1037400000610405005C04050057040500520405EF
:10375000004D04050048040500430405003E040430
:10376000003A04050035040500300404002C04056B
:103770000027040400230405001E0404001A0404A6
:103780000016040500110404000D040400090405DA
:10379000000404040000040400FC030400F8030413
:1037A00000F4030400F0030400EC030400E8030445
:1037B00000E4030400E0030400DC030400D8030475
:1037C00000D4030400D0030400CC030400C80303A6
:1037D00000C503030024F404D9201BC40C5C0E981C
:1037E00004C4095F0265077101F405F900FB04B325
:1037F0000048048700C103690058035500030345CE
:1038000000BE023A008402310053022A0029022538
:103810000004022000E4011C00C8011900AF0117D8
:10382000009801140084011300710110006101105F
:103830000051010E0043010D0036010B002B010B5E
:103840000020010B00150109000C0109000301080B
:1038500000FB000800F3000800EB000700E400068E
:1038600000DE000600D8000600D2000600CC0005ED
:1038700000C7000500C2000500BD000400B9000437
:1038800000B5000400B1000400AD000400A900046C
:1038900000A5000300A20003009F0004009B00039A
:1038A00000980003009500020093000300900003BD
:1038B000008D0002008B00030088000200860002D9
:1038C0000084000300810002007F0002007D0002EE
:1038D000007B000200790002007700010076000200
:1038E000007400020072000100710002006F00020B
:1038F000006D0001006C0002006A00010069000216
:10390000006700010066000100650001006400021C
:10391000006200010061000100600001005F000220
:10392000005D0001005C0001005B0001005A000125
:103930000059000100580001005700010056000125
:103940000055000100540001005300000053000125
:10395000005200010051000100500001004F000121
:10396000004E0000004E0001004D0001004C00011F
:10397000004B0000004B0001004A0001004900011B
:103980000048000000480001004700010046000018
:103990000046000100450000004500010044000110
:1039A000004300000043000100420000004200010B
:1039B000004100000041000100400001003F000004
:1039C000003F0001003E0000003E0001003D0000FD
:1039D000003D0001003C0000003C0000003C0001F4
:1039E000003B0000003B0001003A0000003A0001EB
:1039F00000390000003900010038000000380000E4
:103A000000380001003700000037000100360000D8
:103A100000360000003600010035000000350000CF
:103A200000350001003400000034000000340001C3
:103A300000330000003300000033000100320000BA
:103A400000320000003200010031000000310000AF
:103A500000310001003000000030000000300001A3
:103A6000002F0000002F0000002F0000002F000199
:103A7000002E0000002E0000002E0001002D00008E
:103A8000002D0000002D0000002D0001002C000082
:103A9000002C0000002C0000002C0001002B000076
:103AA000002B0000002B0000002B0001002A00006A
:103AB000002A0000002A0000002A0001002900005E
:103AC0000029000000290000002900000029000151
:103AD0000028000000280000002800000028000046
:103AE0000028000100270000002700000027000038
:103AF000002700000027000100260000002600002B
:103B0000002600000026000000260001002500001D
:103B10000025000000250000002500000025000011
:103B20000025000100240000002400000024000003
:103B300000240000002400010023000000230000F6
:103B400000230000002300000023000000230000E9
:103B500000230001002200000022000000220000DB
:103B600000220000002200000022000100210000CD
:103B700000210000002100000021000000210000C1
:103B800000210000002100010020000000200000B2
:103B900000200000002000000020000000200000A5
:103BA0000020000000200001001F0000001F000096
:103BB000001F0000001F0000001F0000001F000089
:103BC000001F0001001E0000001E0000001E00007B
:103BD000001E000000232C0000B822000056180030
:103BE000003A0F0000B8080000B1040000710200A4
:103BF000003E01000020436F756E7420583A004269
:103C0000656400453100626564002C20737973742B
:103C1000656D2073746F70706564212048656174F0
:103C200065725F49443A200048656174696E672097
:103C30004661696C65640048656174696E672066F9
:103C400061696C6564004D3131322053687574646C
:103C50006F776E001000C90210012C014001220193
:103C600070011801B0010E01F00104015002FA00C8
:103C7000B002F0003003E600D003DC009004D20074
:103C80007005C800A006BE000008B400B009AA0074
:103C9000D00BA000600E960060118C000015820011
:103CA00020197800C01D6E00A0226400B0275A00C1
:103CB000902C500000314600E0343C0010383200B7
:103CC000903A2800603C1E00A03D1400803E0A008F
:103CD000203F0000544845524D414C2052554E4122
:103CE00057415900546865726D616C2052756E6160
:103CF000776179004572723A204D415854454D50D4
:103D0000004D415854454D50207472696767657283
:103D10006564004572723A204D494E54454D50003D
:103D20004D494E54454D5020747269676765726500
:103D30006400202F002042403A0020403A002057E3
:103D40003A0020573A00496E76616C6964206578C4
:103D50007472756465720A007C3C3E5E2B3D3F2F99
:103D60005B5D3B2C2A225C0043616E6E6F74206F9A
:103D700070656E2073756264697220005344204937
:103D80006E6974204661696C0053442063617264FB
:103D9000206F6B0A006F70656E526F6F74206661E2
:103DA000696C65640A00766F6C756D652E696E6965
:103DB00074206661696C65640A004E6F205344206C
:103DC000636172640A000A4D3234004D323320259B
:103DD00073002E0A006F70656E206661696C656401
:103DE0002C2046696C653A200046696C6520736535
:103DF0006C65637465640A002053697A653A200033
:103E000046696C65206F70656E65643A2000454EAA
:103E10004420535542524F5554494E450A002220E2
:103E2000706F73002220706172656E743A220053C5
:103E30005542524F5554494E452043414C4C2074F5
:103E400061726765743A220053756263616C6C201D
:103E50004F766572666C6F7700457863656564655B
:103E600064206D617820535542524F5554494E4558
:103E70002064657074683A002E0A0044656C6574AD
:103E8000696F6E206661696C65642C2046696C659B
:103E90003A200046696C652064656C657465643A17
:103EA00000363726033C3D380E2E303E121A1C18C1
:103EB0000AFF4309070844000124F404D9201BC465
:103EC0000C5C0E9804C4095F0265077101F405F9E2
:103ED00000FB04B30048048700C103690058035580
:103EE0000003034500BE023A008402310053022A57
:103EF000002902250004022000E4011C00C8011969
:103F000000AF011700980114008401130071011023
:103F1000006101100051010E0043010D0036010B3C
:103F2000002B010B0020010B00150109000C0109F9
:103F30000003010800FB000800F3000800EB000785
:103F400000E4000600DE000600D8000600D20006ED
:103F500000CC000500C7000500C2000500BD00043C
:103F600000B9000400B5000400B1000400AD000475
:103F700000A9000400A5000300A20003009F0004A4
:103F8000009B0003009800030095000200930003CB
:103F900000900003008D0002008B000300880002E7
:103FA000008600020084000300810002007F0002FE
:103FB000007D0002007B0002007900020077000112
:103FC000007600020074000200720001007100021D
:103FD000006F0002006D0001006C0002006A000129
:103FE0000069000200670001006600010065000131
:103FF0000064000200620001006100010060000135
:10400000005F0002005D0001005C0001005B000138
:10401000005A00010059000100580001005700013A
:10402000005600010055000100540001005300003B
:104030000053000100520001005100010050000136
:10404000004F0001004E0000004E0001004D000135
:10405000004C0001004B0000004B0001004A000131
:10406000004900010048000000480001004700012D
:104070000046000000460001004500000045000128
:104080000044000100430000004300010042000022
:104090000042000100410000004100010040000119
:1040A000003F0000003F0001003E0000003E000114
:1040B000003D0000003D0001003C0000003C00000D
:1040C000003C0001003B0000003B0001003A000002
:1040D000003A0001003900000039000100380000FA
:1040E00000380000003800010037000000370001F0
:1040F00000360000003600000036000100350000E8
:1041000000350000003500010034000000340000DC
:1041100000340001003300000033000000330001D0
:1041200000320000003200000032000100310000C7
:1041300000310000003100010030000000300000BC
:1041400000300001002F0000002F0000002F0000B1
:10415000002F0001002E0000002E0000002E0001A4
:10416000002D0000002D0000002D0000002D00019A
:10417000002C0000002C0000002C0000002C00018E
:10418000002B0000002B0000002B0000002B000182
:10419000002A0000002A0000002A0000002A000176
:1041A000002900000029000000290000002900006B
:1041B000002900010028000000280000002800005D
:1041C0000028000000280001002700000027000050
:1041D0000027000000270000002700010026000043
:1041E0000026000000260000002600000026000136
:1041F000002500000025000000250000002500002B
:10420000002500000025000100240000002400001B
:10421000002400000024000000240001002300000E
:104220000023000000230000002300000023000002
:1042300000230000002300010022000000220000F3
:1042400000220000002200000022000000220001E5
:1042500000210000002100000021000000210000DA
:1042600000210000002100000021000100200000CA
:1042700000200000002000000020000000200000BE
:10428000002000000020000000200001001F0000AE
:10429000001F0000001F0000001F0000001F0000A2
:1042A000001F0000001F0001001E0000001E000093
:1042B000001E0000001E00000024F4D43050C38E05
:1042C00020C2A24017828B7011127A910D816CD995
:1042D0000AA861E108C7586607615143061E4B5D95
:1042E00005C145A7041A411104093D9803713931EC
:1042F000034036DB0265339102D4305402802E1D18
:1043000002632CEE01752AC501B028A00110278197
:10431000018F2564012B244B01E0223401AC211FC5
:10432000018D200D01801FFC00841EED00971DDF14
:1043300000B81CD200E61BC600201BBC00641AB2E9
:1043400000B219A8000A19A0006A189900D11791A3
:104350000040178B00B516840031167E00B3157926
:10436000003A157300C7146F0058146A00EE136604
:10437000008813630025135E00C7125B006C1257A0
:104380000015125400C111510070114F0021114B42
:1043900000D61049008D104700461044000210421C
:1043A00000C00F4000800F3E00420F3C00060F3B54
:1043B00000CB0E3800930E37005C0E3500270E340C
:1043C00000F30D3200C10D3100900D3000600D2E54
:1043D00000320D2D00050D2C00D90C2B00AE0C2940
:1043E00000850C29005C0C2700350C27000E0C26DC
:1043F00000E80B2400C40B2400A00B23007D0B233A
:10440000005A0B2100390B2100180B2000F80A1F5D
:1044100000D90A1E00BB0A1E009D0A1D00800A1D4D
:1044200000630A1C00470A1B002C0A1B00110A1A11
:1044300000F7091A00DD091900C4091900AB0919B0
:1044400000920917007B091800630917004C091630
:104450000036091600200916000A091500F508158E
:1044600000E0081400CC081400B8081400A40814D4
:1044700000900813007D0812006B08130058081202
:104480000046081200340811002308110012081118
:104490000001081100F0071000E0071000D007101D
:1044A00000C0071000B0070F00A107100091070E11
:1044B0000083070F0074070F0065070E0057070EF3
:1044C0000049070E003B070D002E070E0020070DC8
:1044D0000013070D0006070D00F9060C00ED060D90
:1044E00000E0060C00D4060C00C8060C00BC060C4C
:1044F00000B0060C00A4060B0099060C008D060BFC
:104500000082060B0077060B006C060B0061060AA2
:104510000057060B004C060A0042060A0038060A3D
:10452000002E060A0024060A001A060A00100609D0
:104530000007060A00FD050900F4050900EB05095E
:1045400000E2050900D9050900D0050900C70509E1
:1045500000BE050900B5050800AD050800A5050960
:10456000009C050800940508008C050800840508D7
:10457000007C050800740508006C05070065050847
:10458000005D050700560508004E050700470507B2
:10459000004005080038050700310507002A050717
:1045A00000230507001C050600160507000F050778
:1045B000000805060002050700FB040600F50407D5
:1045C00000EE040600E8040600E2040700DB04062F
:1045D00000D5040600CF040600C9040600C3040683
:1045E00000BD040600B7040600B1040500AC0406D3
:1045F00000A6040600A00405009B0406009504051F
:1046000000900406008A0405008504050080040665
:10461000007A04050075040500700405006B0405AC
:104620000066040500610405005C040500570405EC
:1046300000520405004D040500480405004304052C
:10464000003E0404003A040500350405003004046B
:10465000002C04050027040400230405001E0404A4
:10466000001A04040016040500110404000D0404DB
:1046700000090405000404040000040400FC030411
:1046800000F8030400F4030400F0030400EC030446
:1046900000E8030400E4030400E0030400DC030476
:1046A00000D8030400D4030400D0030400CC0304A6
:1046B00000C8030300C5030300726F746174696F5F
:1046C0006E206D61747269783A0A0024F404D9206E
:1046D0001BC40C5C0E9804C4095F0265077101F4E9
:1046E00005F900FB04B30048048700C103690058C2
:1046F00003550003034500BE023A00840231005313
:10470000022A002902250004022000E4011C00C83E
:10471000011900AF01170098011400840113007102
:104720000110006101100051010E0043010D00361F
:10473000010B002B010B0020010B00150109000CDF
:1047400001090003010800FB000800F3000800EB6A
:10475000000700E4000600DE000600D8000600D2D4
:10476000000600CC000500C7000500C2000500BD22
:10477000000400B9000400B5000400B1000400AD5D
:10478000000400A9000400A5000300A20003009F8C
:104790000004009B000300980003009500020093B2
:1047A000000300900003008D0002008B00030088CE
:1047B0000002008600020084000300810002007FE6
:1047C0000002007D0002007B0002007900020077F9
:1047D0000001007600020074000200720001007106
:1047E0000002006F0002006D0001006C0002006A10
:1047F0000001006900020067000100660001006519
:10480000000100640002006200010061000100601C
:104810000001005F0002005D0001005C0001005B20
:104820000001005A00010059000100580001005722
:104830000001005600010055000100540001005322
:10484000000000530001005200010051000100501F
:104850000001004F0001004E0000004E0001004D1D
:104860000001004C0001004B0000004B0001004A19
:104870000001004900010048000000480001004715
:104880000001004600000046000100450000004510
:104890000001004400010043000000430001004209
:1048A0000000004200010041000000410001004002
:1048B0000001003F0000003F0001003E0000003EFC
:1048C0000001003D0000003D0001003C0000003CF4
:1048D0000000003C0001003B0000003B0001003AEA
:1048E0000000003A000100390000003900010038E2
:1048F00000000038000000380001003700000037D9
:1049000000010036000000360000003600010035CE
:1049100000000035000000350001003400000034C4
:1049200000000034000100330000003300000033B9
:1049300000010032000000320000003200010031AE
:1049400000000031000000310001003000000030A4
:10495000000000300001002F0000002F0000002F99
:104960000000002F0001002E0000002E0000002E8D
:104970000001002D0000002D0000002D0000002D82
:104980000001002C0000002C0000002C0000002C76
:104990000001002B0000002B0000002B0000002B6A
:1049A0000001002A0000002A0000002A0000002A5E
:1049B0000001002900000029000000290000002952
:1049C0000000002900010028000000280000002845
:1049D0000000002800000028000100270000002738
:1049E000000000270000002700000027000100262B
:1049F000000000260000002600000026000000261F
:104A00000001002500000025000000250000002511
:104A10000000002500000025000100240000002403
:104A200000000024000000240000002400010023F6
:104A300000000023000000230000002300000023EA
:104A400000000023000000230001002200000022DB
:104A500000000022000000220000002200000022CE
:104A600000010021000000210000002100000021C1
:104A700000000021000000210000002100010020B2
:104A800000000020000000200000002000000020A6
:104A90000000002000000020000000200001001F96
:104AA0000000001F0000001F0000001F0000001F8A
:104AB0000000001F0000001F0001001E0000001E7B
:104AC0000000001E0000001E00000024F4D430503E
:104AD000C38E20C2A24017828B7011127A910D8171
:104AE0006CD90AA861E108C7586607615143061EE0
:104AF0004B5D05C145A7041A411104093D98037196
:104B00003931034036DB0265339102D430540280E0
:104B10002E1D02632CEE01752AC501B028A00110DC
:104B20002781018F2564012B244B01E0223401AC45
:104B3000211F018D200D01801FFC00841EED0097B8
:104B40001DDF00B81CD200E61BC600201BBC0064A1
:104B50001AB200B219A8000A19A0006A189900D167
:104B600017910040178B00B516840031167E00B3F4
:104B70001579003A157300C7146F0058146A00EED7
:104B80001366008813630025135E00C7125B006C78
:104B900012570015125400C111510070114F00211D
:104BA000114B00D61049008D1047004610440002FA
:104BB000104200C00F4000800F3E00420F3C000634
:104BC0000F3B00CB0E3800930E37005C0E350027EC
:104BD0000E3400F30D3200C10D3100900D30006035
:104BE0000D2E00320D2D00050D2C00D90C2B00AE22
:104BF0000C2900850C29005C0C2700350C27000EC1
:104C00000C2600E80B2400C40B2400A00B23007D1D
:104C10000B23005A0B2100390B2100180B2000F840
:104C20000A1F00D90A1E00BB0A1E009D0A1D008033
:104C30000A1D00630A1C00470A1B002C0A1B0011F6
:104C40000A1A00F7091A00DD091900C4091900AB96
:104C5000091900920917007B091800630917004C15
:104C600009160036091600200916000A091500F574
:104C7000081500E0081400CC081400B8081400A4BB
:104C8000081400900813007D0812006B08130058E8
:104C900008120046081200340811002308110012FF
:104CA00008110001081100F0071000E0071000D003
:104CB000071000C0071000B0070F00A107100091F7
:104CC000070E0083070F0074070F0065070E0057DB
:104CD000070E0049070E003B070D002E070E0020AF
:104CE000070D0013070D0006070D00F9060C00ED77
:104CF000060D00E0060C00D4060C00C8060C00BC33
:104D0000060C00B0060C00A4060B0099060C008DE2
:104D1000060B0082060B0077060B006C060B006189
:104D2000060A0057060B004C060A0042060A003825
:104D3000060A002E060A0024060A001A060A0010B7
:104D400006090007060A00FD050900F4050900EB45
:104D5000050900E2050900D9050900D0050900C7C9
:104D6000050900BE050900B5050800AD050800A548
:104D70000509009C050800940508008C05080084BE
:104D80000508007C050800740508006C050700652F
:104D90000508005D050700560508004E0507004799
:104DA0000507004005080038050700310507002AFF
:104DB000050700230507001C050600160507000F60
:104DC0000507000805060002050700FB040600F5BC
:104DD000040700EE040600E8040600E2040700DB16
:104DE000040600D5040600CF040600C9040600C36B
:104DF000040600BD040600B7040600B1040500ACBB
:104E0000040600A6040600A00405009B0406009505
:104E1000040500900406008A04050085040500804E
:104E20000406007A04050075040500700405006B93
:104E300004050066040500610405005C04050057D4
:104E4000040500520405004D040500480405004314
:104E50000405003E0404003A040500350405003052
:104E60000404002C04050027040400230405001E8C
:104E70000404001A04040016040500110404000DC3
:104E8000040400090405000404040000040400FCF8
:104E9000030400F8030400F4030400F0030400EC2E
:104EA000030400E8030400E4030400E0030400DC5E
:104EB000030400D8030400D4030400D0030400CC8E
:104EC000030400C8030300C503030024F404D9202D
:104ED0001BC40C5C0E9804C4095F0265077101F4E1
:104EE00005F900FB04B30048048700C103690058BA
:104EF00003550003034500BE023A0084023100530B
:104F0000022A002902250004022000E4011C00C836
:104F1000011900AF011700980114008401130071FA
:104F20000110006101100051010E0043010D003617
:104F3000010B002B010B0020010B00150109000CD7
:104F400001090003010800FB000800F3000800EB62
:104F5000000700E4000600DE000600D8000600D2CC
:104F6000000600CC000500C7000500C2000500BD1A
:104F7000000400B9000400B5000400B1000400AD55
:104F8000000400A9000400A5000300A20003009F84
:104F90000004009B000300980003009500020093AA
:104FA000000300900003008D0002008B00030088C6
:104FB0000002008600020084000300810002007FDE
:104FC0000002007D0002007B0002007900020077F1
:104FD00000010076000200740002007200010071FE
:104FE0000002006F0002006D0001006C0002006A08
:104FF0000001006900020067000100660001006511
:105000000001006400020062000100610001006014
:105010000001005F0002005D0001005C0001005B18
:105020000001005A0001005900010058000100571A
:10503000000100560001005500010054000100531A
:105040000000005300010052000100510001005017
:105050000001004F0001004E0000004E0001004D15
:105060000001004C0001004B0000004B0001004A11
:10507000000100490001004800000048000100470D
:105080000001004600000046000100450000004508
:105090000001004400010043000000430001004201
:1050A00000000042000100410000004100010040FA
:1050B0000001003F0000003F0001003E0000003EF4
:1050C0000001003D0000003D0001003C0000003CEC
:1050D0000000003C0001003B0000003B0001003AE2
:1050E0000000003A000100390000003900010038DA
:1050F00000000038000000380001003700000037D1
:1051000000010036000000360000003600010035C6
:1051100000000035000000350001003400000034BC
:1051200000000034000100330000003300000033B1
:1051300000010032000000320000003200010031A6
:10514000000000310000003100010030000000309C
:10515000000000300001002F0000002F0000002F91
:105160000000002F0001002E0000002E0000002E85
:105170000001002D0000002D0000002D0000002D7A
:105180000001002C0000002C0000002C0000002C6E
:105190000001002B0000002B0000002B0000002B62
:1051A0000001002A0000002A0000002A0000002A56
:1051B000000100290000002900000029000000294A
:1051C000000000290001002800000028000000283D
:1051D0000000002800000028000100270000002730
:1051E0000000002700000027000000270001002623
:1051F0000000002600000026000000260000002617
:105200000001002500000025000000250000002509
:1052100000000025000000250001002400000024FB
:1052200000000024000000240000002400010023EE
:1052300000000023000000230000002300000023E2
:1052400000000023000000230001002200000022D3
:1052500000000022000000220000002200000022C6
:1052600000010021000000210000002100000021B9
:1052700000000021000000210000002100010020AA
:10528000000000200000002000000020000000209E
:105290000000002000000020000000200001001F8E
:1052A0000000001F0000001F0000001F0000001F82
:1052B0000000001F0000001F0001001E0000001E73
:1052C0000000001E0000001E00000024F4D4305036
:1052D000C38E20C2A24017828B7011127A910D8169
:1052E0006CD90AA861E108C7586607615143061ED8
:1052F0004B5D05C145A7041A411104093D9803718E
:105300003931034036DB0265339102D430540280D8
:105310002E1D02632CEE01752AC501B028A00110D4
:105320002781018F2564012B244B01E0223401AC3D
:10533000211F018D200D01801FFC00841EED0097B0
:105340001DDF00B81CD200E61BC600201BBC006499
:105350001AB200B219A8000A19A0006A189900D15F
:1053600017910040178B00B516840031167E00B3EC
:105370001579003A157300C7146F0058146A00EECF
:105380001366008813630025135E00C7125B006C70
:1053900012570015125400C111510070114F002115
:1053A000114B00D61049008D1047004610440002F2
:1053B000104200C00F4000800F3E00420F3C00062C
:1053C0000F3B00CB0E3800930E37005C0E350027E4
:1053D0000E3400F30D3200C10D3100900D3000602D
:1053E0000D2E00320D2D00050D2C00D90C2B00AE1A
:1053F0000C2900850C29005C0C2700350C27000EB9
:105400000C2600E80B2400C40B2400A00B23007D15
:105410000B23005A0B2100390B2100180B2000F838
:105420000A1F00D90A1E00BB0A1E009D0A1D00802B
:105430000A1D00630A1C00470A1B002C0A1B0011EE
:105440000A1A00F7091A00DD091900C4091900AB8E
:10545000091900920917007B091800630917004C0D
:1054600009160036091600200916000A091500F56C
:10547000081500E0081400CC081400B8081400A4B3
:10548000081400900813007D0812006B08130058E0
:1054900008120046081200340811002308110012F7
:1054A00008110001081100F0071000E0071000D0FB
:1054B000071000C0071000B0070F00A107100091EF
:1054C000070E0083070F0074070F0065070E0057D3
:1054D000070E0049070E003B070D002E070E0020A7
:1054E000070D0013070D0006070D00F9060C00ED6F
:1054F000060D00E0060C00D4060C00C8060C00BC2B
:10550000060C00B0060C00A4060B0099060C008DDA
:10551000060B0082060B0077060B006C060B006181
:10552000060A0057060B004C060A0042060A00381D
:10553000060A002E060A0024060A001A060A0010AF
:1055400006090007060A00FD050900F4050900EB3D
:10555000050900E2050900D9050900D0050900C7C1
:10556000050900BE050900B5050800AD050800A540
:105570000509009C050800940508008C05080084B6
:105580000508007C050800740508006C0507006527
:105590000508005D050700560508004E0507004791
:1055A0000507004005080038050700310507002AF7
:1055B000050700230507001C050600160507000F58
:1055C0000507000805060002050700FB040600F5B4
:1055D000040700EE040600E8040600E2040700DB0E
:1055E000040600D5040600CF040600C9040600C363
:1055F000040600BD040600B7040600B1040500ACB3
:10560000040600A6040600A00405009B04060095FD
:10561000040500900406008A040500850405008046
:105620000406007A04050075040500700405006B8B
:1056300004050066040500610405005C04050057CC
:10564000040500520405004D04050048040500430C
:105650000405003E0404003A04050035040500304A
:105660000404002C04050027040400230405001E84
:105670000404001A04040016040500110404000DBB
:10568000040400090405000404040000040400FCF0
:10569000030400F8030400F4030400F0030400EC26
:1056A000030400E8030400E4030400E0030400DC56
:1056B000030400D8030400D4030400D0030400CC86
:1056C000030400C8030300C503030070012C01900C
:1056D000012701B0012201C0011D01F001180110D4
:1056E00002130130020E016002090190020401C0A0
:1056F00002FF000003FA004003F5008003F000D031
:1057000003EB002004E6007004E100E004DC00404C
:1057100005D700C005D2004006CD00D006C80080E5
:1057200007C3003008BE00F008B900C009B400B0DB
:105730000AAF00B00BAA00D00CA500000EA00050CC
:105740000F9B00C01096005012910000148C00C0F6
:10575000158700B0178200B0197D00D01B780000BB
:105760001E730040206E0090226900F02464004007
:10577000275F0090295A00E02B5500102E50002082
:10578000304B0010324600E033410090353C0010B1
:1057900037370070383200A0392D00B03A2800A009
:1057A0003B2300603C1E00103D1900903D1400108A
:1057B0003E0F00703E0A00C03E0500003F00004062
:1057C0003FFBFF803FF6FFC03FF1FF1000C9021012
:1057D000012C014001220170011801B0010E01F0FD
:1057E0000104015002FA00B002F0003003E600D0DC
:1057F00003DC009004D2007005C800A006BE0000C3
:1058000008B400B009AA00D00BA000600E9600609A
:10581000118C000015820020197800C01D6E00A0B8
:10582000226400B0275A00902C500000314600E05E
:10583000343C0010383200903A2800603C1E00A032
:105840003D1400803E0A00203F00005A5F6D6F76D5
:10585000655F636F6D700A00473238580047323811
:1058600059004732385A004732384F0A4D343820F1
:10587000503130004D3834004732395034523939C4
:10588000395400473239503454004732380A4732CD
:105890003643504930004732380A47323643504980
:1058A00031004732394A30004732395033543000E2
:1058B0004732395032425430004732380A4D31397C
:1058C0003049300A4D31303949300A473239503188
:1058D0000A4D31303453300A4D31343053300047A3
:1058E00032380A4D31393049310A4D313039493178
:1058F0000A47323950310A4D31303453300A4D3174
:1059000034305330004732394E503100473239502D
:105910003143004732394900473239543000473269
:1059200039543100473239532D3100473239493922
:1059300039390A4732395032425430004732394EF1
:1059400050310047323950335430004732395034E7
:10595000523939395400473239503452393939546F
:105960000047323944004732394100473239570045
:10597000417869732000206D696E3A00206D61786E
:105980003A00416363656C65726174696F6E206C87
:10599000696D697465642E0A004641535400534C86
:1059A0004F5700050000060100040006010006052F
:1059B000000000060004004572726F722077726961
:1059C00074696E6720746F20454550524F4D210A0F
:1059D0000053544F505045442E20005072696E744D
:1059E00065722073746F70706564206475652074CF
:1059F0006F206572726F72732E204669782074680A
:105A000065206572726F7220616E64207573652007
:105A10004D39393920746F20726573746172742E38
:105A2000202854656D7065726174757265206973A4
:105A30002072657365742E2053657420697420612B
:105A4000667465722072657374617274696E672919
:105A50000A004E6F20436865636B73756D2077692C
:105A60007468206C696E65206E756D6265722C209D
:105A70004C617374204C696E653A20004E6F204370
:105A80006865636B73756D2077697468206C696EE7
:105A900065206E756D6265722C204C617374204CAC
:105AA000696E653A2000636865636B73756D206D80
:105AB00069736D617463682C204C617374204C6948
:105AC0006E653A20004C696E65204E756D62657298
:105AD000206973206E6F74204C617374204C696E62
:105AE00065204E756D6265722B312C204C6173748C
:105AF000204C696E653A20004D313130005365729B
:105B000069616C20737461747573206D69736D6164
:105B10007463680A00776169740A005344207265EF
:105B20006164206572726F720A00486F74656E64FA
:105B30002049646C652054696D656F757400486F09
:105B400074656E642049646C652054696D656F7579
:105B5000740A002121204B494C4C20636175736508
:105B600064206279204B494C4C20627574746F6ECE
:105B70002F70696E0A002121204B494C4C20636133
:105B80007573656420627920746F6F206D7563682A
:105B900020696E6163746976652074696D65202D76
:105BA0002063757272656E7420636F6D6D616E64D3
:105BB0003A20004D656469612052656D6F766564B9
:105BC000004D6564696120496E7365727465640097
:105BD0004D313030305300627573793A2070617501
:105BE00073656420666F7220696E7075740A006256
:105BF0007573793A2070617573656420666F7220E1
:105C0000757365720A00627573793A2070726F63FA
:105C1000657373696E670A00506C65617365205225
:105C200065736574005052494E5445522048414CAA
:105C30005445440025533A20255300706F77657210
:105C40006F6666004B494C4C45442E2000507269EB
:105C50006E7465722068616C7465642E206B696C6B
:105C60006C28292063616C6C6564210A0053544FD1
:105C7000505045442E20005072696E746572207336
:105C8000746F707065642064756520746F20657230
:105C9000726F72732E204669782074686520657271
:105CA000726F7220616E6420757365204D393939C9
:105CB00020746F20726573746172742E202854658D
:105CC0006D70657261747572652069732072657399
:105CD00065742E2053657420697420616674657242
:105CE0002072657374617274696E67290A00656356
:105CF000686F3A004572726F723A00204A002020A5
:105D00004D34323120490020204732392049393979
:105D1000390A006163746976650A00696E000020C3
:105D200053797374656D2076312E30312000202038
:105D3000207C0A004E414E0020202E2020200020F2
:105D40007C004C43443A0A004353563A0A0020660A
:105D50006F7220003A0A0A000A42656420546F708C
:105D60006F677261706879205265706F727400504D
:105D7000726F62696E67204661696C65640A0050E3
:105D8000726F62696E67204661696C656400205AB3
:105D90003A200020593A200042656420583A2000F9
:105DA0004732384C3000446F6E652E0A003F496E12
:105DB00076616C69642073746F7261676520736CBF
:105DC0006F742E0A3F557365203020746F20003F9A
:105DD000454550524F4D2073746F72616765206E58
:105DE0006F7420617661696C61626C652E0A004493
:105DF0006F6E652E0A003F496E76616C6964207390
:105E0000746F7261676520736C6F742E0A3F5573EF
:105E100065203020746F20003F454550524F4D2083
:105E200073746F72616765206E6F7420617661694B
:105E30006C61626C652E0A00473239205032206650
:105E4000696E69736865642E0A005859206F75740D
:105E500073696465207072696E7461626C6520722A
:105E600061646975732E0A003F4572726F72206912
:105E70006E20427573696E6573732043617264208E
:105E80006D6561737572656D656E742E0A004D6186
:105E90006E75616C6C792070726F62696E672075C7
:105EA0006E726561636861626C6520706F696E74A3
:105EB000732E0A00292E0A0A0050726F62696E67FB
:105EC0002061726F756E642028004D6573682069CB
:105ED0006E76616C6964617465642E2050726F62C5
:105EE000696E67206D6573682E0A004D65736820C2
:105EF0007A65726F65642E0A0044656661756C741C
:105F00002073746F7261676520736C6F742030202A
:105F100073656C65637465642E0A004C6F61646917
:105F20006E6720746573745F7061747465726E203F
:105F300076616C7565732E0A0A00496E76616C692C
:105F40006420746573745F7061747465726E20761A
:105F5000616C75652E20282D3120746F2032290A3E
:105F60000A0020696E76616C6964617465642E0A4A
:105F70000A004C6F636174696F6E7300456E7469DB
:105F80007265204D657368005374616E646172645C
:105F900020446576696174696F6E3A20004D6561D1
:105FA0006E204D657368204865696768743A200003
:105FB00023206F662073616D706C65733A20000A50
:105FC0004D657368206F6E6C7920706172746961C1
:105FD0006C6C7920706F70756C617465642E0A0A40
:105FE0000050726F62696E6720506F696E74002591
:105FF000532025692F2569002E0A002F0050726F4B
:1060000062696E67206D65736820706F696E7420B9
:106010000020616E642074616B652061206D656194
:10602000737572656D656E742E0A006D6D207468EF
:1060300069636B2E0A00427573696E657373204342
:10604000617264206973200052656D6F7665202649
:10605000204D656173757265204265640052656DFF
:106060006F7665207368696D00506C61636520739D
:1060700068696D20756E646572206E6F7A7A6C65E2
:10608000000A4D657368206F6E6C792070617274C0
:1060900069616C6C7920706F70756C617465642EC9
:1060A0000A004D65736820506F696E74204D6561FC
:1060B00073757265642061743A20004D6561737573
:1060C000726500506C616365205368696D202620FD
:1060D0004D656173757265004D6F76696E672074EA
:1060E0006F206E657874004D65736820456469742F
:1060F000696E672053746F7070656400446F6E65DD
:106100002045646974696E67204D6573680A0044B0
:106110006F6E652045646974696E67204D657368AC
:106120000046696E652054756E696E67204D657313
:10613000680028582C5929206F757473696465208C
:106140007072696E7461626C6520726164697573E6
:106150002E0A004F6666736574206F7574206F6633
:1061600020626F756E64732E20283020746F20318A
:10617000306D6D290A0A00496E76616C6964206D84
:10618000617020747970652E0A0A003F28462961E3
:1061900064652068656967687420666F722042656F
:1061A00064204C6576656C20436F72726563746918
:1061B0006F6E206E6F7420706C61757369626C65B0
:1061C0002E0A0A003F43616E27742061637469766A
:1061D00061746520616E64206465616374697661D1
:1061E0007465206174207468652073616D65207426
:1061F000696D652E0A0A00426F74682058202620B7
:1062000059206C6F636174696F6E73206D75737460
:10621000206265207370656369666965642E0A0A89
:10622000003F496E76616C6964206772696420730F
:10623000697A6520284A29207370656369666965F3
:10624000642028322D39292E0A0A003F2850296857
:106250006173652076616C756520696E76616C6925
:10626000642028302D36292E0A0A003F2856296539
:1062700072626F7365206C6576656C20696D706CF9
:1062800061757369626C652028302D34292E0A0AE5
:10629000003F285229657065746974696F6E2063C8
:1062A0006F756E7420696E76616C69642028312B7D
:1062B000292E0A0A00446F696E672047323900B2FE
:1062C00059AD59A859A3595D0A0062656420706CE4
:1062D000616E65206E6F726D616C203D205B0043C6
:1062E0006F756C64206E6F7420636F6D706C657475
:1062F00065204C53462100436F7272656374656478
:106300005F5A3D0025532025692F2569000A0A00A0
:106310002F0054696C74696E67206D657368207016
:106320006F696E7420003F4572726F722070726FD9
:1063300062696E6720706F696E742E2041626F72A1
:1063400074696E67206F7065726174696F6E2E0A72
:1063500000436F727265637465645F5A3D00255334
:1063600020332F330054696C74696E67206D657338
:10637000682028332F33290A00436F7272656374D3
:1063800065645F5A3D00255320322F330054696CF9
:1063900074696E67206D6573682028322F33290A6F
:1063A00000436F727265637465645F5A3D0054699F
:1063B0006C74696E6720506F696E740025532031CC
:1063C0002F330054696C74696E67206D65736820A3
:1063D00028312F33290A00646F6E650A00496E73F5
:1063E000756666696369656E7420646174610A002C
:1063F0000000803F66663A426666B842CCCC0943EC
:1064000066663743000065430000803F66663A4297
:106410006666B842CCCC09436666374300006543E4
:106420004578747261706F6C6174696E67206D6518
:1064300073682E2E2E0021212053544F502063616B
:106440006C6C65642062656361757365206F66209E
:10645000424C546F756368206572726F72202D20F4
:10646000726573746172742077697468204D39396C
:10647000390A0021212053544F502063616C6C6510
:10648000642062656361757365206F6620424C54B9
:106490006F756368206572726F72202D207265734C
:1064A000746172742077697468204D3939390A0033
:1064B0005072696E74696E67204F626A656374001A
:1064C0002553202569002F2F616374696F6E3A0090
:1064D000737461727400656E6400486F74656E64F5
:1064E00020746F6F20636F6C640A0053656E6420C4
:1064F0004D31303820746F20726573756D650A00F8
:10650000496E736572742066696C616D656E742086
:10651000616E642073656E64204D3130380A00521C
:10652000656865617420446F6E65005265686561D9
:1065300074696E672E2E2E0052656865617400487E
:1065400065617465722054696D656F75740053657B
:106550006E64204D31303820746F2068656174207E
:106560006E6F7A7A6C650A004E6F7A7A6C6520508D
:1065700061726B656400706175736564005061756C
:10658000736500726573756D656400526573756D32
:10659000696E67004732362043616E63656C6564DF
:1065A0000041425300504C41005344207072696EC8
:1065B00074696E67206279746520004E6F74205391
:1065C00044207072696E74696E670A002F61757479
:1065D0006F25632E670057726974696E6720746F48
:1065E0002066696C653A2000667265736800646FA6
:1065F000696E67002066696C653A20004E6F7720EF
:106600000002FD55555555555FFFFFFFFFFFFFFF8A
:10661000FFFFFE00000000003FFFFFFFFFFFFFFF46
:10662000FFFFFD000007FFFFFFFFFFFFFFFFFFFF72
:10663000FFFFFE07C00555555555555FFFFFFFFF8E
:10664000FFFFFC0A200600000000003FFFFFFFFFE5
:10665000FFFFFE141005000007FFFFFFFFFFFFFF15
:10666000FFFFFC28080607C00555555555555FFF27
:10667000FFFFFE5404040A200600000000003FFF54
:10668000FFFFFC600406141005000007FFFFFFFF7A
:10669000FFFFFE50040428080607C0055555555550
:1066A000555FFC6004065404040A20060000000044
:1066B000003FFE54041C6004061410050000000096
:1066C000001FFC28082E50040428080607C00001FB
:1066D000F03FFE1410546004065404040A20000223
:1066E000081FFC0A206654041C60040614100005F0
:1066F000043FFE07C05428082E5004042808000A4E
:10670000021FFC00002E14105460040654040015EF
:10671000013FFE00001C0A206654041C600400189F
:10672000011FFC00000607C05428082E5004001466
:10673000013FFE00000400002E14105460040018F5
:10674000011FFCFFFFFE00001C0A206654041C15FC
:10675000013FFED5555400000607C05428082A0AF8
:10676000021FFC84104600000400002E1410510586
:10677000043FFEC41044FFFFFE00001C0A2061021B
:10678000881FFC841046D5555400000607C05101EF
:10679000F03FFE84104484104600000400002A00EC
:1067A000001FFCC41046C41044FFFFFE00001C0084
:1067B000003FFE841044841046D55554000000006C
:1067C000001FFCD55556841044841046000000007C
:1067D000003FFCFFFFFCC41046C41044FFFFFFFF56
:1067E000FF9FFE000006841044841046D555555581
:1067F00055BFFD555554D555568410448410410459
:10680000109FFFFFFFFCFFFFFCC41046C4104104B3
:1068100011BFFFFFFFFE00000684104484104104F6
:10682000109FFFFFFFFD555554D555568410410468
:10683000109FFFFFFFFFFFFFFCFFFFFCC4104104A0
:1068400011BFFFFFFFFFFFFFFE00000684104104A1
:10685000109FFFFFFFFFFFFFFD555554D5555555C0
:1068600055BFFFFFFFFFFFFFFFFFFFFCFFFFFFFF25
:10687000FF9FFFFFFFFFFFFFFFFFFFFE0000000085
:10688000003FFFFFFFFFFFFFFFFFFFFD5555555581
:10689000555FFFFFFFFFFFFFFFFFFFFFFFFFFFFF52
:1068A000FFFFFFFFFFFFFFFFFFFFFFFFFFFFFFFFF8
:1068B000FFFFFFFFFFFFFFFFFFFFFFFFFFFFFFFFE8
:1068C000FFFFFFFFFFFFFFFFFFFFFFFFFFFFFFFFD8
:1068D000FFFFE02EFB7DFBFBCFC1DFBB3EC0E1FE37
:1068E0003C1FFDEE7B39F9F3CF9EDFBB3EDFDEFCC4
:1068F000DDE7FDEE3BBBF9EBD7BF5FBB5EDFDEFD47
:10690000EDF7FDEEBBD3FAEBB73FDFBB4EDFDFFFAA
:10691000CDF3FDEEDBC7FAEBBB7FC03B6EC0E3FF00
:106920001DF3FDEECBEFFADBBB7FDFBB66DFF8FFCD
:10693000CDF3FDEEEBEFFB5B033F5FBB76DFFE7F4E
:10694000EDF3FDEEF3EFFB5B79BEDFBB7ADFDE7DBF
:10695000EDF7FDEEF3EFFBBAFD9EDFBB7CDFDEFD66
:10696000CDE7FDEEFBEFFBBAFDC1DFBB7EC0E0FE75
:106970001C1F6D61726C696E66772E6F72670032D4
:106980002E302E375F4457372E33001FFFFFFFFF97
:10699000FFFF600000000001FF400000000000FF5A
:1069A0008000000000007F83CF00000C303F87FF95
:1069B00080000C301F867980000C000F8C30C7835C
:1069C0008C30E78C30CFC7CC31F38C30DCECEC333F
:1069D000B98C30D86C6C33198C30D06C0C33198C6A
:1069E00030D86C0C33198C30DC6C0E3B198C30CFEA
:1069F0007C079F198C30C77C038F19400000000072
:106A00000002600000000000061FFFFFFFFFFFF80C
:106A100070012C0190012701B0012201C0011D016C
:106A2000F00118011002130130020E016002090189
:106A300090020401C002FF000003FA004003F500C9
:106A40008003F000D003EB002004E6007004E100B6
:106A5000E004DC004005D700C005D2004006CD00B0
:106A6000D006C8008007C3003008BE00F008B90097
:106A7000C009B400B00AAF00B00BAA00D00CA5004A
:106A8000000EA000500F9B00C01096005012910005
:106A900000148C00C0158700B0178200B0197D006B
:106AA000D01B7800001E730040206E009022690009
:106AB000F024640040275F0090295A00E02B550025
:106AC000102E500020304B0010324600E0334100C1
:106AD00090353C001037370070383200A0392D0057
:106AE000B03A2800A03B2300603C1E00103D190076
:106AF000903D1400103E0F00703E0A00C03E05009D
:106B0000003F0000403FFBFF803FF6FFC03FF1FF2A
:106B10002020506C616E6E657242756666657242C9
:106B2000797465733A20002046726565204D656D65
:106B30006F72793A2000436F6D70696C65643A201A
:106B400041707220323420323032310A00204C61E0
:106B5000737420557064617465643A203230323148
:106B60002D30342D3138207C20417574686F723A95
:106B70002054696E794D616368696E657333440AA8
:106B800000322E302E375F4457372E330A004D61C6
:106B9000726C696E0020536F667477617265205263
:106BA000657365740A00205761746368646F6720B9
:106BB00052657365740A002042726F776E206F759C
:106BC000742052657365740A002045787465726E8E
:106BD000616C2052657365740A00506F7765725559
:106BE000700A0073746172740A0047323858590091
:106BF0004D31303031006572726F72207772697476
:106C0000696E6720746F2066696C650A00446F6E58
:106C10006520736176696E672066696C652E0A006F
:106C20004D323900456E6473746F707300255320C4
:106C3000256320256320256320256300205A3A0020
:106C400020593A0020583A00656E6473746F70736F
:106C5000206869743A200000000A0B02090C0D0E2E
:106C6000080703040100000000000000000000000D
:106C70000000000000000000000000000000000014
:106C800000000012111000000000000000000000D1
:106C900000000000000000000000000000004D6F38
:106CA00076652025736D6D004D6F766520302E3131
:106CB0006D6D004D6F766520316D6D004D6F7665A1
:106CC0002031306D6D004D6F76652041786973001D
:106CD0004578747275646572004D6F7665205A0050
:106CE0004D6F76652059004D6F7665205800A5657B
:106CF000A1654368616E67652046696C616D656E6C
:106D00007400556E6C6F61642046696C616D656ED0
:106D100074004C6F61642046696C616D656E74002F
:106D20005072656865617420437573746F6D0050AF
:106D30007265686561742024004261636B00707243
:106D40006F6D70745F0073686F7700627574746F35
:106D50006E00626567696E0050757267654D6F728F
:106D6000650050617573656400436F6E74696E757C
:106D700065004C6F61642046696C616D656E7420BE
:106D80005400496E736572742066696C616D656E3E
:106D90007420616E642073656E64204D3130380A52
:106DA00000220A00556E6B6E6F776E20636F6D6DFB
:106DB000616E643A2022002042002050006F6B0078
:106DC000204500205A00205900204D39322058001B
:106DD00020453A00205A3A0020593A00583A0020FB
:106DE000746F6F206C6F6E6720657874727573694D
:106DF0006F6E2070726576656E7465640A0020633C
:106E00006F6C6420657874727573696F6E20707230
:106E10006576656E7465640A00526573656E643AE2
:106E200020006E6F74696669636174696F6E20001B
:106E300000002200250028002B002E003100340025
:106E400002010000050108010B01000021002400DF
:106E500027002A002D00300033000101000004014A
:106E600007010A01050505050705080808080202CB
:106E700002020A0A080804040404010101010101D4
:106E800001010303030303030303040707070C0CB7
:106E90000C0C0C0C0C0C020202020606060606067E
:106EA00006060B0B0B0B0B0B0B0B01021020200823
:106EB0000810204010204080020102010804020155
:106EC00001020408102040808040201008040201C4
:106ED000800402018040201008040201080402011D
:106EE00001020408102040800102040810204080A4
:106EF000D3012F0211241FBECFEFD1E2DEBFCDBFE1
:106F000000E00CBF17E0A0E0B2E0EAEDF3E903E037
:106F10000BBF02C007900D92AE32B107D9F72DE139
:106F2000AEE2B7E001C01D92A732B207E1F717E366
:106F3000C9E7D7E300E006C021970109802FFE01D1
:106F40000F94F7C4C837D10780E00807A9F70F945A
:106F5000E9B20D94DBC90C9400002CEA35EC47E251
:106F60005EE360910B0970910C0980910D0990917D
:106F70000E090F94FAC56093061A7093071A80934E
:106F8000081A9093091A08952CEA35EC47E25EE35B
:106F900060910F0970911009809111099091120967
:106FA0000F9474BE6093021A7093031A8093041AAC
:106FB0009093051A0895FC0184910895FC01808145
:106FC0000895FC01A081B1811C92A281B3818C91B2
:106FD0008F5F8C930280F381E02D90818CE0989FED
:106FE000800D1124E1EDFAE113AE84AF089590E035
:106FF00080E0089590E080E00895282F9091910C12
:10700000833021F495FD0FC094FD0FC0892F90E0CF
:10701000B0E0A0E004C0B695A795979587952A950E
:10702000D2F78170089581E0089580E008950F936C
:107030001F93E62FF0E0EE59F74F008110E030E0AB
:1070400020E0082E04C036952795179507950A94D9
:10705000D2F700FD07C0FA018083618381E01F91B0
:107060000F91089580E0FBCF0F931F93CF938C0176
:10707000C62F8EE690E10F94DC4FC8010F94DC4FD1
:107080008AE30F94514F80E38C0F0F94514F8AE0A5
:10709000CF911F910F910D94514F81EF91E10F947A
:1070A000DC4F60E081EE91E10E94343860E08CECCE
:1070B00091E10E94343861E085EC91E10E9434381E
:1070C00061E08AEB91E10E94343861E08AEA91E163
:1070D0000E94343860E081EA91E10E94343861E036
:1070E00087E991E10E94343861E08DE891E10E94E6
:1070F000343860E086E891E10E94343861E08EE740
:1071000091E10E94343861E080E791E10E943438D7
:1071100061E082E691E10E94343860E083E591E12C
:107120000E94343860E085E491E10E94343860E0E8
:107130008FE291E10E94343861E08EE191E10E949A
:10714000343861E08FE091E10E94343861E088E0FA
:1071500091E10E94343860E081E091E10E9434388E
:1071600061E088EF90E10E94343861E083EE90E1C5
:107170000E94343861E085ED90E10E94343861E08E
:1071800082EC90E10E94343860E085EB90E10E944F
:10719000343861E080EB90E10E94343861E083EAAA
:1071A00090E10E94343860E08FE890E10E9434382A
:1071B00060E08CE790E10E94343860E08FE19BE171
:1071C0000E94FA37682F617083E790E10C9434389D
:1071D000EF92FF920F931F93CF93DF93EC018B01FC
:1071E0007A018A859B858617970731F08881998176
:1071F0000F9477AA1B870A87B701888199810F941A
:10720000BA9C2E813F81820F932F911D9F838E8385
:1072100090E080E0DF91CF911F910F91FF90EF9070
:1072200008959F92AF92BF92CF92DF92EF92FF921A
:107230000F931F93CF93DF93EC018B01942EA52E18
:107240008A859B858617970731F0888199810F94ED
:1072500077AA1B870A8788859985019649F5BC809E
:107260000A818E81080FC880D980D6015596ED918C
:10727000FC91C6011995B80EE92CFA2C10E0F70123
:1072800021917F01211127C08E819F81810F911D46
:107290009F838E8390E080E0DF91CF911F910F91CB
:1072A000FF90EF90DF90CF90BF90AF909F900895A8
:1072B0000E811F81692D7A2D888199810F94BA9C46
:1072C000800F912F911D288539852817390738F6A9
:1072D00081E090E0E1CF4B2D602FC6010F94CFAA43
:1072E000080F180FCCCFDF92EF92FF920F931F93EE
:1072F000CF93DF93EC01D62E1CAD0BAD7C0184E067
:10730000E80EF11CE98DFA8DC7011995412F480F40
:107310002D2D602FC7010F94CFAA9BAD890F8BAF86
:1073200081E090E0DF91CF911F910F91FF90EF905E
:10733000DF900895AF92BF92DF92EF92FF920F938A
:107340001F93CF93DF938C01EB01D42E79018FE053
:10735000481709F486C0A5E14A17B1F1BAE04B130A
:107360000EC0EC81FD8130E020E042E061E0C80128
:10737000199541E756E1BE01C8010F947AAB0A8026
:10738000DB81C02DF2E3DF1609F4E2C0FD1508F43D
:1073900091C085E1D81609F4E0C0A7E1DA1609F436
:1073A000EFC0B4E1DB127BC0EE81FF818D8190E004
:1073B000880F991F8E0F9F1F11928E179F07E1F75D
:1073C000CE010F9497A86BC0AA80BB804CE556E114
:1073D000C8010F947AABF5014481440F406BBE01A4
:1073E000C8010F9462AB41E0BE01C8010F946AABC3
:1073F000D50116962D913C911797EC81FD8115963C
:107400004C9166E0C801199540E0BE01C8010F9497
:1074100072AB4CE556E1BE01C8010F947AABF501A1
:107420004481440F4F5F406BBE01C8010F9462ABB3
:1074300041E0BE01C8010F946AABD50115964C918D
:10744000159716962D913C91240F311DEC81FD81ED
:1074500066E0C801199540E0BE01C8010F9472AB07
:107460008ECF41E0C8010F9472AB40E0BE01C8016D
:107470000F946AAB41E8BE01C8010F9462ABF701FB
:10748000408150E05595479555954795BE01C801F7
:107490000F9462AB40E0BE01C8010F9472AB81E073
:1074A000DF91CF911F910F91FF90EF90DF90BF90F0
:1074B000AF900895E6E4DE1609F471C0F7E4DF1634
:1074C00009F471C08BE3D812EACFD70111969C91D1
:1074D000119713968C9138E0390F813031F0833059
:1074E00011F0392F02C0392F985021E04B814917F4
:1074F00008F420E041E0391708F040E091E05A81BB
:10750000351708F490E0322F342B932311F4242301
:1075100031F2F701128100E0D12C843048F490E080
:10752000FC01EB53FD4FD0808F539D4FDC010C913C
:1075300017FF04C0B701CE010F949EA8F701808108
:107540008D0D80838181800F8183110F89F7A7CFF3
:10755000B701CE010F949EA8A2CFCE010F9481A8AF
:10756000882309F49DCFEE81FF818D8190E0880F03
:10757000991F8E0F9F1F11928E179F07E1F78FCFD4
:10758000D7011C928A8111968C9311978D8181501D
:1075900012968C9312978B8113968C9380CF8D814A
:1075A000F70180837CCF8981D7018C9378CFCF92EC
:1075B000DF92EF92FF920F931F93CF93DF93CDB79C
:1075C000DEB72C970FB6F894DEBF0FBECDBFF0909C
:1075D0000C1BE0900D1B2091740821111DC04DE67D
:1075E00055E16E2D8F2D0F943BAB90E080E0F80EAF
:1075F000F0920C1BE0920D1B99272C960FB6F89475
:10760000DEBF0FBECDBFDF91CF911F910F91FF90D5
:10761000EF90DF90CF900895C090D91AD090DA1AE9
:1076200025ED3AE13A8329832F2D30E03C832B83EB
:107630002E2D30E03E832D8318861F827A8769873E
:107640001C861B8601E119E39E012F5F3F4F4BED26
:1076500057E3BC01C6010F94B582B60185ED9AE1EE
:107660000F9477AA8F819885C2CFCF93C62F0F949E
:10767000D642882319F0CF910D9430428C2FCF91B0
:107680000895CF93DF93EB010F94D642882319F02E
:107690000F942042EB01CE01DF91CF9108950F931B
:1076A0001F93CF93DF9300D01F92CDB7DEB79C011D
:1076B0000CE61CE090E1E7E8FDE0D80101900D92B6
:1076C0009A95E1F7F9012081318142815381F801D6
:1076D00060857185828593850F9400C5F801608768
:1076E00071878287938780E090E0A0EAB0E4898385
:1076F0009A83AB83BC83CE0101960F94C5140F907F
:107700000F900F900F90DF91CF911F910F910895DF
:10771000CF9384E50F94D642C0E08823D9F00F942C
:107720003042C82F1816B4F40F94FD5B8DE40F940B
:10773000514F80916D0890916E080F942EAD6C2F73
:10774000CC0F770B86E19DE00F94BA528AE00F943C
:10775000514FCFEF8C2FCF91089583E50F94D642F0
:107760008823E9F00F94D0A260937C0C70937D0C79
:1077700080937E0C90937F0C0F94584220E030E071
:107780004AE754E40F9474BE0F9473C660930802E2
:107790007093090280930A0290930B0208958091DE
:1077A000580784FD13C080915A0787FD0FC0809150
:1077B0005B07837059F40E945AF780911F09882350
:1077C00021F010921F091092200908950E9449F794
:1077D00088E50F948842882331F05F9A8091E40B0A
:1077E0008E7F8093E40B89E50F948842882331F0E3
:1077F0008A9A8091E40B8D7F8093E40B8AE50F9445
:107800008842882359F08091080180958170809387
:1078100006018091E40B8B7F8093E40B85E40F9449
:107820008842882351F20F94B84CC7CF80912E071D
:1078300090912F07009731F04AE050E070E060E04F
:107840000D94ECBB60E070E0CB0108958091580787
:10785000827149F480915A078C7829F480915B07F2
:10786000837009F475C082E40F948842882351F034
:107870000E94163C6093991470939A1480939B1401
:1078800090939C1483E50F948842882351F00F94C1
:1078900058426093C9147093CA148093CB14909388
:1078A000CC1484E50F948842882351F00F945842F9
:1078B0006093CD147093CE148093CF149093D01412
:1078C00088E50F948842882351F00F9458426093C2
:1078D000AC0D7093AD0D8093AE0D9093AF0D89E517
:1078E0000F948842882351F00F9458426093B00D52
:1078F0007093B10D8093B20D9093B30D8AE50F9400
:1079000088428823B1F00F9458426093B40D70936D
:10791000B50D8093B60D9093B70D2DEC3CEC4CEC6F
:107920005DE30F940EBE181624F083E29CE00F94E2
:10793000DC4F85E40F948842882351F00F9458421D
:107940006093B80D7093B90D8093BA0D9093BB0DF1
:1079500008950F931F93CF93DF9300D000D01F9211
:107960001F92CDB7DEB7FC018B0183A5811112C038
:1079700081E083A784819581A681B781B0588983EE
:107980009A83AB83BC83BE016F5F7F4F8CE69CE024
:107990000F943F401D821E821F82188620E030E037
:1079A00040E05FE360918F0D7091900D8091910D9B
:1079B0009091920D0F9400C569837A838B839C8389
:1079C0009E012B5F3F4FAE014F5F5F4F6BE87DE045
:1079D00087E89DE00F941A3F1D821E821F82188641
:1079E00020E030E040E05FE3F8016085718582854A
:1079F00093850F9400C569837A838B839C83B80138
:107A00006C5F7F4F9E012B5F3F4FAE014F5F5F4F1B
:107A1000C8010F941A3F28960FB6F894DEBF0FBE28
:107A2000CDBFDF91CF911F910F9108952F923F927B
:107A30004F925F926F927F928F929F92AF92BF927E
:107A4000CF92DF92EF92FF920F931F93CF93DF932A
:107A5000CDB7DEB7A2970FB6F894DEBF0FBECDBF8D
:107A60008C011B015E834D834090870D5090880DE3
:107A70006090890D70908A0D80908B0D90908C0D88
:107A8000A0908D0DB0908E0DDB018D919D910D908C
:107A9000BC91A02D8F87988BA98BBA8B9C01AD01CF
:107AA000C301B2010F94FFC46B017C01D101149694
:107AB0008D919D910D90BC91A02D8B8B9C8BAD8B4E
:107AC000BE8B9C01AD01C501B4010F94FFC46F8B47
:107AD000788F898F9A8FAD81BE818D919D910D9008
:107AE000BC91A02D8F839887A987BA879C01AD018F
:107AF000C301B2010F94FFC46B8F7C8F8D8F9E8F5B
:107B0000AD81BE8114968D919D910D90BC91A02D5B
:107B10008B879C87AD87BE879C01AD01C501B401F1
:107B20000F94FFC46F8F78A389A39AA3A70196012E
:107B3000C701B6010F9474BE6B017C012F89388D8B
:107B4000498D5A8DCA01B9010F9474BE9B01AC01D5
:107B5000C701B6010F9400C54B015C012F85388920
:107B600049895A896F81788589859A850F94FFC4E0
:107B70002B013C012B893C894D895E896B857C8575
:107B80008D859E850F94FFC46B017C01A30192013A
:107B9000C301B2010F9474BE2B013C01A7019601F1
:107BA000C701B6010F9474BE9B01AC01C301B201C1
:107BB0000F9400C50F94FEC76B017C012B8D3C8D8B
:107BC0004D8D5E8DCA01B9010F9474BE2B013C012D
:107BD0002F8D38A149A15AA1CA01B9010F9474BED1
:107BE0009B01AC01C301B2010F9400C59B01AC0124
:107BF000C501B4010F9460C71816B4F520E030E059
:107C0000A901C701B6010F9460C787FF2AC0C70149
:107C1000B601905820E030E040EA50E40F9460C78D
:107C2000181614F5A1016D817E81C8010E94163DD0
:107C3000A2960FB6F894DEBF0FBECDBFDF91CF91F5
:107C40001F910F91FF90EF90DF90CF90BF90AF907A
:107C50009F908F907F906F905F904F903F902F906C
:107C60000895C701B601D6CF20E030E040E050E4EF
:107C7000C501B4010F9460C7181624F4B101C801FE
:107C80000E94A93C19821A821B821C82BE016F5F6E
:107C90007F4FC1010F943F402DEC3CEC4CEC5CE37A
:107CA000C701B6010F9474BE9B01AC01F80160815D
:107CB0007181828193810F9474BE69837A838B83EF
:107CC0009C83C8010F94069BBE016F5F7F4F8D811F
:107CD0009E810F943F40ACCF3F924F925F926F9244
:107CE0007F928F929F92AF92BF92CF92DF92EF924C
:107CF000FF920F931F93CF93DF93CDB7DEB76897B3
:107D00000FB6F894DEBF0FBECDBF7C01DB018C91B6
:107D1000342E380E95E0931508F40EC11196EC91AF
:107D2000022F0E0F063008F007C1F0E0EE59F74FB2
:107D30004080512C712C612C082E04C076946794DD
:107D4000579447940A94D2F740FEF6C0E02FF0E033
:107D5000EE59F74F4080512C712C612C032C04C03C
:107D600076946794579447940A94D2F740FEE4C0FF
:107D7000122FA42E6B010F94DD442B013C016A2DC0
:107D8000660F770B072E000C880B990B0F9415BE0E
:107D90004B015C01AC019B01C301B2010F9400C512
:107DA0006D877E878F87988B832D0F94DD44A50187
:107DB00094010F94FFC469837A838B839C83F601BB
:107DC00081810F9447442B013C01612F660F770B93
:107DD000072E000C880B990B0F9415BE4B015C010C
:107DE000AC019B01C301B2010F9400C5698B7A8B72
:107DF0008B8B9C8B802F0F944744A50194010F948B
:107E0000FFC46D837E838F839887F701808591857A
:107E1000A285B38589879A87AB87BC878D8B9E8B1C
:107E2000AF8BB88F4FEE50E061E070E0CE0141962D
:107E30000E94C7EF4FEE50E061E070E0CE01059682
:107E40000E94C7EF4FEE50E061E070E0CE010D966A
:107E50000E94C7EF4FEE50E061E070E0CE01019666
:107E60000E94C7EF49885A886B887C8827E137EBE6
:107E700041ED58EBC301B2010F9460C787FD5CC0B0
:107E800027E030E040E753E4C301B2010F940EBE97
:107E900018160CF451C04D845E846F84788827E1F5
:107EA00037EB41ED58EBC301B2010F9460C787FD7A
:107EB00043C027E030E040E753E4C301B2010F9430
:107EC0000EBE1816CCF14D805E806F80788427E15D
:107ED00037EB41ED58EBC301B2010F9460C787FD4A
:107EE0002BC027E030E040E753E4C301B2010F9418
:107EF0000EBE18160CF149805A806B807C8027E1F9
:107F000037EB41ED58EBC301B2010F9460C787FD19
:107F100013C027E030E040E753E4C301B2010F94FF
:107F20000EBE18164CF0AE014F5F5F4FBE01635F8F
:107F30007F4FC7010E94163D68960FB6F894DEBFCA
:107F40000FBECDBFDF91CF911F910F91FF90EF90AA
:107F5000DF90CF90BF90AF909F908F907F906F9069
:107F60005F904F903F9008954F925F926F927F92F3
:107F70008F929F92AF92BF92CF92DF92EF92FF9239
:107F80001F93CF93DF9300D01F92CDB7DEB7198236
:107F90001A821B821C82CE0101964C0187E8C82EF2
:107FA0008DE0D82E9CE6E92E9CE0F92E2BE7A22E40
:107FB0002DE0B22E10E088E5810F0F94D642F40137
:107FC00081934F01882341F00F9458422B013C01CB
:107FD00080918714882359F0F60180819181A281D4
:107FE000B381F70180839183A283B38314C0812F6F
:107FF0000E94FD37882309F4D0C0F6012081318129
:1080000042815381C301B2010F9400C5F70160831F
:108010007183828393831F5FF4E0CF0ED11C84E0D1
:10802000E80EF11C94E0A90EB11C133021F685E492
:108030000F94D6428C83882309F4B9C00F94584218
:108040006B017C0183E00E94FD37882371F0209151
:10805000930D3091940D4091950D5091960DC7015F
:10806000B6010F9400C56B017C01C092780CD092D0
:10807000790CE0927A0CF0927B0C8091D3098823E2
:1080800059F180911B1B82FF27C08C81882321F12D
:108090008981811103C08A818823F1F02DEC3CECA9
:1080A0004CE45DE36091D20C7091D30C8091D40CC0
:1080B0009091D50C0F9400C59B01AC0160918F0D80
:1080C0007091900D8091910D9091920D0F9460C7D9
:1080D000181614F40F947CAD40E050E0BA0186E429
:1080E0000F94E34220E030E0A9010F9460C7181616
:1080F00084F40F94584220E030E040E752E40F94BB
:10810000FAC56093870270938802809389029093E6
:108110008A028091881483FD2CC08091871481117C
:1081200028C08091D00B882321F12091930D3091AC
:10813000940D4091950D5091960D6091780C709131
:10814000790C80917A0C90917B0C0F94FFC4209154
:10815000DD0B3091DE0B4091DF0B5091E00B0F9463
:1081600000C56093DD0B7093DE0B8093DF0B909363
:10817000E00B0F900F900F900F90DF91CF911F9118
:10818000FF90EF90DF90CF90BF90AF909F908F9037
:108190007F906F905F904F900895F501208131811D
:1081A00042815381C301B2010F94FFC42FCF80914C
:1081B000930D9091940DA091950DB091960D809393
:1081C000780C9093790CA0937A0CB0937B0C55CFDC
:1081D000CF92DF92EF92FF920F931F93CF93DF9393
:1081E000CDB7DEB7A0970FB6F894DEBF0FBECDBFF8
:1081F0000E94883B87FDD1C0482F61E081E00E944A
:1082000086C785E40F948842882309F4D5C00F946B
:1082100058426B017C0120E030E0A9010F9460C757
:1082200087FF04C0F7FAF094F7F8F094F7FAF094A7
:10823000F7F8F094C98ADA8AEB8AFC8A8CE0E5E9DF
:10824000F2E0DE01119601900D928A95E1F78AE540
:108250000F94D642882351F040E050E0BA018AE5FD
:108260000F94E34269877A878B879C8788E50F9410
:10827000D642882351F040E050E0BA0188E50F94DF
:10828000E34269837A838B839C8389E50F94D6428A
:10829000882351F040E050E0BA0189E50F94E342B1
:1082A0006D837E838F83988785E50F94884288232A
:1082B00009F489C00F9458426B017C0120E030E042
:1082C000A901C701B6010F9460C787FF04C0F7FA80
:1082D000F094F7F8F094F7FAF094F7F8F094CD8A68
:1082E000DE8AEF8AF88E198E1A8E1B8E1C8E8CE415
:1082F0000F948842882309F46FC00F9458426B0191
:108300007C0120E030E0A901C701B6010F9460C7ED
:1083100087FF04C0F7FAF094F7F8F094CD8EDE8E64
:10832000EF8EF8A262E070E082E40F940F43F82E23
:108330008091EC09811131C021E0AE014B5E5F4FAD
:10834000BE016F5F7F4FCE0141960F947567882302
:1083500021F16F2D81E00F94897E82E50F94D64242
:10836000882309F442C00F94544240E050E060EA90
:1083700071E44D875E876F87788B2091EC0922230B
:1083800061F08C012F2DAE01435F5F4FBE01635E34
:108390007F4FCE0149960F946665A0960FB6F8946C
:1083A000DEBF0FBECDBFDF91CF911F910F91FF9028
:1083B000EF90DF90CF900895C12CD12C80E8E82E6B
:1083C00080E4F82E33CFC090CB09D090CC09E09058
:1083D000CD09F090CE0972CFC090CF09D090D009CE
:1083E000E090D109F090D2098CCF90E080E0BDCF31
:1083F000CF92DF92EF92FF920F931F93CF93DF9371
:10840000CDB7DEB76C970FB6F894DEBF0FBECDBF09
:108410008CE40F948842882309F4C3C00F94584217
:108420006B017C0120E030E0A9010F9460C787FF59
:1084300004C0F7FAF094F7F8F094F7FAF094F7F82C
:10844000F094C98EDA8EEB8EFC8E8CE0E5E9F2E0DA
:10845000DE01119601900D928A95E1F788E50F945F
:10846000D6428823A1F040E050E0BA0188E50F949D
:10847000E34220917B0D30917C0D40917D0D509118
:108480007E0D0F94FFC469837A838B839C8389E577
:108490000F94D6428823A1F040E050E0BA0189E56C
:1084A0000F94E34220917B0D30917C0D40917D0D26
:1084B00050917E0D0F94FFC46D837E838F839887C8
:1084C0008AE50F94D642882351F040E050E0BA018B
:1084D0008AE50F94E34269877A878B879C87F090BF
:1084E0001B1BF2FAFF24F0F840E061E080E00E94FC
:1084F00086C760E080E50F94FA42E82E1D861E864E
:108500001F86188A8091EC0981113CC02E2DAE0186
:10851000435F5F4FBE016F5F7F4FCE0149960F945F
:108520007567882379F18091D30981110F947CAD0F
:10853000FF2011F0EE2031F160E080E00F94897EA1
:10854000898D9A8DAB8DBC8DB0588D8B9E8BAF8BEA
:10855000B88F198A1A8A1B8A1C8A1D861E861F8656
:10856000188A8091EC09882369F010E000E020E08F
:10857000AE014B5E5F4FBE016F5E7F4FCE010D9629
:108580000F9466656C960FB6F894DEBF0FBECDBF34
:10859000DF91CF911F910F91FF90EF90DF90CF90DF
:1085A0000895C12CD12C80E8E82E80E4F82E45CF28
:1085B000AF92BF92CF92DF92EF920F931F93CF9320
:1085C000DF935B01EA016901882309F463C08CE150
:1085D0009CE00F94DC4FF501608171818281938171
:1085E00046E00F94442EE1100BC083E19CE00F9411
:1085F000DC4F688179818A819B8146E00F94442E0B
:108600008CE09CE00F94DC4FF601608171818281E7
:10861000938143E00F94442E85E09CE00F94DC4F5F
:10862000F801608171818281938143E00F94442E2F
:108630008CEF9BE00F94DC4FF60120813181428169
:108640005381F80160817181828193810F94FFC40D
:1086500043E00F94442EEE20F9F08AE00F94514F3E
:1086600087EE9BE00F94DC4F688179818A819B8142
:1086700046E00F94442E8AE00F94514F8AE0DF9138
:10868000CF911F910F91EF90DF90CF90BF90AF905F
:108690000D94514FE110E4CFDF91CF911F910F91D5
:1086A000EF90DF90CF90BF90AF900895CF93DF937E
:1086B000CDB7DEB720E2488559856F818E810F9452
:1086C000939BDF91CF9108954FE350E0BC0189EE79
:1086D0009BE00D94C1C963E972E084E690E00E94DA
:1086E000D7B06AEB72E084E690E00C94D7B08111C9
:1086F0000C946B4368EB71E084E190E00C94D7B08C
:108700000E9407F30C9477430F94C9390C94774374
:108710000F94171D0C946B43282F1092500C8091CE
:10872000400C9091410CA091420CB091430CB7FFCA
:1087300008C01092400C1092410C1092420C109202
:10874000430C80911E09882331F08091400C809366
:10875000440C10923F0C80913E0C1816FCF4082E2D
:10876000000C990B821B91092091440C022E000CE5
:10877000330B2817390794F097FF02C090E080E090
:108780008093440C092E000CAA0BBB0B8093400C69
:108790009093410CA093420CB093430C8091440CF5
:1087A0006623A9F09091450C891714F48093450C29
:1087B0002091450C022E000C330B2C5F3F4F482FAD
:1087C000082E000C550B241735071CF48450809399
:1087D000450C08958F929F92AF92BF92EF92FF92B5
:1087E0000F931F93CF93DF93EC018B01E42EF22EB6
:1087F0008091CF1A9091D01A8C179D0709F440C030
:108800002091030927FD109203092EEBCA30D207ED
:1088100009F041C085519D4571F40F94D0A26E516D
:108820007B4F8F4F9F4F609305097093060980938C
:10883000070990930809D093D01AC093CF1A30E05B
:1088400020E00093400C1093410C2093420C309395
:10885000430CE092450CF0923E0CC551DD4531F4DD
:10886000109220091092040910921F0982E080934F
:108870007F0281E080933F0C10921B091092130934
:10888000DF91CF911F910F91FF90EF90BF90AF902C
:108890009F908F9008952DE5C531D20761F68A50DB
:1088A0009E4B19F0C5E1DDE5C6CF0F94D0A28090B4
:1088B000050990900609A0900709B0900809681969
:1088C00079098A099B0997FFEDCF8091E40B8770A6
:1088D000873041F7CAE0D9E5AECF20E040E070E054
:1088E00060E085E19DE50C94EA430F931F93CF93DD
:1088F000DF93CDB7DEB76E970FB6F894DEBF0FBE2D
:10890000CDBF282F082E000C330B90911C024091F4
:108910001D028F3F39F0F901EE0FFF1FE25EFD4FA0
:10892000908141814F939F933F938F938FE998E17B
:108930009F938F938E010F5F1F4F1F930F930F9481
:10894000A5BDC8010E9464430E946D440FB6F8940F
:10895000DEBF0FBECDBF6E960FB6F894DEBF0FBE62
:10896000CDBFDF91CF911F910F910895CF930F94B9
:10897000171D0E9407F3C82F882319F080E00F9479
:1089800072328C2F0E947743CF910C946D44AF923A
:10899000BF92CF92DF92EF92FF920F931F93CF93EC
:1089A000DF93CDB7DEB764970FB6F894DEBF0FBE86
:1089B000CDBF0E94883BD82E87FDB5C08AE50F94B5
:1089C000D642882309F4C0C040E050E0BA018AE5ED
:1089D0000F94E3427B018C014D2D63E085E00E9402
:1089E00086C720918F0D3091900D4091910D50913F
:1089F000920D60E070E08AE793E40F94FFC45B019E
:108A00006C019701A8010F9460C7181614F0750146
:108A1000860120E030E0A901B701C8010F9460C7CA
:108A2000181624F4E12CF12C00E010E0B701C80185
:108A30000F946CC6072E000C880B990B0F9415BE73
:108A40006D837E838F83988720E030E0A9010F94A7
:108A50000EBE882321F0CE0105960E944F3B80E098
:108A600090E0A0EAB1E489879A87AB87BC871D862E
:108A70001E861F86188A8CE40F948842882309F486
:108A800068C00F9458426B017C0120E030E0A901DE
:108A9000C701B6010F9460C787FF04C0F7FAF094CE
:108AA000F7F8F094C98ADA8AEB8AFC8A2091FB19DC
:108AB0003091FC192430310574F08091F9199091AE
:108AC000FA19821B930B97FF03C091958195910929
:108AD00001E004970CF400E063E080E00F94FB6495
:108AE000811140C083E08093210210921A090E94F4
:108AF0006D446D817E818F8198858B019C013058FA
:108B000009831A832B833C8320E030E0A9010F9472
:108B10000EBE882321F0CE0101960E944F3B109299
:108B20001A090E946D4464960FB6F894DEBF0FBE1A
:108B3000CDBFDF91CF911F910F91FF90EF90DF900C
:108B4000CF90BF90AF900895E12CF12C00E211E49A
:108B500043CFC090CF09D090D009E090D109F090D8
:108B6000D20993CF83E0E82E22E0AE01475F5F4F4A
:108B7000BE016F5E7F4FCE010D960F941D99B9CF48
:108B80008091991A90919A1A891B8F7011F40D9403
:108B9000A64C81E00895E0910409EE2389F0E150AC
:108BA000E093040988E0E89FF0011124EC53F74FAB
:108BB0006281738127814681808191810C94EA438F
:108BC0000C946D44E0910409E63010F581E08E0FBD
:108BD000809304094091400C5091410C6091420CEB
:108BE0007091430C9091450C80913E0C28E0E29FDF
:108BF000F0011124EC53F74F2091CF1A3091D01A85
:108C00003183208342835383648375839683878370
:108C100008952F923F924F925F926F927F928F9220
:108C20009F92AF92BF92CF92DF92EF92FF920F93FB
:108C30001F93CF93DF9300D000D0CDB7DEB71C01D8
:108C40007A8369832B833C834D835E8327013801BC
:108C500081E080933F0C0E94E24583E080937F0295
:108C6000309202092092010989819A81909300092A
:108C70008093FF088B819C81AD81BE818093FB082E
:108C80009093FC08A093FD08B093FE084092F7086B
:108C90005092F8086092F9087092FA08F12CE12CD1
:108CA000C092400CD092410CE092420CF092430CE6
:108CB000B092D01AA092CF1A9092F6088092F5083E
:108CC0008C8D8093F40826960FB6F894DEBF0FBE05
:108CD000CDBFDF91CF911F910F91FF90EF90DF906B
:108CE000CF90BF90AF909F908F907F906F905F904C
:108CF0004F903F902F900895CF93DF93CDB7DEB77D
:108D00008E819091DF17891778F08093DF179E018D
:108D1000275F3F4F4F81588564E570E08AE897E10F
:108D20000F94D5BD10928917DF91CF9108950F93BD
:108D30001F93CF93DF938C0167FF03C01092DF175F
:108D400060E02091DF17862F062E000C990B281764
:108D5000190609F05CF56093DF1760E08DEE97E18E
:108D60000F94EA4FC8010F94DC4F8AE00F94514FE3
:108D7000C8010F941EBD800F911FEC01C01BD10BC9
:108D8000C535D1053CF00197FC012491207C2038A9
:108D9000D1F3F3CFDD27AE01B8018AE897E10F9454
:108DA0003FBDC657D84E188210928917DF91CF91D8
:108DB0001F910F910895CF938091BC08811109C034
:108DC0008AE498E190930A098093090981E08093ED
:108DD000BC080E94E24520E040E070E060E088E7E7
:108DE00098E50E94EA43C1E0C09320090E9449F738
:108DF000109220090E94CB45C09320094AE358E114
:108E000061E478E184E00F94269A60E08DE298E1D5
:108E10000E94974640E061E080E00E9486C783E2BE
:108E200098E19093E80B8093E70BCF91089510920F
:108E3000840C10927E0280911B1B806480931B1B0C
:108E400061E08BEF97E10F94EA4F40E158E168E170
:108E500078E185E00F94269A60E082E098E10E9434
:108E600097460C946D44CF93C82F0F94E14C811119
:108E70001AC080911B1B82FF0CC080914717811183
:108E800005C08FE59CE0CF910D94B58687E497E10E
:108E9000FACF80913609813061F08EEC97E1CC23D6
:108EA00021F0CF9108958DE298E16FEFCF910C946E
:108EB000974681EE97E1F9CF80E00E943347109208
:108EC000840C10927E020F94D34C882351F0809131
:108ED0001B1B82FD06C08CE598E19093E80B809304
:108EE000E70B61E085E598E10F94EA4F0D945F236D
:108EF0000F931F930F94D0A20091B8081091B90856
:108F00002091BA083091BB08601B710B820B930B48
:108F100097FD0CC086B186FB882780F991E08927F0
:108F2000349B8260329B84608093610780916107EB
:108F300081709091610791FD82609091B7089817B8
:108F400021F18130E1F120F1823051F1833069F17A
:108F5000909160079923B9F09091B608992399F000
:108F60009091B60820911C0930911D09290F311DDF
:108F700097FD3A9530931D0920931C091092B6086D
:108F800091E090937F028093B7081F910F9108950D
:108F9000913079F09230E1F69091B60891500CC082
:108FA000992339F09330C1F3D3CF9130A9F39230A4
:108FB00079F69091B6089F5F9093B608C9CF992330
:108FC00059F3933029F6F5CFCF92DF92EF92FF92CB
:108FD000CF93C82F0F94D0A26B017C0124EA30E715
:108FE0004DE75FE360912D0270912E0280912F0278
:108FF000909130020F940EBE87FD18C08AEF90E06A
:10900000A0E0B0E08C0D9D1DAE1DBF1D8093AA0891
:109010009093AB08A093AC08B093AD08C0931B022B
:10902000CF91FF90EF90DF90CF90089580E090E097
:10903000DC01E8CFCF9393E090937F0281111092EF
:1090400061070F94D0A26C507E4F8F4F9F4F60935B
:10905000B8087093B9088093BA089093BB0868E881
:1090600073E182E090E00E94D7B0C6E0C15049F0C1
:109070000F94D12862E070E080E090E00F949DA210
:10908000F5CFCF910895CF92DF92EF92FF920F9399
:109090001F930F94D0A200917B0810917C0820911F
:1090A0007D0830917E086B017C01C01AD10AE20A6A
:1090B000F30A9701860137FD11C020917A082095A7
:1090C00020937A086A547C4F8F4F9F4F60937B08A0
:1090D00070937C0880937D0890937E0881E0909146
:1090E0007A08911101C080E01F910F91FF90EF90DD
:1090F000DF90CF9008950F942244882339F062E3E3
:1091000070E080E090E00F94764CF5CF62E370E081
:1091100080E090E00D94764C2F923F924F925F92B8
:109120006F927F928F929F92AF92BF92CF92DF9277
:10913000EF92FF920F931F93CF93DF93CDB7DEB7DC
:10914000C957D1090FB6F894DEBF0FBECDBF8EEA66
:1091500099E00F94DC4F87E00F94DF39811190C0C4
:1091600084E50F94D642882329F00F94544281114C
:109170000E94B2EE80E090E0A0E8BFE389839A838A
:10918000AB83BC838D839E83AF83B8878DEC9CECCF
:10919000ACE4BEE389879A87AB87BC8780E090E028
:1091A000A0E2B1E48D879E87AF87B88B8CE390E017
:1091B0009A8B898B8DEC90E09C8B8B8B8DEC9CEC4F
:1091C000ACECBEE38D8B9E8BAF8BB88F80E090E0D4
:1091D000A0EEBFE3898F9A8FAB8FBC8F1BA61CA616
:1091E0004AE959E969E97EE38FE40F94E3426D8F20
:1091F0007E8F8F8F98A360E083E40F94FA4289A357
:1092000060E08BE40F94FA428AA389E40F94D6427B
:10921000312C10E000E08823C9F00F94304290E038
:109220001816190614F481E090E033243394380EB4
:10923000232D2150330BC90126E0289FF001299FDF
:10924000F00D1124E55DF34F0281138182E40F9448
:10925000D642882319F00F9454428C010115110550
:1092600059F1C80188978536910520F16CE870E0C6
:1092700080E899E00F94BA528BE799E00F94DC4FA5
:10928000C758DF4F0FB6F894DEBF0FBECDBFDF91DA
:10929000CF911F910F91FF90EF90DF90CF90BF90F3
:1092A000AF909F908F907F906F905F904F903F9086
:1092B0002F9008951A8B098B8CE40F94D642882343
:1092C000E1F00F9458424B015C0189869A86AB8687
:1092D000BC8620E030E0A9010F9460C787FD0AC07A
:1092E00020E030E040E050E4C501B4010F940EBE30
:1092F00018161CF483E599E0C1CF81E50F948842EC
:10930000882331F180912E0790912F07892BE9F066
:109310000F9458424B015C018D829E82AF82B886C9
:109320002DEC3CEC4CE45DE30F9460C787FD0AC074
:1093300020E030E040E751E4C501B4010F940EBED7
:10934000181634F482E299E099CF87EF98E096CF2F
:1093500083E50F94D6428823E9F00F9458424B01DD
:109360005C018D8A9E8AAF8AB88E2DEC3CEC4CEC69
:109370005DE30F9460C787FD0AC020E030E040E065
:1093800050E4C501B4010F940EBE18161CF480ED14
:1093900098E074CF80E50F948842882341F0809153
:1093A0002E0790912F07892B29F58FEF8BA786E445
:1093B0000F94D642882309F43DC00F9458424B01C4
:1093C0005C01898E9A8EAB8EBC8E20E030E040E846
:1093D0005FE30F9460C787FD0AC020E030E040E8FB
:1093E00050E4C501B4010F940EBE18161CF58FE7AA
:1093F00098E044CF8BA58F5F8BA70F9458424B0109
:109400005C018D869E86AF86B88A20E030E0A90197
:109410000F9460C787FD0BC020E030E048EC51E4BA
:10942000C501B4010F940EBE18160CF0C0CF88EA27
:1094300098E024CF898C9A8CAB8CBC8C4D885E884C
:109440006F88788CA5019401C501B4010F9474BE96
:109450009B01AC0160E070E084E490E40F94FAC5F5
:1094600029813A814B815C810F9474BE6B017C0130
:10947000A3019201C301B2010F9474BEA50194012E
:109480000F9474BE2CEE31E548EB5DE30F94FAC502
:109490009B01AC01C701B6010F9474BE69837A8346
:1094A0008B839C8310E000E0332069F0A32DA15052
:1094B000BB0B26E02A9FF0012B9FF00D1124E55DE8
:1094C000F34F0081118188E40F94D642882319F06C
:1094D0000F9454428C010115110559F0C801855AA9
:1094E00091098838910518F081E598E0C7CE1C8B6A
:1094F0000B8B85E50F9488428823C9F00F94D0A286
:10950000611571058105910511F00F9457B980918E
:109510002E0790912F07892BC9F00F945842609322
:1095200068087093690880936A0890936B0865E2F5
:1095300070E082E50F940F43E1969FAF8EAFE19705
:109540001816190644F08DE198E098CE60E070E0BE
:1095500088E492E4E4CF89E50F94D642882381F130
:109560000F94584220917F0D3091800D4091810DD4
:109570005091820D0F94FFC46B017C0188E50F941C
:10958000D642882331F10F94584220917B0D3091BF
:109590007C0D40917D0D50917E0D0F94FFC46BA307
:1095A0007CA38DA39EA3CFA2D8A6E9A6FAA6CE013E
:1095B00083960F940949811115C083EF97E05ECE21
:1095C000C0908B0DD0908C0DE0908D0DF0908E0D95
:1095D000D5CF6091870D7091880D8091890D909104
:1095E0008A0DDDCF84E40F94884211E081270F9427
:1095F000F24A80E090E0A0EAB0E48DA79EA7AFA772
:10960000B8AB60E0CE018D960F943316B091B00CDC
:10961000EA96BFAFEA971092B00C0E94E4DD80EAB0
:1096200097E00F94DC4F89899A894A970CF094C08F
:1096300063E68DE797E00E94974681E00E941A4812
:109640008B899C890E94CBF641E061E080E00F9419
:10965000E230882309F494C080E00E94334781E01F
:109660000E941A481092930D1092940D1092950D2D
:109670001092960D83E99DE00F94EF081BA511232E
:1096800009F4E2C020E030E040E751E46091B91411
:109690007091BA148091BB149091BC140F94FAC5C8
:1096A00021966CAF7DAF8EAF9FAF21971F3F09F022
:1096B00024C381E08093600763E685ED97E00E9414
:1096C000974668E873E182E090E00E94D7B080E1BD
:1096D000E7E8FDE0ACE6BCE001900D928A95E1F789
:1096E000CE0101960F94069BC12CD12C76010F94CC
:1096F000224481119DC068E873E182E090E00E94FD
:10970000D7B020E030E040E85EE36091780C7091E3
:10971000790C80917A0C90917B0C0F9400C560932A
:10972000780C7093790C80937A0C90937B0C20E0EA
:1097300030E040E85EE3C701B6010F9400C56B015D
:109740007C0120E030E84BE354E40F9460C787FDD0
:109750005FC01092600714C063E680E997E00E9442
:10976000974681E00E941A481093600789899A8978
:109770000F94484061E081E00F945B2F811158CF36
:109780006FEF87EE97E00E9497468CA5811112C07B
:1097900081E08CA78D819E81AF81B885B0588DA75F
:1097A0009EA7AFA7B8ABBE01635D7F4F8CE69CE080
:1097B0000F943F4080E090E0A0EAB0E48093740C06
:1097C0009093750CA093760CB093770C1DA61EA6F3
:1097D0001FA618AABE01635D7F4F8CE69CE00F9424
:1097E0003F40EA96BFADEA97B093B00C0E94E4DD2B
:1097F000109260078AA1811143CD10929E0C1092A5
:109800009D0C0E947CDE90E080E00E94CBF638CD7B
:10981000CE01CD960F94C51480E1E7E8FDE0ACE6FB
:10982000BCE001900D928A95E1F70E9449F75FCF65
:109830000E947B4863E688EC97E00E94974681E0AF
:109840000E941A4810926007E2E6F8E086E0DF0125
:109850001D928A95E9F780E1E7E8FDE0ACE6BCE01F
:1098600001900D928A95E1F789859A85AB85BC8533
:109870008093740C9093750CA093760CB093770C36
:109880001DA61EA61FA618AABE01635D7F4F8CE60B
:109890009CE00F943F40BE01635E7F4F8CE69CE0EE
:1098A0000F943F4081E08093600789A1882309F4E9
:1098B0007BC288E0E7E8FDE0DE019D9601900D9215
:1098C0008A95E1F78FEF8DAF8EAFAE01435C5F4FAE
:1098D00067E178E3CE018D960F94CB49BE01635CBE
:1098E0007F4F82E698E00F94094286E0FE01FD96E4
:1098F000DE01A75ABF4F01900D928A95E1F786E0ED
:10990000FE01E75AFF4FDE01A15ABF4F01900D92B1
:109910008A95E1F786E0FE01E15AFF4FDE01AB597F
:10992000BF4F01900D928A95E1F7CE018B599F4F61
:109930000F943B44882309F4C8C1A6968FADA6971F
:109940000F94DD44762E872E982EA92E862F982DE3
:10995000A92DBA2D65968CAF9DAFAEAFBFAF659701
:10996000A7968FADA7970F9447446B017C0169962A
:10997000CCAEDDAEEEAEFFAE6997CE018F5A9F4FF3
:109980000F940949882309F4A4C1A6966FACA69741
:10999000A796BFACA79720E030E040EA50E4672DDF
:1099A000782D892D9A2D0F9400C5162F072F382E4C
:1099B000292E862F902FA32DB22D21968CAF9DAFEF
:1099C000AEAFBFAF21972596CCAEDDAEEEAEFFAE0B
:1099D0002597611012C2B110EBC120E030E040EADF
:1099E00050E4C701B6010F9400C56B017C01BB2098
:1099F00009F48BC224E0172D082D392C2A2C2B15A5
:109A00000CF4F2C122ED422E23E5522E2BE7622EFA
:109A100021E4722E21968CAC9DACAEACBFAC2197EC
:109A200025968CAD9DADAEADBFAD2597E9968CAFBB
:109A30009DAFAEAFBFAFE9979C01AD0169966CAD2C
:109A40007DAD8EAD9FAD69970F94FFC4E5966CAF69
:109A50007DAF8EAF9FAFE597A501940165966CAD84
:109A60007DAD8EAD9FAD65970F94FFC42D966CAF05
:109A70007DAF8EAF9FAF2D97E5968CAD9DADAEAD12
:109A8000BFADE59761968CAF9DAFAEAFBFAF6197AD
:109A9000A50194016091870D7091880D8091890DC9
:109AA00090918A0D0F94FFC4E5966CAF7DAF8EAF99
:109AB0009FAFE597E9962CAD3DAD4EAD5FADE99713
:109AC00060918B0D70918C0D80918D0D90918E0D0C
:109AD0000F94FFC44B015C01812F902FA32DB22D59
:109AE0008DA79EA7AFA7B8ABC9AADAAAEBAAFCAA12
:109AF000C984DA84EB84FC84CDAADEAAEFAAF8AE8E
:109B00002DEC3CEC4CEC5CE3C301B2010F9474BE51
:109B100029813A814B815C810F9474BE2091930D11
:109B20003091940D4091950D5091960D0F9400C574
:109B300069AF7AAF8BAF9CAFE5962CAD3DAD4EAD26
:109B40005FADE597CA01B9010F9474BE2B013C01CA
:109B5000A5019401C501B4010F9474BE9B01AC0131
:109B6000C301B2010F9400C520E030E040E050E4B2
:109B70000F9460C71816ACF420E030E040E05FE3DB
:109B8000C701B6010F9400C529966CAF7DAF8EAFAB
:109B90009FAF2997BE01635C7F4FCE0101960E9463
:109BA000A93C89859A85AB85BC8529968CAF9DAFEC
:109BB000AEAFBFAF2997AF961CAE1DAE1EAE1FAEA7
:109BC000AF97BE0165597F4FCE01CD960F943F40B0
:109BD000CE0101960F94069BE090B114F090B21460
:109BE0000091B3141091B414A090AD14B090AE14C1
:109BF000C090AF14D090B0149501A601B701C80170
:109C00000F9460C7181614F47501860180908702BE
:109C100090908802A0908902B0908A022DEC3CECD2
:109C20004CEC5DE3B701C8010F9474BE60938702EA
:109C3000709388028093890290938A0240E0BE016B
:109C4000675B7F4FCE018D960F944FA380E1E7E8CD
:109C5000FDE0ACE6BCE001900D928A95E1F78092C0
:109C6000870290928802A0928902B0928A020F9491
:109C70002844811185CD20E04FEFBE016B597F4F05
:109C8000CE0101960E946C3E20E041E0BE016B597E
:109C90007F4FCE0101960E946C3E2FEF40E0BE0147
:109CA0006B597F4FCE0101960E946C3E21E040E04F
:109CB000BE016B597F4FCE0101960E946C3E0E94FF
:109CC00049F70F94284481115BCD8091D314809380
:109CD000D414E196AEADBFADE1971197E196BFAF59
:109CE000AEAFE197AB2B09F44BCDCE018B599F4F13
:109CF0000F943B448111D9CD43CD63E685EB97E0CA
:109D00000E94974681E00E941A4880E1E7E8FDE062
:109D1000ACE6BCE001900D928A95E1F72D853E8579
:109D20004F8558896091780C7091790C80917A0CEC
:109D300090917B0C0F9400C56093780C7093790C14
:109D400080937A0C90937B0CCE01CD960F94C51422
:109D50002D853E854F8558896091780C7091790CDE
:109D600080917A0C90917B0C0F94FFC46093780CD7
:109D70007093790C80937A0C90937B0C8CA5811155
:109D800063CD81E08CA78D819E81AF81B885B0586D
:109D90008DA79EA7AFA7B8ABBE01635D7F4F8CE6D2
:109DA0009CE00F943F4050CD88E0FE01B39684CDF7
:109DB000872D982DA92DBA2D21968CAF9DAFAEAFD2
:109DC000BFAF219720E030E040EA50E4C701B60180
:109DD0000F94FFC425966CAF7DAF8EAF9FAF2597D4
:109DE000B4E0BB150CF0F9CD92ED492E93E5592E58
:109DF0009BEF692E90E4792E0DCE34E036150CF0F1
:109E000056C062961FAD629763960FAD63976496D6
:109E10003FAC649765962FAC65973B15FCF420E04A
:109E200030E040EA50E4672D782D892D9A2D0F946B
:109E3000FFC421966CAF7DAF8EAF9FAF219720E01E
:109E400030E040EA50E4C701B6010F94FFC46B0153
:109E50007C0184E08B150CF0D5CDC6CF872D982DD5
:109E6000A92DBA2D21968CAF9DAFAEAFBFAF219774
:109E700020E030E040EA50E4C701B6010F9400C58D
:109E800025966CAF7DAF8EAF9FAF2597B110D7CF22
:109E900020E030E040EA50E4612F702F832D922DB6
:109EA0000F94FFC4162F072F382E292E9DCFB110E7
:109EB0000FC020E030E040E251E4612F702F832D8D
:109EC000922D0F94FFC4162F072F382E292E9ACDCE
:109ED00094E082ED482E83E5582E8BEF682E81E4C6
:109EE000782E9B150CF096CD20E030E040E251E456
:109EF000612F702F832D922D0F94FFC421966CAF8C
:109F00007DAF8EAF9FAF21977DCD172D082D392CBA
:109F10002A2C6ACFFC0180E09491992331F0907C47
:109F2000903809F08F5F3196F7CF0895FC0180E0FB
:109F30009191992329F0907C9038D1F38F5FF8CFDD
:109F40000895AF92BF92CF92DF92EF92FF920F935C
:109F50001F93CF93DF93EC015B018A01FB011995FD
:109F600087FD16C0C82ED12CF12CE12C2196F801CA
:109F7000C082D182E282F382CE01DF91CF911F9124
:109F80000F91FF90EF90DF90CF90BF90AF9008952A
:109F9000982F907E903CA9F48F7190E0B0E0A0E003
:109FA0006C017D0156E0CC0CDD1CEE1CFF1C5A95AB
:109FB000D1F7CE010196F50119958F73C82A229623
:109FC000D6CF982F907F903E11F58F7090E0B0E043
:109FD000A0E06C017D0136E0CC0CDD1CEE1CFF1C0A
:109FE0003A95D1F7CE010196F50119958F73C82ADC
:109FF00046E0CC0CDD1CEE1CFF1C4A95D1F7CE01CF
:10A000000296F50119958F73C82A2396B0CF982F21
:10A01000987F903F79F5877090E0B0E0A0E06C0108
:10A020007D0186E0CC0CDD1CEE1CFF1C8A95D1F76F
:10A03000CE010196F50119958F73C82A96E0CC0CD4
:10A04000DD1CEE1CFF1C9A95D1F7CE010296F5019E
:10A0500019958F73C82A26E0CC0CDD1CEE1CFF1C62
:10A060002A95D1F7CE010396F50119958F73C82A69
:10A0700024967DCF982F907C903841F4807C803856
:10A0800069F42196CE01F5011995F8CF8E7F8D3FA9
:10A0900028F02196CE01F5011995F8CFC12CD12CCD
:10A0A000760165CF8F929F92AF92BF92CF92DF924F
:10A0B000EF92FF920F93FC01C080D180E280F38089
:10A0C0008090760890907708A0907808B0907908F2
:10A0D000A5019401C701B6010F940EBE8823E9F0D3
:10A0E00020E030E0A901C701B6010F940EBE88231D
:10A0F00009F484C0A5019401C701B6010F940EBEF6
:10A1000087FD7EC081E080937508C0927608D0926A
:10A110007708E0927808F09279088091091B8131E4
:10A1200098F480910B1B833078F08091750844E09F
:10A13000481B54E4E52E56E1F52E0CE022E062E4E3
:10A1400085ED9AE10F94E3AB8091091B853180F492
:10A1500080910B1B843160F041E4E42E46E1F42E43
:10A1600001E023E044E16CE385ED9AE10F94E3AB79
:10A170008091091B8F33C0F580910B1B8F32A0F1AA
:10A180008091750840E3481B87E2E82E86E1F82EAF
:10A190000DE022E06AE585ED9AE10F94E3AB809152
:10A1A000750841E3481B9DE0E92E96E1F92E22E077
:10A1B00065E085ED9AE10F94E3AB2DEDE22E25E10C
:10A1C000F22E00E123E04FE262E185ED9AE10F9487
:10A1D000E3AB3DEAE32E35E1F32E23E04FE267E601
:10A1E00085ED9AE10F94E3AB0F91FF90EF90DF9034
:10A1F000CF90BF90AF909F908F90089580E083CFD5
:10A200008FEF81CF9CE0899F802D112491E0980FE2
:10A21000909319092CE0280F2093590C30E02E5F01
:10A220003F4F4091091B4217130619F014F080E0CC
:10A23000089520910B1B9217D0F7662341F08E5F93
:10A240000F9491A98091590C8E5F0F9491A98091E0
:10A25000590C9091091B891750F320910B1B909179
:10A260001909291720F310920C1B80930D1B81E014
:10A27000089520917208022E000C330B82171306EA
:10A2800041F0809372086FEA78E185ED9AE10D94D0
:10A2900077AA08951F93CF93DF931F92CDB7DEB7B0
:10A2A0008F3F910519F014F08FEF90E088379105FA
:10A2B00014F488E790E09093560280935502182F8B
:10A2C00080910E1B811105C081E080930E1B0F94BD
:10A2D000B8A86091D71A7091D81A19839E012F5F80
:10A2E0003F4F4FE085ED9AE10F94B4A80F90DF91B6
:10A2F000CF911F910895CF938091730881114FC022
:10A3000010920C1B10920D1B10920E1B1092DA1A59
:10A310001092D91A1092DC1A1092DB1A1092DE1ADF
:10A3200081E08093DD1A82E28093DF1A1092E41AB2
:10A330001092E31AE8EFFAE126E03BE18FEF819318
:10A340002E173F07E1F7C1E0C093F51A29E932E083
:10A350003093EB1A2093EA1AC093EC1A1092ED1A7C
:10A360001092EE1A90E49093EF1A1092F01A2FEEDA
:10A3700032E03093071B2093061B23E132E0309339
:10A38000D81A2093D71A99E19093FA1A9BE19093E7
:10A39000F91A8093F81A0F94B8A8C09373088091A3
:10A3A0005502909156020E944A5181E080937408B0
:10A3B0008DEA95E19093EC198093EB191092EE19C8
:10A3C0001092ED19CF9108950E947B513E98469AC4
:10A3D0003C98449A3A98429A0E9478471092B6085C
:10A3E0000895CF92DF92EF92FF920F931F93CF9336
:10A3F000DF93CDB7DEB72C970FB6F894DEBF0FBE54
:10A40000CDBF6F3F71058105910509F0D0F481ED55
:10A410009AE10E947339E091D91AF091DA1A3196D3
:10A42000849190E02C960FB6F894DEBF0FBECDBF9E
:10A43000DF91CF911F910F91FF90EF90DF90CF9020
:10A440000895F0900C1BE0900D1B209174082111D1
:10A450000FC04DE855E16E2D8F2D0F943BAB90E072
:10A4600080E0F80EF0920C1BE0920D1B9927DACFDA
:10A47000C090D91AD090DA1A25ED3AE13A832983AF
:10A480002F2D30E03C832B832E2D30E03E832D8317
:10A4900018861F822FEF3FEF3A8729871C861B867D
:10A4A00001E119E39E012F5F3F4FAB01BC01C601E3
:10A4B0000F94F181B60185ED9AE10F9477AA8F810F
:10A4C0009885CFCF4F925F926F927F928F929F929B
:10A4D000BF92CF92DF92EF92FF920F931F93CF9391
:10A4E000DF9300D000D01F921F92CDB7DEB77C0162
:10A4F0006A014901FB0190818CE0989F800D112435
:10A50000982FF7012081822F880F820F880F809368
:10A510000C1B90930D1B4115510571F1FA82E982D4
:10A520007C836B83011121C0AE014B5F5F4FB4018F
:10A53000C6010E94A14F6C016D817E818F8198853B
:10A540006115710581059105B9F00E94F151F7017E
:10A5500080818F5F8083853138F3CE0101960E9420
:10A56000E137E2CFB12C860129C08A01B12C26C087
:10A57000452846284728B1F728960FB6F894DEBF3D
:10A580000FBECDBFDF91CF911F910F91FF90EF9044
:10A59000DF90CF90BF909F908F907F906F905F9053
:10A5A0004F900895B39407C0B1102EC00115110546
:10A5B000C9F20F5F1F4F01151105A9F2AE014B5FE4
:10A5C0005F4FB401C6010E94A14F6C014D805E80B7
:10A5D0006F8078844114510461047104A9F0F0E2A1
:10A5E0004F16510461047104F9F2D301C2018D9731
:10A5F000A109B1090297A105B10530F04BE244165B
:10A6000051046104710471F6F7018081482F4B0DEC
:10A610005527551F4631510534F0853020F0CE01C5
:10A6200001960E94E13781E04114510461047104F4
:10A6300009F480E0B80EF70180818B0D8083BB2088
:10A6400009F496CFBA94AE014B5F5F4FB401C801D5
:10A650000E94A14F8C016D817E818F8198850E941F
:10A66000F151EDCF2F923F924F925F926F927F9276
:10A670008F929F92AF92BF92CF92DF92EF92FF9212
:10A680000F931F93CF93DF9300D0CDB7DEB74C016C
:10A690003B015A01222E3B8328014091400C5091EE
:10A6A000410C6091420C7091430C411551056105BC
:10A6B000710579F081E0141615060CF080E08093A6
:10A6C00013091092400C1092410C1092420C1092FF
:10A6D000430C1091130930903D0C10923D0C311039
:10A6E00005C080917F02882309F472C0C2010E94D4
:10A6F0008A4F082F80E0C114D10419F0C6010E94CE
:10A700008A4F1A821982E114F104B1F4402F50E00B
:10A71000282F30E0CA01820F931F46976CF485E121
:10A7200090E0841B950B821B930B97FD01969595EA
:10A7300087958A8381E0898301E02BED37E3A201CD
:10A74000BE016F5F7F4FCE0102960E946252E114FC
:10A75000F10491F08A81882321F01A8289818F5F28
:10A76000898300E02EED37E3A701BE016F5F7F4FC5
:10A77000CE0102960E946252C114D10459F000E049
:10A780002BED37E3A601BE016F5F7F4FCE0102962E
:10A790000E94625241E04127B30181E00F940EAA6A
:10A7A000C4010E948A4F412FB40194E1981B892F64
:10A7B0000F940EAA332049F0111102C0A22CBB80C5
:10A7C000A114B104D9F0F501199581E08093200915
:10A7D0000F900F900F90DF91CF911F910F91FF90ED
:10A7E000EF90DF90CF90BF90AF909F908F907F9031
:10A7F0006F905F904F903F902F9008950E94CB45AF
:10A80000E4CFAF92BF92CF92DF92EF92FF920F937D
:10A810001F93CF93DF9300D01F92CDB7DEB77C019B
:10A82000062F6A01122F86E0A82EB12C11160CF00B
:10A8300040C0AE014F5F5F4F6BED77E3C7010E94F1
:10A84000A14F7C0169817A818B819C8161157105A1
:10A850008105910571F16D3371058105910509F44B
:10A8600050C06E3771058105910509F44AC06A32FE
:10A8700071058105910569F507FF12C082EA96E12D
:10A880000E3F11F08EE996E126E01202B00111248C
:10A890000E94D73A66E070E00F94E3C4161B61C0D3
:10A8A00065E470E080E090E00E94F151115059F5AC
:10A8B00010E0812F0F900F900F900F90DF91CF91AC
:10A8C0001F910F91FF90EF90DF90CF90BF90AF90CE
:10A8D0000895643271058105910579F4C114D1049C
:10A8E00061F026E01202B0011124C6010E94D73A9D
:10A8F000B5010F94E3C4161B99CF0E94F15111507A
:10A9000095CF07FDBBCF61E089819A81AB81BC8186
:10A91000CD97A105B10509F460E0600F6A30ACF095
:10A920001150862F6AE00F94C1C4092F682F880F39
:10A93000770B605D7F4F072E000C880B990B0E94F0
:10A94000F151112309F4B4CF602F062E000C770BC0
:10A95000605D7F4F072E000C880B990B0E94F15110
:10A960001150112309F4A4CF86E01802B00111247C
:10A97000C7010E94D73A66E070E00F94E3C4161B4B
:10A9800098CF6FEF7FEF0C94D73ACF93DF93FC0112
:10A9900025AD211104C021E025AF0F94B8A8C091C6
:10A9A000D71AD091D81AE091061BF091071B82E0CC
:10A9B0001995E091061BF091071B81E0199530E095
:10A9C00020E044E1BE0185ED9AE10F94B4A828E0AF
:10A9D0003BE147E1BE0185ED9AE10F94B4A8E09117
:10A9E000061BF091071B80E0DF91CF9119944F92E5
:10A9F0005F926F927F928F929F92AF92BF92CF920F
:10AA0000DF92EF92FF920F931F93CF93DF9300D0CB
:10AA10001F92CDB7DEB70F94D0A26B017C0180915D
:10AA20001B028F3FF1F10F94D0A28090AA08909062
:10AA3000AB08A090AC08B090AD08681979098A09F4
:10AA40009B0997FD2EC08091991A90919A1A8F5F59
:10AA50008F70891731F1E0911B0280E090E0A8E44B
:10AA6000B3E4E43050F424E0E29FF0011124E35514
:10AA7000FD4F80819181A281B38189839A83AB83C9
:10AA8000BC838E010F5F1F4F23E93DE04FE85DE07F
:10AA90006BE87DE087E89DE00F949F978FEF8093B0
:10AAA0001B020E94784780916007811116C00F94A5
:10AAB0002244882391F08091B508811110C091E063
:10AAC0009093B5088091840C892780933D0C109257
:10AAD000840C81E00E941A4802C01092B50880914F
:10AAE0005C0790915D07A0915E07B0915F07A70199
:10AAF0009601281B390B4A0B5B0BDA01C901B7FF22
:10AB000005C080911B09882309F4EAC1D701C60159
:10AB10008C599F4FAF4FBF4F80935C0790935D0759
:10AB2000A0935E07B0935F076091B608062E000CF5
:10AB3000770B77FF03C07195619571099091B60805
:10AB40008091B408981302C0633068F0633069F4F0
:10AB50008091B60887FD6BC081E0880F880F8093D5
:10AB6000B60864E002C01092B6088091B6088093DF
:10AB7000B408643008F05DC080913D0C8111DBC0E9
:10AB80008091CF1A9091D01A3DE58531930709F055
:10AB9000F6C080918002882309F4DFC08150809341
:10ABA00080020E9474FA8090C00D9090C10DA09018
:10ABB000C20DB090C30D81110F94594CD501C40141
:10ABC0003AE0B695A795979587953A95D1F700976E
:10ABD00051E0A507B10520F08FEF9FEFA0E0B0E0B6
:10ABE0009695879520917F022111F8C030911B091D
:10ABF0003111A4C18091CF1A9091D01A85519D45F1
:10AC000009F483C18091200981117FC18091B0082E
:10AC10009091B108A091B208B091B308C81AD90AAE
:10AC2000EA0AFB0AF7FC7FC10E946D447CC18FEFEA
:10AC300094CF8091500C21E030E040E050E0882338
:10AC400009F456C080904C0C90904D0CA0904E0C86
:10AC5000B0904F0C81149104A104B104E9F170E0AB
:10AC600090E080E00F9413BE20E030E040E85EE327
:10AC70000F9474BE2B013C01C701B6016819790914
:10AC80008A099B090F9413BE9B01AC01C301B20159
:10AC90000F94FAC520E030E04AE754E40F9474BE04
:10ACA0004B015C0120E030E042E053E40F9460C7C8
:10ACB00024E630E040E050E087FF12C020E030E0C2
:10ACC00040EA52E4C501B4010F9460C72AE030E0C5
:10ACD00040E050E087FF04C021E030E040E050E079
:10ACE000C0924C0CD0924D0CE0924E0CF0924F0C56
:10ACF000A091B6080A2E000CBB0B0F949EC424E052
:10AD000030E040E050E00F9474C48091400C90918A
:10AD1000410CA091420CB091430C820F931FA41FD1
:10AD2000B51F8093400C9093410CA093420CB093BC
:10AD3000430C1092B608D701C6018856954CAF4F08
:10AD4000BF4F8093B0089093B108A093B208B0931E
:10AD5000B30881E080937F0213CF8CE08093800260
:10AD60008091AE089091AF08009729F001979093D9
:10AD7000AF088093AE0881E080937F0212CF8754A2
:10AD80009C4B09F00ECF809180029FEF980F90931B
:10AD90008002811106CF80915D0C8F5F80935D0CE6
:10ADA00090915E0C24E0891708F02CE0209380023B
:10ADB000981710F410925D0C81E080937F02D70108
:10ADC000C6018856954CAF4FBF4F8093B008909303
:10ADD000B108A093B208B093B308E3CE009741F056
:10ADE0004091AE085091AF084817590708F002CFBC
:10ADF00080911B09811112C0223038F0243008F4F0
:10AE000041C0243011F410927F0281ED9AE10E943A
:10AE1000C55481E080931E0980931B0983E00E9442
:10AE2000395181E08093F51AE091CF1AF091D01A50
:10AE3000199510921E0980911B09811127C010924B
:10AE40003D0C8091CF1A9091D01A85519D4509F003
:10AE5000D9CE0F94D0A2DC01CB018C199D09AE098B
:10AE6000BF098090AE089090AF08B12CA12C881635
:10AE70009906AA06BB0608F0BDCE9093AF08809352
:10AE8000AE08B8CE81E080937F02BFCF85ED9AE116
:10AE90000F9445AA91E0811101C090E090931B09A5
:10AEA000882369F28091CF1A9091D01A85519D45DF
:10AEB000B9F40F94D0A2DC01CB018C199D09AE0925
:10AEC000BF09C090AE08D090AF08F12CE12CC81695
:10AED000D906EA06FB0620F49093AF088093AE08EB
:10AEE0000F900F900F900F90DF91CF911F910F91C6
:10AEF000FF90EF90DF90CF90BF90AF909F908F909A
:10AF00007F906F905F904F90089558E9C50E5AE377
:10AF1000D51EE11CF11CC092B008D092B108E0929D
:10AF2000B208F092B30880911B098111D9CF8091AA
:10AF30007F028130A9F610927F02D2CF009709F4E8
:10AF40006DCF4ECFCF92DF92EF92FF920F931F9370
:10AF5000CF93DF93CDB7DEB72C970FB6F894DEBF53
:10AF60000FBECDBFF0900C1BE0900D1B209174081C
:10AF700021111DC04DE455E16E2D8F2D0F943BAB7B
:10AF800090E080E0F80EF0920C1BE0920D1B9927E8
:10AF90002C960FB6F894DEBF0FBECDBFDF91CF91D8
:10AFA0001F910F91FF90EF90DF90CF900895C09088
:10AFB000D91AD090DA1A25ED3AE13A8329832F2D58
:10AFC00030E03C832B832E2D30E03E832D8318868A
:10AFD0001F827A8769871C861B8601E119E39E011F
:10AFE0002F5F3F4F4EED57E3BC01C6010F94B58272
:10AFF000B60185ED9AE10F9477AA8F819885C2CF2B
:10B00000BF92CF92DF92EF92FF920F931F93CF9355
:10B01000DF938B01F42EE90141FB662760F90E9462
:10B020000251882309F45AC0B12C0115110521F0F1
:10B03000C8010E948A4FB82EE12C209721F0CE0142
:10B040000E94964FE82E80E8C82ED12CF0FE1EC03C
:10B0500085E190E08B199109B7FC93958E199109C0
:10B06000E7FC939597FD019695958795F82E30E826
:10B07000C32ED12CFA94F7FC09C060E270E080E0A6
:10B0800090E00E94F151C81AD90AF4CFBB2099F080
:10B09000C60166E070E00F94CFC4262F40915B0C90
:10B0A00050915C0C60915A0CC8010E94015496E0CA
:10B0B000899F60011124EE2031F0B601CE010E947B
:10B0C000A257C81AD90A87E0C816D10438F060E23E
:10B0D00070E080E090E00E94F151F3CFDF91CF91DA
:10B0E0001F910F91FF90EF90DF90CF90BF90089548
:10B0F00080917F02882351F06091090970910A09BB
:10B1000030E020E041E081E00C94005808956FEFBA
:10B110007FEF0C94A257AF92BF92CF92DF92EF9243
:10B12000FF920F931F93CF93DF935C016B010E94FB
:10B130008A4FE82EC6010E94964FF12C03E110E0E1
:10B14000081B1109C5E20E151F050CF4CFE18C2F69
:10B1500090E09C012E5F3F4F4091091B4217130660
:10B1600009F0CCF5099720910B1B281719069CF1C3
:10B1700040915B0C50915C0C60915A0C10920C1B2E
:10B18000C0930D1B25E1C5010E940154D1E0C114FB
:10B19000D104B1F06AE370E080E090E00E94F151E8
:10B1A0000E151F05D4F4C45F8091091BC81740F029
:10B1B00020910B1B4C2F4950550B241715067CF47E
:10B1C000DF91CF911F910F91FF90EF90DF90CF9083
:10B1D000BF90AF900895D0E0DACFDD2389F3802FC0
:10B1E000880F080F000F00930C1BC0930D1B60E22B
:10B1F00070E080E090E00E94F151C601DF91CF91B4
:10B200001F910F91FF90EF90DF90CF90BF90AF9084
:10B210000C948758CF92DF92EF92FF92CF93DF93F7
:10B2200080913D0C10923D0C882351F01092200922
:10B23000DF91CF91FF90EF90DF90CF900C94CB45B2
:10B2400081E0809320098091400C9091410CA09165
:10B25000420CB091430C0097A105B10509F44BC015
:10B260002AE0289FE001299FD00D11241092400C64
:10B270001092410C1092420C1092430CBE010D2E04
:10B28000000C880B990B0F9415BE2091CE0D3091B8
:10B29000CF0D4091D00D5091D10D0F9474BE2091DF
:10B2A000901A3091911A4091921A5091931A0F94DA
:10B2B00000C56B017C0120E030E040E151EC0F94CF
:10B2C00060C787FD18C020E030E040E151E4C701CD
:10B2D000B6010F940EBE181674F0CE010F9409A398
:10B2E000C092901AD092911AE092921AF092931A08
:10B2F00082E080937F0280917F02882399F080E929
:10B300009AE10F94D49BBC0180E698E10E948B588F
:10B3100080E99AE1DF91CF91FF90EF90DF90CF909D
:10B320000C945250DF91CF91FF90EF90DF90CF902F
:10B3300008950F931F93CF93DF93FC01EB0180914E
:10B34000400C9091410CA091420CB091430CB7FF7E
:10B3500008C01092400C1092410C1092420C1092B6
:10B36000430C8091F7089091F808A091F908B091EA
:10B37000FA084091400C5091410C6091420C709140
:10B38000430C84179507A607B70744F48093400C35
:10B390009093410CA093420CB093430C80917F0298
:10B3A0008823E1F06091400C7091410C8091420C37
:10B3B0009091430C0091FB081091FC082091FD082E
:10B3C0003091FE08600F711F821F931F1995BC01F9
:10B3D00080910109909102090E948B5880913D0C47
:10B3E000811108C08091F4088823D1F180917F02F7
:10B3F0008823B1F18091FF08909100090097B1F086
:10B400004091400C5091410C6091420C7091430C62
:10B410000091FB081091FC082091FD083091FE0876
:10B42000400F511F621F731FFE011995E091F5082F
:10B43000F091F608309741F08091F408811103C033
:10B4400080913D0C8111199580913D0C10923D0C1D
:10B45000882331F0DF91CF911F910F910C94CB4550
:10B46000DF91CF911F910F9108958F929F92AF928C
:10B47000BF92CF92DF92EF92FF920F931F93CF93E1
:10B48000DF93CDB7DEB72C970FB6F894DEBF0FBEB3
:10B49000CDBF982F862F5A017901D02E692F0E9497
:10B4A0000251882309F487C010917408C701002352
:10B4B00081F10E948A4FC82E8090D91A9090DA1A92
:10B4C000111143C01FEF23E12C1940915B0C5091E7
:10B4D0005C0C60915A0CC5010E940154CC2009F407
:10B4E0006AC0B6E08B9F500111246AE370E080E0EF
:10B4F00090E00E94F15157E0A516B10408F442C053
:10B5000060E270E080E090E00E94F151A81AB90A70
:10B51000F2CF0E94964FC82E8090D91A9090DA1AD6
:10B52000112381F2FE0133968AE0DF011D928A9594
:10B53000E9F785ED9AE19A83898308EE18E39E0185
:10B540002F5F3F4F4EED57E312C0FE0133968AE066
:10B55000DF011D928A95E9F785ED9AE19A83898347
:10B5600008EE18E39E012F5F3F4F4BED57E3B70105
:10B57000C4010F94B582B40185ED9AE10F9477AAC6
:10B580001F81A1CF4091590C212F30E0A6E0CA9E27
:10B59000C00111242E5F3F4F281739070CF49C017E
:10B5A00080E8821B80930C1B40930D1BC701DD209C
:10B5B000A9F00E94C1542C960FB6F894DEBF0FBEBE
:10B5C000CDBFDF91CF911F910F91FF90EF90DF9052
:10B5D000CF90BF90AF909F908F9008950E94875812
:10B5E000EACF2F923F924F925F926F927F928F920B
:10B5F0009F92AF92BF92CF92DF92EF92FF920F9302
:10B600001F93CF93DF9300D000D0CDB7DEB761E0BA
:10B6100081E00E948C438091450C8D83582E8B5F76
:10B6200089834424439473E0372EE4EE6E2EEDEDCF
:10B630007E2E82E085198A83942D95199B83852D12
:10B6400081958C83232C25188D81811181C0809157
:10B65000440C882309F455C080917F02882359F057
:10B6600081E09091440C911180E024E04FE25FE191
:10B670006C810F94939B8091B00C882309F435C1A1
:10B680008D81833009F05CC18091440C833009F4D2
:10B69000CDC080917F0281110EC194E09E838E8186
:10B6A0008F5F9D81891322C08091440C891709F412
:10B6B0007FC180917F028823C9F011E08091440C02
:10B6C0009D81891310E06091CF097091D00980911C
:10B6D000D1099091D2090E94D0C700E09C014FE6A9
:10B6E00058E16D816519812F0E94355A8D818F5FD8
:10B6F0008D8399818913A8CF8E818E5F80933E0CB4
:10B700000EC080913D0C10923D0C882309F4A4CF0B
:10B710000E94CB4580913F0C882309F49DCF26964B
:10B720000FB6F894DEBF0FBECDBFDF91CF911F9152
:10B730000F91FF90EF90DF90CF90BF90AF909F90D0
:10B740008F907F906F905F904F903F902F900895D3
:10B750009D819130A1F58091440C8130F9F0809168
:10B760007F02882309F487CF81E08E838091440C87
:10B77000813009F01E826091BC0D7091BD0D8091E9
:10B78000BE0D9091BF0D0E9495C600E09C0145E959
:10B7900058E16B818E810E94355A6DCF80913D0CAE
:10B7A00010923D0C8823D9F26CEB7DE085E998E19D
:10B7B0000F94B29E80913F0C882389F2B0CF9D8177
:10B7C000923009F058CF8091440C8230C1F08091C2
:10B7D0007F02882309F44FCF81E09091440C92308E
:10B7E00009F080E09091B00C2AE43EE1911102C092
:10B7F00026E43EE101E04BE858E16A81CCCF80913C
:10B80000B00C90913D0C10923D0C992301F38425CE
:10B810008093B00C30927F026114710411F00E9489
:10B82000E4DD80913F0C882391F279CF80913D0C2B
:10B8300010923D0C882309F42CCF0F94EE9C20E04D
:10B8400030E04AE754E46091AC0C7091AD0C80910B
:10B85000AE0C9091AF0C0F9474BE20E030E0A901C3
:10B860000F9400C520E030E84BEB54E40F94FFC484
:10B870000F9473C61F9244EE842E4DED942E5FE616
:10B88000A52E56E9B52E6B0116EDE12E16E0F12E30
:10B8900000E010E02CED35E040E050E06CEA7CE0A8
:10B8A00081E898E10E9409460F9080913F0C88231F
:10B8B00009F4EFCE34CF81E08E838091440C833045
:10B8C00009F01E826091AC0C7091AD0C8091AE0CB1
:10B8D0009091AF0C0E9411C800E09C0141E858E132
:10B8E000622D8E810E94355AD8CE83E08E838E8160
:10B8F0009D818913D4CE8091440C9E81891719F1C2
:10B9000080917F02882309F4CACEFD80F51811E0EA
:10B910008091440C9D81891310E06091CB09709156
:10B92000CC098091CD099091CE090E94D0C700E04A
:10B930009C0147E758E16F2D812F0E94355AAFCE09
:10B9400094E09E83D4CF80913D0C10923D0C8823CF
:10B95000B9F20F94EE9C20E030E0A9016091CB0990
:10B960007091CC098091CD099091CE090F9400C5BA
:10B970000F9473C61F92912C812C29E6A22E26E9E2
:10B98000B22E6B011EEEE12E12E0F12E00E010E06F
:10B9900020E030E0A9016BEC79E087E798E10E94B4
:10B9A00009460F9080913F0C882309F4A9CFB7CEA8
:10B9B00080913D0C10923D0C882309F47ACE0F94AF
:10B9C000EE9C20E030E0A9016091CF097091D00990
:10B9D0008091D1099091D2090F9400C50F9473C63C
:10B9E0001F92912C812C89E6A82E86E9B82E6B0136
:10B9F0001EEEE12E12E0F12E00E010E020E030E03B
:10BA0000A9016FEC79E08FE698E10E9409460F905A
:10BA100080913F0C882309F44CCE81CEE1EDFAE110
:10BA200083AF64AFCA010C9487584F925F926F92B4
:10BA30007F928F929F92AF92BF92CF92DF92EF92BE
:10BA4000FF920F931F93CF93DF9300D01F921F920B
:10BA5000CDB7DEB71092500C80913D0C10923D0C8A
:10BA60008823F9F020E040E070E060E08AE09EEB9F
:10BA70000E94EA430F900F900F900F900F90DF916C
:10BA8000CF911F910F91FF90EF90DF90CF90BF90DB
:10BA9000AF909F908F907F906F905F904F900C949D
:10BAA0007B5120918102309182024091400C509153
:10BAB000410CCA01820F931F2436310509F066C478
:10BAC0004730510544F006978A3091050CF06DC45B
:10BAD0008AE090E074C406964A3F5F4FACF38091D1
:10BAE0001E09882309F4DAC181E04091FB195091C5
:10BAF000FC192091F9193091FA19241735070CF027
:10BB000080E040919D0C50919E0C20919B0C3091B7
:10BB10009C0C241735070CF482608093A9082091AF
:10BB20007B0D30917C0D40917D0D50917E0D60918B
:10BB3000870D7091880D8091890D90918A0D0F94D9
:10BB400000C54B015C0120917F0D3091800D40912B
:10BB5000810D5091820D60918B0D70918C0D8091B3
:10BB60008D0D90918E0D0F9400C569837A838B8320
:10BB70009C832091830D3091840D4091850D5091CF
:10BB8000860D60918F0D7091900D8091910D909127
:10BB9000920D0F9400C52B013C0120E030E040E203
:10BBA00051E40F9474BE20E030E048EC52E40F946E
:10BBB00074BE6B017C0120E030E0A901C301B20139
:10BBC0000F940EBE20E030E040EA50EC87FD04C048
:10BBD00020E030E040EA50E4C701B6010F9400C510
:10BBE00020E030E040E251E40F94FAC50F946CC6B7
:10BBF0002B013C0180E277FE09C070946094509460
:10BC00004094411C511C611C711C8DE28093510CAD
:10BC100060E2F0E14F16F7E25F06610471048CF018
:10BC2000C301B20120E137E240E050E00F9474C458
:10BC3000CA01B9012AE030E040E050E00F9474C43A
:10BC4000605D6093520C60E248EE441643E0540697
:10BC5000610471048CF0C301B20128EE33E040E0CE
:10BC600050E00F9474C4CA01B9012AE030E040E00A
:10BC700050E00F9474C4605D6093530CC301B20133
:10BC800024E630E040E050E00F9474C46AE0C62E31
:10BC9000D12CE12CF12CCA01B901A70196010F9416
:10BCA00074C4605D6093540CC301B201A701960196
:10BCB0000F9474C46D83CA01B901A70196010F9452
:10BCC00074C49D81992309F48AC38EE28093550C34
:10BCD000605D6093560C905D9093570C61E57CE03D
:10BCE00081EA98E00F94ACC920E030E0A901C501D9
:10BCF000B4010F940EBE20E030E040E05FEB87FD22
:10BD000004C020E030E040E05FE3C501B4010F94DF
:10BD100000C50F946CC6CB010F944E25BC018CE975
:10BD200098E00F94ACC920E030E0A90169817A81E4
:10BD30008B819C810F940EBE20E030E040E05FEBF1
:10BD400087FD04C020E030E040E05FE369817A8154
:10BD50008B819C810F9400C50F946CC6CB010F940E
:10BD60004E25BC0187E998E00F94ACC9E091030926
:10BD7000EF77E983E11127C00F94D34C882319F1A1
:10BD80008091131B9091141BA091151BB091161B51
:10BD90000097A105B105B9F0BC01CD016D597F4FE8
:10BDA0008F4F9F4F24E630E040E050E00F9452C4A4
:10BDB0006091171B7091181B8091191B90911A1B91
:10BDC0000F9452C429830F949D22162FA72EB82EAC
:10BDD000092FF62E80911A02F9818F17C9F0F0937E
:10BDE0001A0248E4F49FB001112490E080E00F941F
:10BDF00013BE2AE037ED43E25CE30F9474BE0F9468
:10BE000073C66093960869816111FBC21092910814
:10BE100080911902F81609F441C010931902612F9C
:10BE20007A2D8B2D902F20E13EE040E050E00F94E2
:10BE300052C469012CE3422E512C612C712C612FCC
:10BE40007A2D8B2D902FA30192010F9452C4CA0119
:10BE5000B901A30192010F9452C4E4E6CE16D104B5
:10BE600008F0F7C27F936F93DF92CF9286EB96E153
:10BE70009F938F9381E898E09F938F930F94A5BD34
:10BE80000FB6F894DEBF0FBECDBF85E0982F990F97
:10BE9000990F891B880F8058809380080E9443481F
:10BEA000898381E00E9439518091091B863180F499
:10BEB00080910B1B833060F095E9E92E97E1F92E14
:10BEC00003E123E043E068E085ED9AE10F94E3AB02
:10BED0008091A908982F927042E102E081FF02C090
:10BEE00048E00CE08091091B843180F480910B1BA9
:10BEF000841760F0992309F4C1C281E797E17C01BE
:10BF000023E068E485ED9AE10F94E3AB8091091B8F
:10BF10008431C0F480910B1B8230A0F0F981FF23A3
:10BF200009F4AFC28091C40D882309F4AAC285E345
:10BF300097E17C0102E123E042E068E685ED9AE1C9
:10BF40000F94E3AB8091091B8C3108F00CC1C090B9
:10BF5000F919D090FA19A090FB19B090FC1984310E
:10BF600098F480910B1B883078F08091A90880FFAD
:10BF70008BC287EE96E17C010CE022E048E068E2AB
:10BF800085ED9AE10F94E3AB8091091B883048F569
:10BF90004981411104C08091E409811122C0C50189
:10BFA0000F94F825FC01808193E0803229F481818F
:10BFB00092E0803209F491E043E050E0491B5109DE
:10BFC0004E0F5F1F892F880F880F981B892F67E0FE
:10BFD000815D0E940E5D69E070E080E090E00E946B
:10BFE000F1518091091B8C3130F580910B1B84310C
:10BFF00010F1C6010F94F825FC01808193E0803296
:10C0000029F4818192E0803209F491E043E050E02C
:10C01000491B51094E0F5F1F892F880F880F981BEE
:10C02000892F6CE1815D0E940E5D69E070E080E027
:10C0300090E00E94F15100919B0C10919C0C80911A
:10C04000091B883060F56981611104C08091E9099C
:10C05000811125C080919D0C90919E0C0F94F82524
:10C06000FC01808193E0803229F4818192E080326A
:10C0700009F491E043E050E0491B51094E0F5F1F66
:10C08000892F880F880F981B892F67E08E5A0E948E
:10C090000E5D69E070E080E090E00E94F1518091D7
:10C0A000091B8C3130F580910B1B843110F1C801D4
:10C0B0000F94F825FC01808193E0803229F481817E
:10C0C00092E0803209F491E043E050E0491B5109CD
:10C0D0004E0F5F1F892F880F880F981B892F6CE1E7
:10C0E0008E5A0E940E5D69E070E080E090E00E9450
:10C0F000F1518091091B8C31B0F580910B1B84317B
:10C1000090F19091C40D292F30E02115310559F19E
:10C1100089818111BCC18091640287FDB8C1989F5B
:10C1200090011124220F232F221F330B31951AE285
:10C1300044E6429FC001439F900D112481589F4FB8
:10C140006FEF70E00F94E3C4CB010F94F825AC01BE
:10C150006CE187E60E940E5D612F110F770B880B53
:10C16000990B0E94F1510F94D34C882369F180916F
:10C17000091B843348F580910B1B8A3228F107E0B4
:10C1800028E04AE26AE285ED9AE10F94F1A905E020
:10C1900022E04CE262E385ED9AE10F94F1A96AE0B6
:10C1A0008AE20F94AAA96091D71A7091D81A82E3F3
:10C1B0008093F11A8BE28093F21A21EF3AE142E385
:10C1C00085ED9AE10F94B4A88091091B853340F462
:10C1D00080910B1B813320F06AE486E30F94AAA9B7
:10C1E0008091091B843368F480910B1B823348F0E3
:10C1F00002E02091960842E367E385ED9AE10F940F
:10C20000F1A98091091B8033D8F480910B1B8832EF
:10C21000B8F080919108882361F041E958E060E32B
:10C2200087E30E940E5D65E270E080E090E00E948E
:10C23000F15141E858E060E3809180080E940E5D72
:10C240008091091B873208F050C080910B1B8F3101
:10C2500008F44BC083E080930C1B16E210930D1B77
:10C2600068E570E080E090E00E94F1518BE08093FF
:10C270000C1B10930D1B9981992309F40AC18CE9B9
:10C2800098E00E94875888E280930C1B16E2109376
:10C290000D1B69E570E080E090E00E94F15180E3C1
:10C2A00080930C1B10930D1BF981FF2309F412C11D
:10C2B00087E998E00E9487588DE480930C1B16E272
:10C2C00010930D1B6AE570E080E090E00E94F15150
:10C2D00085E580930C1B10930D1BF981FF2309F456
:10C2E0001CC181EA98E00E9487588091091B833322
:10C2F00038F580910B1B8B3218F183E00E94395185
:10C3000083E080930C1B83E380930D1B66E070E059
:10C3100080E090E00E94F15181E00E9439518091CB
:10C320008102909182020F94F825AC0163E38CE0C6
:10C330000E940E5D65E270E080E090E00E94F151A5
:10C340008091091B813408F084C180910B1B8633D6
:10C3500008F47FC110920C1B8EE380930D1B8AE8BA
:10C3600097E10E94964F182F863108F0FBC08AE8AB
:10C3700097E10E948758153109F46BC160E270E0C3
:10C3800080E090E00E94F1511F5FF5CF2436310527
:10C390004CF48536910504F58A30910534F48AE031
:10C3A00090E009C084369105BCF0883EE3E09E072A
:10C3B00014F087EE93E02817390709F490CB909397
:10C3C0008202809381021092400C1092410C1092D4
:10C3D000420C1092430C83CB84E690E0F0CF6623AE
:10C3E00051F08EE28093550C605D6093560C80E2B4
:10C3F0008093570C73CC80E28093560C8093550C3D
:10C40000F6CF8981843608F164E60F94B5C4805D67
:10C410008093550C99819A30D0F02AE0892F622FB1
:10C420000F94B5C40F94B5C4905D9093560C898158
:10C430006AE00F94B5C4905D9093570C65E57CE07D
:10C4400081E998E00F94ACC9E3CC80E2E1CF90E2BF
:10C45000ECCF7F936F93DF92CF928CEA96E19F931C
:10C460008F9381E898E09F938F930F94A5BD0FB6AB
:10C47000F894DEBF0FBECDBF86E008CD8BE697E116
:10C480003ECD8FEF96E155CD8FEC96E174CD15E260
:10C490004FCE87E00F94070B80FF13C00CE918E024
:10C4A000F80161918F01662309F4EDCE6F320CF033
:10C4B0006FE3062E000C770B880B990B0E94F1514D
:10C4C000EFCF8091E40B80FDDACE8AEC96E10E94FA
:10C4D000C154D9CE87E00F94070B869580FF13C017
:10C4E00007E918E0F80161918F01662309F4E4CEB1
:10C4F0006F320CF06FE3062E000C770B880B990B54
:10C500000E94F151EFCF8091E40B869580FDD0CE53
:10C510008AEC96E10E94C154CFCE87E00F94070BBE
:10C520008695869580FF13C001EA18E0F8016191B5
:10C530008F01662309F4D9CE6F320CF06FE3062E1B
:10C54000000C770B880B990B0E94F151EFCF809173
:10C55000E40B8695869580FDC4CE82EC96E10E9420
:10C56000C154C3CE80917F08F981F817B1F01091C2
:10C570008917F0937F088AE897E10E94964F181771
:10C5800008F064C01F5FE12FF0E0E657F84E8081AD
:10C59000807C8038B9F3109389170091891710E0D7
:10C5A0000657184EC8010E94964F898360E870E0D4
:10C5B000C8010E94A2574981453108F04AC060E293
:10C5C00070E080E090E00E94F1516981643109F4EB
:10C5D00040C060E270E080E090E00E94F15189810B
:10C5E0008331B9F160E270E080E090E00E94F151A7
:10C5F0009981923171F1292F30E02E5F3F4F4AEF40
:10C600004203B001439F700D112460587F4F8AE8A8
:10C6100097E10E94A25760E270E080E090E00F9006
:10C620000F900F900F900F90DF91CF911F910F916E
:10C63000FF90EF90DF90CF90BF90AF909F908F9042
:10C640007F906F905F904F900C94F15110928917EA
:10C65000A4CF0F900F900F900F900F90DF91CF917C
:10C660001F910F91FF90EF90DF90CF90BF90AF9010
:10C670009F908F907F906F905F904F9008952F9232
:10C680003F924F925F926F927F928F929F92AF9262
:10C69000BF92CF92DF92EF92FF920F931F93CF93AF
:10C6A000DF93D62FC72FFC0180809180A280B380BA
:10C6B000C501B40120E831E541E050E00F9452C4D7
:10C6C000C9016DE671E00F94CFC46B017C01C50117
:10C6D000B40120E13EE040E050E00F9452C4CA01B2
:10C6E000B90128E130E040E050E00F9452C4362E0A
:10C6F000272E062F172F8CE3482E512C612C712CDE
:10C70000C501B401A30192010F9452C4B62EA72E05
:10C71000CA01B901A30192010F9452C4CB01C11403
:10C72000D10479F1AF92BF927F936F932F923F9292
:10C73000FF92EF92DF92CF928BEA93E19F938F93D8
:10C74000CF93DF930F94A5BD8DB79EB70E960FB60E
:10C75000F8949EBF0FBE8DBF8D2F9C2FDF91CF9180
:10C760001F910F91FF90EF90DF90CF90BF90AF900F
:10C770009F908F907F906F905F904F903F902F9001
:10C780000895E114F104C9F0AF92BF927F936F93C3
:10C790002F923F92FF92EF928BE993E19F938F93B9
:10C7A000CF93DF930F94A5BDEDB7FEB73C960FB6C0
:10C7B000F894FEBF0FBEEDBFCFCF012BB9F0AF9203
:10C7C000BF927F936F932F923F928FE893E19F9355
:10C7D0008F93CF93DF930F94A5BD8DB79EB70A9625
:10C7E0000FB6F8949EBF0FBE8DBFB6CF892BA9F0B0
:10C7F000AF92BF927F936F9387E893E19F938F935C
:10C80000CF93DF930F94A5BDEDB7FEB738960FB663
:10C81000F894FEBF0FBEEDBF9FCFAF92BF9283E8EB
:10C8200093E19F938F93CF93DF930F94A5BD0F90C8
:10C830000F900F900F900F900F908ECFAB01BC0117
:10C840004093171B5093181B6093191B70931A1B6E
:10C8500080E89CE10C94E4E6CF93DF93DB01F901DF
:10C860009C919130C1F0943080F094509C9388302A
:10C87000D1F480819181009771F001979183808339
:10C88000480F591FEA01188206C08C3539F49C5FA5
:10C890009C93943041F4DF91CF9108958B3339F715
:10C8A00081E08C93F8CF20813181B9016F5F7F4F98
:10C8B00071836083420F531FEA01888380819181D5
:10C8C0008F3591056CF7E7CF0F931F9381E00091AF
:10C8D000171B1091181B2091191B30911A1B4091A6
:10C8E000131B5091141B6091151B7091161B04179C
:10C8F00015072607370708F480E01F910F91089568
:10C900004F925F926F927F928F929F92AF92BF925F
:10C91000CF92DF92EF92FF920F931F93CF931092DB
:10C920007108109270082FE320936F0810926E0820
:10C9300010926D0810926C081092580710925907C7
:10C9400010925A0710925B079C01F90190812F5FAA
:10C950003F4F9032D1F39E34C9F4818190ED980F0E
:10C960009A3020F08D3211F08B3281F432969F0193
:10C970002F5F3F4F808180538A3008F47EC09F0133
:10C980002F5F3F4F8081803209F479C0F093880C8B
:10C99000E093870C8F010F5F1F4FC0816AE270E048
:10C9A000C8010F94A1C9009731F0FC013197808133
:10C9B0008032E1F31182CD3429F0C43519F0C73447
:10C9C00009F04BC0F80180810F5F1F4F8032D1F317
:10C9D00080538A3008F041C0C0936F0890E080E037
:10C9E0004AE0DF011196489F9001499F300D1124C4
:10C9F000C901C0972081820F911D27FD9A95218141
:10CA000030ED320F3A30E8F190936E0880936D0864
:10CA10002E3261F4329630E04AE0DF0131962C91FB
:10CA200050ED520F5A3078F130936C089D01D901C6
:10CA30002F5F3F4F4C914032D1F3CD34A1F58E3171
:10CA4000910539F030F58731910519F08C31910558
:10CA500051F5B0937108A0937008CF911F910F9179
:10CA6000FF90EF90DF90CF90BF90AF909F908F900E
:10CA70007F906F905F904F900895F90178CFF90102
:10CA80007ECFFD01AECF349F200D112430ED320F4B
:10CA9000C4CF8537910538F087379105D0F2803AB9
:10CAA00023E09207B1F25091870C70E060E0C12C56
:10CAB000D12C7601C394FD0131964C91442309F4A5
:10CAC00092C04132A1F4CD3491F48032910579F4D1
:10CAD000F0937108E093700863E270E0CF010F9467
:10CAE000A1C9009709F4B9CFFC011082B6CF415417
:10CAF0004A3108F073C0DF012D91203209F459C08A
:10CB000030ED320F3A3008F465C02E3209F053C0D0
:10CB1000218120532A3008F45DC030E020E0611507
:10CB2000710519F4BF0161507109A42FB0E026010D
:10CB3000370104C0440C551C661C771C4A95D2F77B
:10CB40008090580790905907A0905A07B0905B07C3
:10CB500084289528A628B7288092580790925907CC
:10CB6000A0925A07B0925B0721153105A9F1251B48
:10CB7000A25CB84F2C9320812154DF012A3108F4A4
:10CB80009ACFDF012191222309F495CF30ED320FA6
:10CB90003A30B8F333ED320F323098F32B3289F359
:10CBA0009D012F5F3F4F4C91403209F084CFD90156
:10CBB000F7CFFD01A0CF2D3219F02B3209F0ADCF08
:10CBC000218130ED320F3A3028F02E3209F0A5CF16
:10CBD00022819FCF9F01A9CF20E0CACF61157105A7
:10CBE00051F6BD01C8CF709371086093700835CFBE
:10CBF000CF93DF93EC018991882319F00F94514F63
:10CC0000FACF8DE00F94514F8AE0DF91CF910D94D0
:10CC1000514FFC01659175918591949108952F92E2
:10CC20003F924F925F926F927F928F929F92AF92BC
:10CC3000BF92CF92DF92EF92FF920F931F93CF9309
:10CC4000DF93CDB7DEB7C654D1090FB6F894DEBF77
:10CC50000FBECDBF70E060E085E40F940F43182F46
:10CC60008F3F09F484C08823E9F089E295E1CA5B2B
:10CC7000DF4F0FB6F894DEBF0FBECDBFDF91CF916F
:10CC80001F910F91FF90EF90DF90CF90BF90AF90EA
:10CC90009F908F907F906F905F904F903F902F90DC
:10CCA0000D94DC4F24EB30E03A83298383E50F9425
:10CCB000D642882321F00F9454429A83898365E0F9
:10CCC00070E083E40F940F438AA760E085E50F943A
:10CCD000FA4225968FAF259760E08CE195E10E949E
:10CCE0009746A981BA81BD01BB0F880B990B0F94A0
:10CCF00015BE6D837E838F8327969FAF27970F94F2
:10CD0000D0A2688B798B8A8B9B8B1F3F09F046C41E
:10CD100020E030E04CE053E46D817E818F812796E6
:10CD20009FAD27970F9460C718160CF0ABC181EF29
:10CD300094E10F94DC4F80E0CA5BDF4F0FB6F894AC
:10CD4000DEBF0FBECDBFDF91CF911F910F91FF903E
:10CD5000EF90DF90CF90BF90AF909F908F907F909B
:10CD60006F905F904F903F902F900C94334746E424
:10CD700050E05A8349839ACF1FAEAFC12496EEADDF
:10CD8000FFAD2497808383C2FBEE4F2E512C612C84
:10CD9000712C04C384E190E0A0E0B0E08C8B9D8B0B
:10CDA000AE8BBF8BE4E14E2E512C612C712C04C351
:10CDB0004C8A5D8A6E8A7F8AFFC22496EEADFFADF3
:10CDC00024978083D4C389819A81AB81BC8129A9AE
:10CDD0003AA94BA95CA9821B930BA40BB50BB7FD19
:10CDE00059C08FAD0F94E82E8AE00F94514F89817E
:10CDF0009A81AB81BC818053984FAF4FBF4F89ABB5
:10CE00009AABABABBCAB9DA9911177C02EA93FA942
:10CE100048AD59ADB101802F26969FAD26970F944E
:10CE200060C718160CF053C020E030E040E050E43A
:10CE3000B101802F26969FAD26970F9400C56EAB4B
:10CE40007FAB88AF99AF2CA53DA54EA55FA5898185
:10CE50009A81AB81BC81280F391F4A1F5B1F2AAF03
:10CE60003BAF4CAF5DAF20E030E040EC50E46D8173
:10CE70007E818F8127969FAD27970F94FFC49101E4
:10CE8000402F26965FAD26970F940EBE881F8827E9
:10CE9000881F8DAB88899989AA89BB89C816D9064C
:10CEA000EA06FB0610F4D701C60129813A814B81BD
:10CEB0005C81281B390B4A0B5B0BDA01C9018138F5
:10CEC0009F44A241B105A8F18DE394E10EC289818E
:10CED0009A81AB81BC812AAD3BAD4CAD5DAD821B6F
:10CEE000930BA40BB50B48E25CE367E37CE3B7FD6F
:10CEF000D1CF812F0E9409F0CDCF20E030E040EF6C
:10CF000051E46D817E818F8127969FAD27970F9485
:10CF1000FFC49B01AC01B101802F26969FAD2697DF
:10CF20000F940EBE87FFB6CF44ED5CE364EE7CE366
:10CF3000E0CF4AA55BA5888D998D481759070CF05D
:10CF40009EC003970CF49BC080EE93E10F94DC4FDE
:10CF50001F3F09F076C0A0EDB3E1BA83A9838FEB40
:10CF600093E10F94DC4F89819A810F94DC4F4885BF
:10CF700059856A857B858CED93E10F9499528AE0FF
:10CF80000F94514F8FEB93E10F94DC4F89819A817D
:10CF90000F94DC4F49A15AA16BA17CA188ED93E1CC
:10CFA0000F9499528AE00F94514F8FEB93E10F94B5
:10CFB000DC4F89819A810F94DC4FB501A40184ED87
:10CFC00093E10F9499528AE00F94514F2596FFAD4B
:10CFD0002597FF2391F12CEA35EC47E25EE369A146
:10CFE0007AA18BA19CA10F9474BE6B017C012CEAE9
:10CFF00035EC47E25EE3C501B4010F94FAC528851C
:10D0000039854A855B851F3F09F52093A00C309335
:10D01000A10C4093A20C5093A30CC092A40CD092EC
:10D02000A50CE092A60CF092A70C6093A80C70934C
:10D03000A90C8093AA0C9093AB0C81E080936602BC
:10D040007ACEEDE9FCE6FA83E98389CF2093FE19D5
:10D050003093FF194093001A5093011AC092021A9C
:10D06000D092031AE092041AF092051A6093061AFD
:10D070007093071A8093081A9093091ADECF0E94C2
:10D08000F75480C08DED94E10F94DC4F0E94FCEECC
:10D090008FE780939F0C24EB30E0A8EEB3E00F9471
:10D0A000A6C46CA77DA78EA79FA7288939894A891E
:10D0B0005B89260F371F481F591F2AAF3BAF4CAF64
:10D0C0005DAF1092660281E080937E0232E0310F04
:10D0D0003EAF323008F450CE1FAFC888D988EA88F6
:10D0E000FB88C9AADAAAEBAAFCAA812C912C5401CC
:10D0F00089A29AA2ABA2BCA288869986AA86BB8680
:10D100008FE790E0A0E0B0E08C8B9D8BAE8BBF8B67
:10D110001C8690E49A8FACE1AB8FB6E4BC8F1D8E79
:10D120001E8E1F8E18A23FE7432E512C612C712CAE
:10D130001DAA8EAA9FAAA8AEB9AE1EA21FA218A6AB
:10D1400019A6E1E0EDA3198E188E212C312C00E0F8
:10D1500026961FAE2697F5E11F02C00111249C01FF
:10D160002B50364E22963FAF2EAF2297285F3F4F6F
:10D1700024963FAF2EAF24974AA5042E000C550BE2
:10D180005BA74AA780917E02882309F4B0C00F9460
:10D19000D0A269837A838B839C835091EA0958AB30
:10D1A000552309F48BC00E94AFEF60919B0C7091E6
:10D1B0009C0C1F3F39F02296AEADBFAD229714965E
:10D1C0006D917C91072E000C880B990B0F9415BE66
:10D1D0001B01082F26969FAF26972D8D3E8D4F8DD4
:10D1E00058A126969FAD26970F9460C718163CF459
:10D1F0002D8E3E8E0F8F2696BFAD2697B8A32C8519
:10D200003A8D4B8D5C8DB101802F26969FAD269770
:10D210000F940EBE87FF07C02C863A8E0B8F269682
:10D22000EFAD2697EC8FFDA19101402F26965FADC3
:10D2300026976D817E818F8127969FAD2797FF234B
:10D2400009F45AC00F940EBE87FF38C049815A8135
:10D250006B817C814C195D096E097F09DB01CA0174
:10D2600088589341A109B109B7FD28C08C899D89CF
:10D27000AE89BF8984199509A609B709B595A795FF
:10D28000979587951F3F09F079CD80939F0C4EA30A
:10D290005FA368A779A7FD81FD8F2E812E8F3F8127
:10D2A0003F8F27964FAD279748A389819A81AB81FD
:10D2B000BC81888B998BAA8BBB8B1DA220E030E0B0
:10D2C00040EF51E46D817E818F8127969FAD279736
:10D2D0000F9400C59101402F26965FAD26970F94BD
:10D2E0000EBE87FF70CD8BE594E10F94DC4F10925A
:10D2F0007E020E94FCEEA1CE0F9460C71816F4F6D1
:10D3000089819A81AB81BC81288939894A895B8965
:10D31000821B930BA40BB50BAC01BD0148585341C4
:10D320006109710977FDCACF488D598D452B09F4E4
:10D330000DC1CEA0DFA0E8A4F9A4C80ED91EEA1E34
:10D34000FB1E2EA13FA148A559A5281B390B4A0B4E
:10D350005B0BC301B2010F9442C4A70196010F9465
:10D3600074C44C885D886E887F88420E531E641E8C
:10D37000751E54E145165104610471040CF40ACD84
:10D380008CEE48165104610471040CF0FDCC90E859
:10D3900049165104610471040CF40ACD4C8A5D8A6B
:10D3A0006E8A7F8A2EEF30E040E050E02419350984
:10D3B0004609570929013A014C895D896E897F899F
:10D3C00085ED94E10F94A952B301A20180ED94E19F
:10D3D0000F94A9524C855A8D6B8D7C8D89EC94E10C
:10D3E0000F9499524D8D5E8D6F8D78A182EC94E1F2
:10D3F0000F949952A88DB98D13970CF4A7C0C3014F
:10D40000B2010F9415BE20E030E040E850E40F94E4
:10D4100074BE4B015C012C853A8D4B8D5C8D6D8DFE
:10D420007E8D8F8D98A10F94FFC42BED3FE049E4D2
:10D4300050E40F9474BE20E030E040E05FE30F94CE
:10D4400074BE9B01AC01C501B4010F94FAC56C8791
:10D450007D878E879F87C701B6010F9415BE2FE683
:10D4600032E143E85AE30F9474BE6B017C011E3F26
:10D4700059F02AE939E949E15FE3812C912CA12C8B
:10D480006EE3B62E1F3F59F42DEC3CEC4CE45EE30A
:10D490007BEA872E7AEA972EA92C7EE3B72E6C853D
:10D4A0007D858E859F850F9474BE688779878A876E
:10D4B0009B879B01AC010F9400C5A70196010F94B7
:10D4C000FAC569A37AA38BA39CA3288539854A85CD
:10D4D0005B85C701B6010F9474BEA50194010F943A
:10D4E00074BE4B015C014C855D856E857F858CEB40
:10D4F00094E10F949952B701A60186EB94E10F9441
:10D5000099528AE00F94514FBEAD87EA94E1B23050
:10D5100010F088E994E10F94DC4F488559856A85BD
:10D520007B8582E994E10F94995249A15AA16BA19C
:10D530007CA18CE894E10F949952B501A40186E88E
:10D5400094E10F9499528AE00F94514F8C899D89F0
:10D55000AE89BF89840D951DA61DB71DB595A795EC
:10D56000979587951F3F09F028CC80939F0C288DB5
:10D57000398D2F5F3F4F398F288F3D813C874E81FA
:10D580004A8F5F815B8F27968FAD27978C8FC980DD
:10D59000DA80EB80FC8098A99DA390CEE12E012E2D
:10D5A000000CFF08F70183E0EE0FFF1F8A95E1F7FB
:10D5B000EA58FD4F668177816F507109072E000C84
:10D5C000880B990B0F9415BE9B01AC016D817E8178
:10D5D0008F8127969FAD27970F9460C718160CF47C
:10D5E000A6CB8DED94E10F94DC4F0E94FCEE85E11B
:10D5F0008E9DF0018F9DF00D1124EB50F64E8FE7BC
:10D60000808722E330E049CD3F924F925F926F9244
:10D610007F928F929F92AF92BF92CF92DF92EF92C2
:10D62000FF920F931F93CF93DF9380915A0787FD4B
:10D6300038C080915B078370A1F5C091941AD09196
:10D64000951A488159816A817B8180E693E10F9424
:10D6500099524C815D816E817F8186EC9DE60F94AD
:10D6600099524091901A5091911A6091921A70912A
:10D67000931A83EC9DE60F9499528AE0DF91CF9143
:10D680001F910F91FF90EF90DF90CF90BF90AF90E0
:10D690009F908F907F906F905F904F903F900D94F0
:10D6A000514F6090881A7090891A80908A1A9090D1
:10D6B0008B1AA0908C1AB0908D1A00918E1A10912E
:10D6C0008F1AC090901AD090911AE090921AF09010
:10D6D000931A88E50F94D642C82F882309F49AC07C
:10D6E0000F945842362E472E582ED92F20E030E086
:10D6F00046E653EC0F9460C787FD0DC020E030E094
:10D7000046E653E4632D742D852D9D2F0F940EBE98
:10D7100018160CF081C066EE70E08DE493E10F9472
:10D72000BA5266EE70E088E493E10F94BA5285E451
:10D7300093E10F94DC4FC0E089E50F94D642882333
:10D7400061F10F945842362E472E582ED92F20E0E3
:10D7500030E046E653EC0F9460C787FD0DC020E033
:10D7600030E046E653E4632D742D852D9D2F0F94F4
:10D770000EBE18160CF055C066EE70E082E393E121
:10D780000F94BA5266EE70E08DE293E10F94BA52B4
:10D790008AE293E10F94DC4FC0E08AE50F94D64211
:10D7A000882309F443C00F9458426B017C0120E0A8
:10D7B00030E040E151EC0F9460C787FD0AC020E0E3
:10D7C00030E040E151E4C701B6010F940EBE1816D7
:10D7D0006CF567EF7FEF88E193E10F94BA5269E04F
:10D7E00070E083E193E10F94BA5280E193E1DF911D
:10D7F000CF911F910F91FF90EF90DF90CF90BF904E
:10D80000AF909F908F907F906F905F904F903F90E0
:10D810000D94DC4FC1E090CF632C742C852C9D2E91
:10D820008BCFA32CB42C052D1D2FB7CFCC23E1F02B
:10D83000C301D4018093881A9093891AA0938A1AFD
:10D84000B0938B1AC501D80180938C1A90938D1ACE
:10D85000A0938E1AB0938F1AC092901AD092911AF8
:10D86000E092921AF092931ADF91CF911F910F914B
:10D87000FF90EF90DF90CF90BF90AF909F908F90F0
:10D880007F906F905F904F903F900895CF92DF927E
:10D89000EF92FF928AE50F94D642882309F45AC08A
:10D8A0000F94584220E030E040E050EC0F940EBE60
:10D8B000C12CD12CE12C90ECF92E87FD0FC00F94D8
:10D8C000584220E030E040E050E40F9460C7181662
:10D8D0000CF462C00F9458426B017C012091A51496
:10D8E0003091A6144091A7145091A814C701B60115
:10D8F0000F9474BE0F946CC6CB010F9409A380E5FE
:10D900000F94884281114EC0A70196016091901A30
:10D910007091911A8091921A9091931A0F9400C568
:10D920006093901A7093911A8093921A9093931A1D
:10D930000F94FD5B4091901A5091911A6091921A48
:10D940007091931A81E093E10F9499528AE00F94B9
:10D95000514F05C083E50F94D6428111A1CF80912C
:10D960005A0787FD24C080915B07837001F50F94EF
:10D97000FD5B4091901A5091911A6091921A7091AA
:10D98000931A82EF92E10F9499528AE0FF90EF9000
:10D99000DF90CF900D94514FC12CD12CE12C80E41D
:10D9A000F82E9CCF0F9444428111AECFD8CF82E5A0
:10D9B0000F9488428111DBCFFF90EF90DF90CF90E2
:10D9C00008954F925F926F927F928F929F92AF9243
:10D9D000BF92CF92DF92EF92FF92CF93DF93CDB7BA
:10D9E000DEB72C970FB6F894DEBF0FBECDBF4090C8
:10D9F0007B0D50907C0D60907D0D70907E0D209180
:10DA00003D0230913E0240913F0250914002C301DD
:10DA1000B2010F9400C569837A838B839C838090C5
:10DA20007F0D9090800DA090810DB090820D20917F
:10DA30004102309142024091430250914402C5019B
:10DA4000B4010F9400C56D837E838F839887C09047
:10DA5000830DD090840DE090850DF090860D20917F
:10DA60004502309146024091470250914802C70159
:10DA7000B6010F9400C569877A878B879C872091B0
:10DA8000490230914A0240914B0250914C02C3012D
:10DA9000B2010F9400C52B013C0120914D02309141
:10DAA0004E0240914F0250915002C501B4010F94B3
:10DAB00000C54B015C01209151023091520240910E
:10DAC000530250915402C701B6010F9400C56B0177
:10DAD0007C010F94FD5B87E69CE00F94DC4F83E5AF
:10DAE0000F948842882321F00F94444280933B0294
:10DAF00080913B02811151C082E390E10F94DC4F91
:10DB00008FE59CE00F94DC4F49815A816B817C81C9
:10DB10008FED91E30F9499524D815E816F817885ED
:10DB200086EC9DE60F94995249855A856B857C85D4
:10DB300083EC9DE60F9499528DE59CE00F94DC4FA9
:10DB400085E59CE00F94DC4FB301A2018FED91E3DA
:10DB50000F949952B501A40186EC9DE60F94995259
:10DB6000B701A60183EC9DE60F9499528AE02C96AA
:10DB70000FB6F894DEBF0FBECDBFDF91CF91FF90FF
:10DB8000EF90DF90CF90BF90AF909F908F907F905D
:10DB90006F905F904F900D94514F86E390E1AECF20
:10DBA0002F923F924F925F926F927F928F929F92AD
:10DBB000AF92BF92CF92DF92EF92FF920F931F939B
:10DBC000CF93DF93CDB7DEB7CB54D1090FB6F8941E
:10DBD000DEBF0FBECDBF2DB73EB739AF28AF87E050
:10DBE0000F94DF3981110BC061E086E50E94353B5F
:10DBF0008DA3853060F082EC9BE00F94DC4FA8ADE4
:10DC0000B9AD0FB6F894BEBF0FBEADBF3EC33DA1C8
:10DC1000332321F082EA9BE00F94DC4F6AE080E539
:10DC20000E94353B182F8CEF810F8F3218F08EE752
:10DC30009BE0E3CF60E085E40F94FA42882309F487
:10DC400048C081E08FABE090941AF090951AD7010C
:10DC50002D913D914D915C916091870D7091880D52
:10DC60008091890D90918A0D0F9400C5AB01BC0184
:10DC700088E50F94E34269877A878B879C87F70151
:10DC8000248135814681578160918B0D70918C0D77
:10DC900080918D0D90918E0D0F9400C5AB01BC014C
:10DCA00089E50F94E3426D877E878F87988BBE014D
:10DCB000635F7F4FCE0109960F944A43382E81113E
:10DCC0000BC063E68AE69BE00E94974682E59BE0F4
:10DCD00094CF92E09FABB7CF8CE40F948842082F8B
:10DCE000882309F430C10F9430428EA3803118F09C
:10DCF0008BE29BE082CFFEA1F13009F426C160E007
:10DD000083E50F94FA428AAF882321F0011102C003
:10DD100037E03EA38DA1833020F081E19BE00F949A
:10DD2000DC4F9091960C9DAF80E00F94F24A0F94D7
:10DD3000A6141D8A1E8A1F8A188E198E1A8E1B8E93
:10DD40001C8E83EF9FE4A3ECB7E48D8F9E8FAF8F83
:10DD5000B8A383EF9FE4A3ECB7EC89A39AA3ABA38A
:10DD6000BCA3A12FB0E0BCA7ABA7EDB7FEB724E0E2
:10DD7000129FE019F10911240FB6F894FEBF0FBEEF
:10DD8000EDBF8DB79EB701969CAF8BAF01E021E050
:10DD90004DA16FA9CE0109960F94F6539B01AC01DA
:10DDA0000F944DC8811161C20F94D0A26115710505
:10DDB0008105910511F00F9457B9212C1BAA1CAABB
:10DDC0001DAA1EAAAEA1A150BB0B2C96BFAFAEAF31
:10DDD0002C97E22DF0E0F8A7EFA32BA53CA5E217C6
:10DDE000F3070CF073C23196FEA7EDA73F932F9374
:10DDF000FF93EF938DEF9AE09F938F9387E09BE0E3
:10DE00009F938F931F920E947C468DB79EB7099671
:10DE10000FB6F8949EBF0FBE8DBF9EA1992309F443
:10DE200058C10F9408B92AE030E040E050E00F9468
:10DE300074C40F9415BE20E030E040EA50E40F9423
:10DE400060C70FEF1FEF181614F001E010E00F94F9
:10DE500008B928E631E040E050E00F9474C40F9414
:10DE600015BE2B013C010F9408B927E130E040E0DA
:10DE700050E00F9474C46B5F7F4F8F4F9F4F0F9490
:10DE800015BE4B015C01ADA1A430D1F4BC01A401CD
:10DE90008FEE9AE00F949952B301A20187EE9AE0B7
:10DEA0000F94995281EE9AE00F94DC4F01301105E6
:10DEB00019F483E40F94514F8DED9AE00F94DC4FE9
:10DEC000312CC801110FAA0BBB0B2A968CAF9DAF4A
:10DED000AEAFBFAF2A972C96AEADBFAD2C973A161A
:10DEE0001B060CF0F6C02A966CAD7DAD8EAD9FADD5
:10DEF0002A970F9415BE6B017C01BAADBB2341F18B
:10DF0000AC019B010F9400C520E030E040E952E4F1
:10DF10000F9474BE9B01AC01C301B2010F9400C504
:10DF20002B013C0120E030E044EB53E40F9460C748
:10DF30001816FCF420E030E044EB53E4C301B201D6
:10DF40000F94FFC4EDCF1EA2DACE22E02EA3D7CECF
:10DF50000F9408B924E130E040E050E00F9474C41D
:10DF6000675E7F4F8F4F9F4F0F9415BEA70196019D
:10DF7000CFCF20E030E0A901C301B2010F940EBE63
:10DF800087FF0BC020E030E044EB53E4C301B20153
:10DF90000F9400C52B013C01ECCF0091941A109115
:10DFA000951AF80124813581468157816D857E85DA
:10DFB0008F8598890F94FFC422966CAF7DAF8EAF8A
:10DFC0009FAF22972BED3FE049E450E4C301B2013B
:10DFD0000F9474BE20E030E044E353E40F94FAC59C
:10DFE0006B017C010F94F5C56FA778AB89AB9AAB39
:10DFF000D8012D913D914D915C9169857A858B85F4
:10E000009C850F94FFC426966CAF7DAF8EAF9FAFFB
:10E010002697A50194016FA578A989A99AA90F94BB
:10E0200074BE9B01AC0126966CAD7DAD8EAD9FADEF
:10E0300026970F9400C569837A838B839C83C701DD
:10E04000B6010F94F0C7A50194010F9474BE2296F7
:10E050002CAD3DAD4EAD5FAD22970F9400C56D83E5
:10E060007E838F83988740EF50E070E060E0CE01C0
:10E0700001960E94C7EF40EF50E070E060E0CE01F3
:10E0800005960E94C7EFBDA1B43099F449815A8129
:10E090006B817C8181ED9AE00F9499524D815E8174
:10E0A0006F81788586EC9DE60F9499528AE00F94F3
:10E0B000514F198A1A8A1B8A1C8AAE014F5E5F4F24
:10E0C000BE016B5F7F4FCE0101960F948316339490
:10E0D00002CF01E021E040E06FA9CE0109960F9444
:10E0E000F6536B017C01312CAC019B010F944DC8A0
:10E0F000811102C033243394A7019601C701B601F0
:10E100000F944DC88111E2C0EFA1F8A5EE0FFF1FDB
:10E11000EE0FFF1F2BAD3CADE20FF31FC082D1828B
:10E12000E282F3822D8D3E8D4F8D58A1C701B6013D
:10E130000F940EBE87FF04C0CD8EDE8EEF8EF8A248
:10E1400029A13AA14BA15CA1C701B6010F9460C7F8
:10E15000181624F4C9A2DAA2EBA2FCA2A701960128
:10E160006BA97CA98DA99EA90F9400C56BAB7CAB54
:10E170008DAB9EABADA5BEA5BD01BB0F880B990BAA
:10E180000F9415BE2B013C01AC019B016BA97CA92E
:10E190008DA99EA90F94FAC56FA378A789A79AA7FE
:10E1A0006D8B7E8B8F8B988FEBADFCADF8ABEFA7B3
:10E1B00010E0812C912C5401AFA5B8A96D917D91EF
:10E1C0008D919D91B8ABAFA72FA138A549A55AA5B0
:10E1D0000F94FFC49B01AC010F9474BE9B01AC0172
:10E1E000C501B4010F9400C54B015C011F5F2116EE
:10E1F00018F7A30192010F94FAC50F94FEC7698F17
:10E200007A8F8B8F9C8FBDA1B23068F18DA59EA5B2
:10E210000F9492836BA57CA58CEC9AE00F94BA5274
:10E2200086EC9AE00F94DC4F43E0C701B6010F94EF
:10E23000442E80E20F94514F81E0EDA1E3300CF4C5
:10E2400080E0E12C8E010F5D1F4F9E01235E3F4F4A
:10E25000AE01475E5F4FBE016B5E7F4F0E94D842AA
:10E260008AE00F94514F2394B4CD0F941E430F9422
:10E270008D148DAD0F94F24A0F94E21B88AD99ADC9
:10E280000FB6F8949EBF0FBE8DBFE8ADF9AD0FB6C7
:10E29000F894FEBF0FBEEDBFC55BDF4F0FB6F8941D
:10E2A000DEBF0FBECDBFDF91CF911F910F91FF90C9
:10E2B000EF90DF90CF90BF90AF909F908F907F9026
:10E2C0006F905F904F903F902F9008950F941E4352
:10E2D000332069F28BEB9AE00F94DC4F81E0FDA1D3
:10E2E0001F160CF080E0EE24E3948E010F5D1F4FAB
:10E2F0009E01235E3F4FAE01475E5F4FBE016B5EE6
:10E300007F4F0E94D842698D7A8D8B8D9C8D0052F3
:10E31000110926E042E00F949EB89F938F938AEAFA
:10E320009AE09F938F9384EB9AE09F938F931F9231
:10E330000E947C462DB73EB7295F3F4F0FB6F89439
:10E340003EBF0FBE2DBF93CFAF92BF92CF92DF9251
:10E35000EF92FF920F931F93CF93DF93CDB7DEB76A
:10E36000E6970FB6F894DEBF0FBECDBF00917008E0
:10E3700010917108F80101900020E9F731976F01C1
:10E38000C01AD10AF801CF01801B910B8C159D0595
:10E390003CF481918F32B9F7DF0111971C92F3CFD2
:10E3A0008BE1ECE3FBE1DE015C9601900D928A9536
:10E3B000E1F7F12CE12CEC14FD040CF05DC0F80148
:10E3C000EE0DFF1D8081811103C08FEFE81AF80A5E
:10E3D0005801AE0CBF1CF5018081882309F44CC0A4
:10E3E000FFEFEF1AFF0AF801EE0DFF1D7F01E01AA3
:10E3F000F10A81918111FACFCE014C960E9436EB41
:10E400008BE1FE017C96DE01119601900D928A95BA
:10E41000E1F7B501CE0101960E9450E3CE010196CD
:10E420000F947B408FE20F94514F809147178111D9
:10E430003BC08DE197E00F94C52880911B1B84FFA2
:10E440001BC019821C8221E0A501BE01645E7F4FC2
:10E45000CE0101960E9409ED811129C08AE00F9436
:10E46000514F0F94FD5BB5018FE693E10F94E85394
:10E47000CE0101960F947B408AE00F94514FCE015C
:10E480004C960F947B40E6960FB6F894DEBF0FBE15
:10E49000CDBFDF91CF911F910F91FF90EF90DF9053
:10E4A000CF90BF90AF90089587E497E1C4CFCE019D
:10E4B0004C960E94A5EA8BE1FE013196DE015C9646
:10E4C00001900D928A95E1F7CE0101960F947B4061
:10E4D00072CFBF92CF92DF92EF92FF920F931F9372
:10E4E000CF93DF9300D000D0CDB7DEB76FEF7FEFD3
:10E4F00089E40F940F43B82E6FEF7FEF8AE40F94F7
:10E500000F43182F83E40F948842F82E8EE40F9463
:10E510008842C82E8AE50F948842E82ED12C8111BA
:10E5200004C081E50F948842D82E012F2B2DFF20A7
:10E5300049F030E020E040E067E87DE081E00F94C2
:10E54000764A032F4F2D50E080E0B7FC05C0812FA5
:10E550008095881F8827881F840F952F911D01970C
:10E5600031F4E11019C0D11017C0C11015C00F94BB
:10E57000F2538AE89AE026960FB6F894DEBF0FBEF3
:10E58000CDBFDF91CF911F910F91FF90EF90DF9062
:10E59000CF90BF900D94DC4F263010F4063028F059
:10E5A0000F94F25381E79AE0E6CFE22E220FFF08A4
:10E5B000002E000C110B60E070E080EC9FE7C110B2
:10E5C0001DC00F9458429B01AC0160E070E0CB018C
:10E5D000DD2091F086E08E9DF0018F9DF00D1124DD
:10E5E000E00FF11FEE0FFF1FEE0FFF1FE55CF64F70
:10E5F00060817181828193810F9400C526E02E9DF8
:10E60000F0012F9DF00D1124E00FF11FEE0FFF1F01
:10E61000EE0FFF1FE55CF64F608371838283938367
:10E6200026960FB6F894DEBF0FBECDBFDF91CF9117
:10E630001F910F91FF90EF90DF90CF90BF900895C2
:10E640004F925F926F927F928F929F92AF92BF9202
:10E65000CF92DF92EF92FF92CF93DF9300D000D062
:10E660001F921F92CDB7DEB783E50F948842F82E34
:10E67000D090960C882319F00F944442D82E4090E5
:10E68000870D5090880D6090890D70908A0D809054
:10E690008B0D90908C0DA0908D0DB0908E0D809173
:10E6A0008F0D9091900DA091910DB091920D8D8351
:10E6B0009E83AF83B887FF2029F0D11003C080E08C
:10E6C0000F94F24A8CE40F948842882309F44BC0DB
:10E6D00080E00F94F24A80912E0790912F07C0900E
:10E6E000D409892B19F00F945442C82E0E9473F25A
:10E6F0007C01892BC9F481E59AE00F94DC4F2896C0
:10E700000FB6F894DEBF0FBECDBFDF91CF91FF9063
:10E71000EF90DF90CF90BF90AF909F908F907F90C1
:10E720006F905F904F900895C7FC07C08C2D0C2C04
:10E73000000C990B8E159F057CF089E39AE00F94ED
:10E74000DC4FB701615071098EE29AE00F94BA5222
:10E750008AE00F94514FD3CF70E060E08C2D0E947F
:10E760007FF2C092D4098091590783FD04C0809143
:10E770005A0785FF1FC060E084E50E94353B90E0AA
:10E780000F94606E85E29AE00F94DC4F0F94314C49
:10E79000811104C082E29AE00F94DC4F6091D409A9
:10E7A000062E000C770B8DE09AE00F94BA528AE0A7
:10E7B0000F94514F86E50F948842F82E0F94314CF8
:10E7C000882341F183E40F948842882379F00F94E1
:10E7D000584269837A838B839C8380E00F94F24A4A
:10E7E000BE016F5F7F4F81E00F94C4528AE50F94A2
:10E7F0008842882359F00F94584269837A838B8327
:10E800009C8360E0CE0101960F94514B8D2D0F94A7
:10E81000F24A0AC0D11002C0FF2041F30F94FD5B01
:10E820008EEF99E00F94DC4FDD2051F08091960C33
:10E83000811106C00F94F2538FED99E00F94DC4FD5
:10E840000F94FD5B81ED99E00F94DC4F8091960C65
:10E85000811159C082E390E10F94DC4F8AE00F945C
:10E86000514F0F94FD5B84EC99E00F94DC4FC09006
:10E87000920CD090930CE090940CF090950C20E0CA
:10E8800030E0A901C701B6010F9460C71816F4F56E
:10E8900042E0C701B6010F94442E8DE00F94514F12
:10E8A0008AE00F94514FA30192016091870D7091FE
:10E8B000880D8091890D90918A0D0F940EBE811163
:10E8C0001FC0A501940160918B0D70918C0D8091FA
:10E8D0008D0D90918E0D0F940EBE811111C020915F
:10E8E0008F0D3091900D4091910D5091920D6D8151
:10E8F0007E818F8198850F940EBE882309F4FFCE08
:10E900000F94E21BFCCE86E390E1A6CF8FEB99E05B
:10E910000F94DC4FC8CF2F923F924F925F926F922D
:10E920007F928F929F92AF92BF92CF92DF92EF929F
:10E93000FF920F931F93CF93DF93CDB7DEB7E59789
:10E940000FB6F894DEBF0FBECDBF8DAB2091850C06
:10E950002CAB81E08093850C80916F088D3409F495
:10E9600082C5843511F40C94738A873409F091C1FF
:10E9700080916D0890916E088B31910509F4DCC18E
:10E9800008F079C18430910508F030C120912A0C3B
:10E990008230910508F48EC1213009F091C111E057
:10E9A000029709F010E00E94B43F19821A821B827C
:10E9B0001C821D821E821F82188682E50F94D64219
:10E9C000882309F48FC10F9458426B017C0120E029
:10E9D00030E0A9010F940EBE882309F4EAC04090EC
:10E9E000870D5090880D6090890D70908A0D8091F0
:10E9F0008B0D90918C0DA0918D0DB0918E0D8CA7EB
:10EA00009DA7AEA7BFA780906C0C90906D0CA090B6
:10EA10006E0CB0906F0C8091700C9091710CA09165
:10EA2000720CB091730C88AB99ABAAABBBABA501D0
:10EA30009401C301B2010F940EBE81110DC028A92B
:10EA400039A94AA95BA96CA57DA58EA59FA50F94A0
:10EA50000EBE882309F4ADC0A3019201C501B40123
:10EA60000F94FFC420E030E040E05FE30F9474BEF9
:10EA700068A779A78AA79BA72CA53DA54EA55FA54A
:10EA800068A979A98AA99BA90F94FFC420E030E066
:10EA900040E05FE30F9474BE2B013C0120E030E0C6
:10EAA000A901C701B6010F940EBE881F8827881FD1
:10EAB000181709F40EC180E090E0A0E8BFEB8CA726
:10EAC0009DA7AEA7BFA728A539A54AA55BA5CA01E2
:10EAD000B9010F9474BE4B015C01A3019201C30103
:10EAE000B2010F9474BE9B01AC01C501B4010F9437
:10EAF00000C50F94FEC74B015C01AC019B01C7012F
:10EB0000B6010F94FFC468AB79AB8AAB9BABA50190
:10EB10009401C701B6010F9400C59B01AC0168A91F
:10EB200079A98AA99BA90F9474BE6B017C0120E08E
:10EB300030E0A9010F9460C787FDD0C0C701B601BE
:10EB40000F94FEC76B017C01C301B2019058A5016F
:10EB500094010F94FAC52CA53DA54EA55FA50F9471
:10EB600074BEA70196010F9474BE28A539A54AA5C5
:10EB70005BA50F9400C569837A838B839C83A50171
:10EB8000940168A579A58AA59BA50F94FAC52CA523
:10EB90003DA54EA55FA50F9474BEA70196010F94E5
:10EBA00074BEA30192010F9400C56D837E838F8391
:10EBB000988720E030E0A90169817A818B819C816E
:10EBC0000F940EBE8111A2C020E030E0A9016D813A
:10EBD0007E818F8198850F940EBE811197C00F940E
:10EBE000F25389E29DE00F94DC4F6AC085319105B4
:10EBF00009F466C08A31910509F49BC0049709F0B5
:10EC000048C080E50F94D642C12CD12C76018823D0
:10EC100021F00E94163C6B017C0183E50F94D642E3
:10EC2000882361F00F94584220E030E04AE754E432
:10EC30000F9474BE0F9473C66B017C010E9449F758
:10EC400080918A17811105C060E08FE39DE00E94EA
:10EC500097460F94D0A2C60ED71EE81EF91E0F9439
:10EC6000D0A26C197D098E099F0997FF29C080E009
:10EC70000F942D5EF4CF8A32910509F498C260F4A6
:10EC80008D31910509F417C208F46FC04E9709F44D
:10EC900015C20F940F9914C08B35910509F43BC32D
:10ECA0008C35910509F43BC38A35910591F7109293
:10ECB000910C06C0213021F40E94B43F0F94D50B73
:10ECC0003DA9311102C00F94D8AC8CA98093850C5A
:10ECD0006AC580E090E0A0E8BFE3F1CEC12CD12C62
:10ECE000760132CF89E40F94D642882331F00F9415
:10ECF000584269837A838B839C838AE40F94D6423B
:10ED0000882309F456CF0F9458424FCF412FBE01AC
:10ED10006F5F7F4F8CE69CE00F944FA30F94D0A2BF
:10ED200060937C0C70937D0C80937E0C90937F0C91
:10ED3000C7CF0E948C48C4CF87E00F94DF39811180
:10ED4000BFCF8CE0E1EAF2E0DE01119601900D9276
:10ED50008A95E1F770E060E080E50E94413BBE01EA
:10ED60006F5F7F4F0F945826ABCF87E00F94070B50
:10ED7000811106C060E08FE40F94FA428111A0CFA8
:10ED80000E9449F710923C026091960C8CE40F941B
:10ED9000FA42E82E80E00F94F24A0F94D0A26093DA
:10EDA0007C0C70937D0C80937E0C90937F0C0F9461
:10EDB000A61481E08093E20B0F94081D8AE50F945E
:10EDC0008842F82E882369F081E00F94070B182FF2
:10EDD00082E00F94070B11110C94D18A11E081117C
:10EDE00001C010E088E50F948842082F81110C942F
:10EDF000888A11110CC089E50F948842811342C1A1
:10EE0000012FF11204C001E011E0FF24F39482E528
:10EE10000F94D642882309F438C10F9458426CA34A
:10EE20007DA38EA39FA320E030E0A9010F940EBE26
:10EE3000882381F0011105C0111103C0FF2009F4DE
:10EE400010C160E0CE0184960F9433160F94DA4E11
:10EE50000F94894E002309F47FC0112309F479C06F
:10EE60001092870D1092880D1092890D10928A0DC4
:10EE700010928B0D10928C0D10928D0D10928E0DA4
:10EE80000F947B1783E49DE20E9409664B015C01AD
:10EE900087E49DE20E9409662B013C01AC019B01C5
:10EEA000C501B4010F9460C718160CF0F3C0A5019A
:10EEB0009401C301B2010F94FAC59B01AC010F94F8
:10EEC00074BE20E030E040E85FE30F9400C50F948B
:10EED000FEC720E030E048E452E40F9474BE68A31B
:10EEE00079A38AA39BA320E030E040EC5FE3C30159
:10EEF000B2010F9474BE905869837A838B839C838C
:10EF000020E030E040EC5FE3C501B4010F9474BE33
:10EF100090586C8F7D8F8E8F9F8FAE01405E5F4FBC
:10EF2000BE016F5F7F4FCE014C960F9483160F94F6
:10EF3000391F1092870D1092880D1092890D109232
:10EF40008A0D10928B0D10928C0D10928D0D1092D7
:10EF50008E0D80E00F942820112319F081E00F948A
:10EF60002820FF2009F47DC083E00F94DF39811150
:10EF700078C00F947B172091BD0C3091BE0C40914E
:10EF8000BF0C5091C00C60E070E086EE92E40F94EC
:10EF9000FFC42B013C012091C10C3091C20C409167
:10EFA000C30C5091C40C60E070E086EE92E40F94C4
:10EFB000FFC44B015C0180918F0D9091900DA09149
:10EFC000910DB091920D8093740C9093750CA09359
:10EFD000760CB093770C0091941A1091951AD80181
:10EFE0002D913D914D915C91C301B2010F94FFC4ED
:10EFF00060936C0C70936D0C80936E0C90936F0CFF
:10F00000F8012481358146815781C501B4010F94EF
:10F01000FFC46093700C7093710C8093720C90938A
:10F02000730C8CE69CE00F9409498823C1F11C8E77
:10F030001D8E1E8E1F8E88E0ECE6FCE0DE01119630
:10F0400001900D928A95E1F7AE01445E5F4FBE01DB
:10F050006B5F7F4FCE0101960F94831682E00F9471
:10F0600028200F947B178091E10B8093E20B8E2D6B
:10F070000F94F24A0F948D1483E080937F020F94D3
:10F08000E21B1ECE012F182FC2CE60E070E080E898
:10F0900090E4C5CEA3019201C501B4010CCF60E09C
:10F0A0008AE59DE00E9497460F94FD5B88E49DE011
:10F0B0000F94DC4FD6CF0F94AD7702CE0091941A07
:10F0C0001091951AD8012D913D914D915C916091CF
:10F0D000870D7091880D8091890D90918A0D0F9404
:10F0E00000C5AB01BC0188E50F94E34269837A83D4
:10F0F0008B839C83F80124813581468157816091FF
:10F100008B0D70918C0D80918D0D90918E0D0F94C3
:10F1100000C5AB01BC0189E50F94E3426D837E839A
:10F120008F839887BE016B5F7F4FCE0101960F944E
:10F130004A43882309F4C4CD80E00F94F24A0F9427
:10F14000A61461E085E40F94FA42182F01E021E053
:10F1500041E0682FCE0101960F94F6536B017C01BC
:10F16000AC019B010F944DC8811119C049815A818E
:10F170006B817C8185E79DE00F9499524D815E8182
:10F180006F81788580E79DE00F949952B701A601C1
:10F190008BE69DE00F9499528AE00F94514F0F94A3
:10F1A0008D1411110F9430430F94E21B89CD80917F
:10F1B0002A0C813009F084CD89E40F94D642182FAF
:10F1C000E12C882319F00F945442E82E8AE40F941E
:10F1D000D642082F882379F00F945442F82E112339
:10F1E00009F490C0F5E0FE1508F089C08DE79DE0B8
:10F1F0000F94DC4F65CDF12C1111F4CF80E1E7E8DD
:10F20000FDE0ACE6BCE001900D928A95E1F7112398
:10F2100059F08E2D0F94DD4460936C0C70936D0C3F
:10F2200080936E0C90936F0C002359F08F2D0F94E8
:10F2300047446093700C7093710C8093720C9093A0
:10F24000730C60E080E50F94FA428823C1F111232A
:10F25000D1F0E091941AF091951A20813181428188
:10F26000538160916C0C70916D0C80916E0C90913B
:10F270006F0C0F94FFC460936C0C70936D0C8093B3
:10F280006E0C90936F0C0023D1F0E091941AF091E2
:10F29000951A24813581468157816091700C709157
:10F2A000710C8091720C9091730C0F94FFC4609359
:10F2B000700C7093710C8093720C9093730C40E0FF
:10F2C00050E0BA0186E40F94E3426B017C0120E038
:10F2D00030E0A9010F9460C71816CCF420E030E0AC
:10F2E00040E752E4C701B6010F94FAC569837A83F7
:10F2F0008B839C83CE0101960F94C514E1CC00232F
:10F3000009F47CCF25E02F1508F078CF6FCF60E0AF
:10F3100070E0CB01EBCF8FE08093910CD1CC80914A
:10F320006C08882381F1893009F0CACC0DEBA02E3E
:10F3300002E0B02E87E8C82E8DE0D82EE12C00E048
:10F3400010E0D5018D915D010F94D642F82E8823EF
:10F3500061F0133011F4082FFE2C0F945842F6017F
:10F360006083718382839383EF2C1F5FF4E0CF0E61
:10F37000D11C143031F7EE2009F457C00F947B17DD
:10F380000F94E21B9DCC1DEBC12E12E0D12EF12C6F
:10F39000E12C00E010E0D6018D916D010F94D64272
:10F3A000382E8823D9F10F9458424B015C01133059
:10F3B00059F0F701E558F24F2081318142815381A4
:10F3C0000F94FFC44B015C01F701E957F24F208114
:10F3D000318142815381C501B4010F94FFC42B01D7
:10F3E0003C012DEB37E346E855EB0F9460C787FDF2
:10F3F0000AC02DEB37E346E855E3C301B2010F9491
:10F400000EBE18165CF41330C1F48092930D9092E6
:10F41000940DA092950DB092960D032D1F5FB4E050
:10F42000EB0EF11C143009F0B6CF002309F4A8CF7D
:10F4300083E99DE00F94EF08A3CFF701EF54F34F5A
:10F440005F01A301920160817181828193810F9498
:10F4500000C5D5016D937D938D939C931397812F58
:10F460000F94E70ADBCF80916D0890916E088D377D
:10F47000910509F463C608F05FC28E34910509F462
:10F4800002C708F022C18B31910509F45BC608F070
:10F49000B2C08531910509F4D1C508F07BC0813136
:10F4A000910509F48AC508F045C0029708F0F1CB30
:10F4B00080E50F94D642C12CD12C7601882321F00F
:10F4C0000E94163C6B017C0183E50F94D642882391
:10F4D00061F00F94584220E030E04AE754E40F9482
:10F4E00074BE0F9473C66B017C010E9449F7809132
:10F4F000700890917108009709F459C50F94B5866A
:10F5000080916D0890916E086EE97DE0892B11F471
:10F5100066E97DE030E020E049E65DE682E00F94B8
:10F52000315040E0C701B6010F944D7E80E00E944B
:10F530003347C6CB8231910511F40C9495834497DF
:10F5400009F0A7CB80911B1B83FF70C581ED9DE067
:10F550000F94DC4F80911B1B83FF17C08CE39BE152
:10F560000E9436EB8BE1ECE3FBE1DE0111960190AA
:10F570000D928A95E1F770E060E0CE0101960F945C
:10F58000692CCE0101960F947B4082EC9DE00F9494
:10F59000DC4F96CB8831910509F465C5B0F486310E
:10F5A000910509F44FC5479709F073CB8091700816
:10F5B00090917108FC012191222309F44DC520325C
:10F5C000D1F7DF0111971C92F6CF8931910509F42B
:10F5D000B5C54A9709F05DCB80911B1B83FF70CBAB
:10F5E00083E50F94D642882309F46ACB0F94204216
:10F5F0000E941E6465CB8132910509F415C608F09E
:10F600003EC08E31910509F4FFC568F48C31910537
:10F6100009F4F2C54D9709F03CCB80911B1B8E7FFE
:10F6200080931B1B4DCB8F31910509F401C6809748
:10F6300009F02FCB80911B1B82FD0E9449F780911E
:10F640001B1B83FF3DCB60E080E50F94FA42182F2F
:10F65000682F80917008909171080F94502D83E568
:10F660000F94D642882321F00F9420420E941E64FA
:10F670000E94BDE2111124CB0F94F74C21CB8B34A7
:10F68000910509F4F8C5B0F48033910509F4EFC58C
:10F690008934910509F0FDCA80E50F9488428823DA
:10F6A00009F40ECB0F943042853608F084E680933F
:10F6B000030906CB8C34910509F4E1C58D3491051D
:10F6C00009F0E7CA0F940A4DFBCA8D36910509F47B
:10F6D0009CC608F08AC08C35910511F40C9499836E
:10F6E00008F042C08335910511F40C948D8380F4A9
:10F6F0008135910511F40C9470838235910509F0E0
:10F70000C8CA8091910C8F7D80618093910CD8CA7A
:10F710008435910511F40C9495838535910509F094
:10F72000B8CA83E50F948842882309F4C9CA0F94A4
:10F73000D0A260937C0C70937D0C80937E0C909390
:10F740007F0C0F94584220E030E04AE754E40F94D5
:10F7500074BE0F9473C660933A0770933B0780930F
:10F760003C0790933D07ACCA8A36910509F4ABC6B5
:10F7700098F58836910509F419C68936910509F07E
:10F7800088CA0E94883B182F87FD0AC08FE99EE037
:10F790000F94DC4F812F0F94E82E8AE00F94514F85
:10F7A0002CA92093850CE5960FB6F894DEBF0FBE0A
:10F7B000CDBFDF91CF911F910F91FF90EF90DF9020
:10F7C000CF90BF90AF909F908F907F906F905F9001
:10F7D0004F903F902F9008958B36910509F4AEC657
:10F7E0008C36910509F46CCA54CA8337910511F41B
:10F7F0000C943A8408F05DC08037910509F460CA22
:10F8000008F048C08E36910509F4A7C68F369105D9
:10F8100009F03FCA83E50F948842882331F060E005
:10F8200083E50E94353B809388140F94FD5B80EB49
:10F830009EE00F94DC4F80918814882309F4A0C6C1
:10F8400010E000E020E08091881490E0B0E0A0E0BB
:10F85000002E04C0B695A795979587950A94D2F780
:10F8600080FF12C0FF24F394F20E222319F08CE2E1
:10F870000F94514FF801EE0FFF1FEA55F14F85919C
:10F8800094910F94DC4F2F2D0F5F1F4F0530110502
:10F89000D1F67FC48137910509F475C68237910589
:10F8A00009F0F7C90F9437988BEA9AE10E94C9F1E1
:10F8B00007CA8737910511F40C94698470F5853770
:10F8C000910509F4DBC78637910509F0E2C900917B
:10F8D00070081091710894E0F12C40E0915009F407
:10F8E000E7C7F8018081282F2B7F213409F0D9C781
:10F8F0002181213309F0DCC7813409F4E7C785345D
:10F9000009F441E098012E5F3F4F89012F5F3F4F7F
:10F91000F80180818032C9F3E1CF8837910509F47D
:10F92000DCC78937910509F0B4C91092E20B109237
:10F93000E10B0F94081DC4C98239E1E09E0711F460
:10F940000C94458808F040C18C3D910511F40C944D
:10F95000CB8508F0CAC0893C910511F40C94E2846F
:10F9600008F075C08B39910509F493C6B8F48C384A
:10F97000910509F42AC68139910509F08AC970E018
:10F9800060E083E50F940F43823008F4AFC70F9413
:10F99000F25380EF9EE00F94DC4F92C98E3B9105AD
:10F9A00009F439C6883C910509F073C90E94883B67
:10F9B000182F87FD85C90091B00C84E40F94D642BE
:10F9C000B82E8823D9F10F9458426B017C0120E0B6
:10F9D00030E0A9010F940EBE882311F40C94E0844A
:10F9E00024E01202F0011124E455F34FC082D182C9
:10F9F000E282F38220E030E0A901C701B6010F9452
:10FA000060C71816D4F420E030E040E05FE3C7019F
:10FA1000B6010F9474BE9B01AC010F9474BE2BED24
:10FA20003FE049E450E40F9474BE60930D0270937C
:10FA30000E0280930F02909310020B2D602F83E52E
:10FA40000F94FA428093B00C0E94E4DD39C98D3CDA
:10FA5000910511F40C947785E0F58B3C910509F440
:10FA6000DBC78C3C910509F014C98091590787FFC9
:10FA700002C00C942F8580915A078E7011F00C945F
:10FA80002F854091BD145091BE146091BF147091A8
:10FA9000C01485E19FE00F9499524091C114509198
:10FAA000C2146091C3147091C41482E19FE00F945A
:10FAB00099524091C5145091C6146091C714709129
:10FAC000C8148EE692E30F9499528AE00F94514F36
:10FAD000F7C88E3C910511F40C947B85833D91050C
:10FAE00009F0D7C80E94E16CEBC88D3221E0920783
:10FAF00011F40C94058708F044C08831A1E09A07FE
:10FB000011F40C946586F0F48D3D910511F40C947C
:10FB10000E868A3F910509F0BCC883E40F948842A1
:10FB2000882321F00F9454420E944A51609155025B
:10FB30007091560283E89FE00F94BA528AE00F94C6
:10FB4000514FBEC88232E1E09E0711F40C94018748
:10FB50008C32914009F09DC864E071E083E50E9419
:10FB6000413B8C0168EE73E080E50E94413B89389F
:10FB700023E1920710F088E893E1B8010E94D7B022
:10FB80009FC8803321E0920711F40C94878768F4B2
:10FB90008E32A1E09A0711F40C94FB878F329140CA
:10FBA00009F077C80E940F668BC88039E1E09E0794
:10FBB00011F40C9441888139914009F06AC80F947E
:10FBC00027430F94E21B7CC88C3022E0920711F48B
:10FBD0000C94EE8808F002C1863EA1E09A0711F469
:10FBE0000C946A8808F0C6C0843AE1E09E0711F4DC
:10FBF0000C944D88B8F48A3921E0920709F460C862
:10FC00008D39914009F045C883E50F9488428823D7
:10FC100011F40C94598A0F9444428093D3090F94A1
:10FC20005B404EC8853AA1E09A0711F40C945188C4
:10FC30008C3A914009F02DC887E00F94DF3981118B
:10FC40003FC877E3C72E7DE2D72E87E89DE099A7CE
:10FC500088A7DE0111961D017D0110E000E0C601BC
:10FC60000E940966E8A5F9A581909190A190B190B4
:10FC7000F9A7E8A7A50194010F94FFC42B013C014B
:10FC8000D7014D925D926D927C92139720E030E007
:10FC900040EA51EC0F9460C787FD0AC020E030E0D5
:10FCA00040EA51E4C301B2010F940EBE18167CF471
:10FCB000F801E55AF24DE4911E164CF4B7FAB094EF
:10FCC000B7F8B094F70180829182A282B382D70103
:10FCD0008D909D90AD90BD907D0120E030E040EA98
:10FCE00051ECC501B4010F9460C787FF02C00C94AA
:10FCF000558820E030E040EA51E4C501B4010F949A
:10FD00000EBE181614F40C9455880F5F1F4FB4E004
:10FD1000CB0ED11C0330110509F0A1CF6DEBE62EFF
:10FD20006CE0F62E10E0F10181919191A191B191D9
:10FD30001F01F70181939193A193B1937F01812FCB
:10FD40000F94E70A1F5F133071F70F94E21B60E016
:10FD500081EC9FE00E94974663E972E084E690E0C0
:10FD60000E94D7B06AEB72E084E690E00E94D7B0C0
:10FD70000C946076863FE1E09E0711F40C94E088D5
:10FD800078F4843F21E0920711F40C94DC88853FDD
:10FD9000914011F00C9449760F94C9390C94607617
:10FDA000873FA1E09A0711F40C94E488883F9140C2
:10FDB00011F00C94497681E08093D5090F94BD39F8
:10FDC0001092D509882311F40C9460760F94FD5B92
:10FDD0008DEF9FE00F94DC4F0C9460768C36E3E05F
:10FDE0009E0711F40C94607608F091C08D3B22E0E0
:10FDF000920711F40C94198908F07AC08835A2E0B2
:10FE00009A0711F40C94FF888B35924011F00C94F2
:10FE100049760E94883B082F87FF02C00C946076C9
:10FE200085E50F948842882369F10F9458424B016D
:10FE30005C01E02E002E000CFF0820E030E0A9015C
:10FE40000F9460C787FF04C0B7FAB094B7F8B094B6
:10FE500020E030E84BE354E4C501B4010F9460C7DF
:10FE6000970153E0220F331F5A95E1F72553364F80
:10FE7000181614F40C940389D9018D929D92AD92B9
:10FE8000BC9213978CE40F948842882311F40C944D
:10FE900060760F9458426B017C01002E000C110B10
:10FEA00020E030E0A9010F9460C787FF04C0F7FA93
:10FEB000F094F7F8F09420E030E84BE354E4C70105
:10FEC000B6010F9460C7980143E0220F331F4A9593
:10FED000E1F72553364F181614F40C940E89D90106
:10FEE0001496CD92DD92ED92FC9217970C94607669
:10FEF0008E3BE2E09E0711F40C941D8983359340FC
:10FF000011F00C9449760E94046B0C946076873E45
:10FF100023E0920711F40C94498AC8F48438A3E0D2
:10FF20009A0711F40C94DE89803A934011F00C94F6
:10FF30004976209170083091710890911B1B926056
:10FF400090931B1BC9010E9469EE0C946076883E59
:10FF5000E3E09E0711F40C946F8A893E934011F000
:10FF60000C9449760F9492AE81110C9460760F94A4
:10FF700053400F944AAE0F949D226D337105810555
:10FF8000910520F08AE690E10E94048B86E690E1DC
:10FF90000E94048B84EE8093030982E590E10F9424
:10FFA000DC4F8EE490E10E94048B0C94607660E05C
:10FFB00086EA9DE00E949746A3CA8091580784FD77
:10FFC00017C080915A0787FD13C080915B0783702B
:10FFD00079F460E089EB9DE00E9497465F988A98EB
:10FFE0008091080181708093060112980C946076CC
:10FFF00088E50F94884281115F9889E50F948842C3
:020000021000EC
:1000000081118A988AE50F948842882329F080918B
:10001000080181708093060185E40F94884288234B
:1000200011F40C94607612980C9460760F94FD5B3A
:1000300082EE9DE00F94DC4F0C9460760E94D0EA33
:100040000C94607680911B1B82FF02C00C9460763A
:100050000E94BFEA0C94607660E00F94502D1092DD
:1000600003090C94607683E50F94D642882321F02F
:100070000F9420420E941E6484E50F94D642882388
:10008000A9F00F9420426B017C010F944423C0928D
:100090003209D0923309E0923409F0923509CD2823
:1000A000CE28CF2819F081E0809336098091EC09A1
:1000B0008823F9F080E090E0A0EAB1E489839A8394
:1000C000AB83BC831C8E1D8E1E8E1F8E18A219A2A0
:1000D0001AA21BA210E000E020E0AE014F5F5F4FCC
:1000E000BE01645E7F4FCE0180960F9466650C94CE
:1000F00060760F94D34C882381F00E94BDE20F9468
:10010000F74C87E09DE00E945EEA1092BC151092C9
:10011000BD151092BE151092BF1561E085E598E1FE
:100120000F94EA4F40E158E16CEE7DE085E00F94DA
:10013000269A80E00E9433470C9460760E94F84132
:100140000C94607683E40F948842882361F182E006
:100150009EE00F94DC4F8091831C8823F9F0BE0150
:100160006F5F7F4F80E89CE10E94F1E9CE0101962C
:100170000F94C528CE0101960F9464AE8091471765
:10018000882339F080E20F94514F87E497E10F9470
:10019000C5288AE00F94514F0C94607688EF9DE05B
:1001A0000F94DC4FF6CF83E50F94D642882301F1FC
:1001B0000F943042182F8C3308F08CE3809334076F
:1001C0000F94D0A26B017C01212F30E0A8EEB3E0A8
:1001D0000F94A6C4C60ED71EE81EF91EC0923007A3
:1001E000D0923107E0923207F09233070C94607698
:1001F0000F94EBAE0C94607680917008909171082A
:100200000E9469EE0C94607680911B1B83FD02C0F6
:100210000C9460760F94F598809170089091710815
:100220000E9401EE0C9460760E94A4710C9460769A
:100230000F949D226C8F7D8F8E8F9F8FBE016F5F7D
:100240007F4FCE014C960E943F63CE0101960F94E2
:10025000B5860F94FD5BBE016F5F7F4F81E19EE02D
:100260000F94E8538AE00F94514F0C9460760E94EB
:10027000D06D0C9460760F94F74C0C9460760F94CC
:1002800097230C94607670E060E083E50F940F4351
:100290008E34910539F40E9467F680E00E9433475E
:1002A0000C9460768CE79EE00F94DC4F6091D10B4C
:1002B0007091D20B83E79EE00F948F526091D30B25
:1002C0007091D40B86E69EE00F948F526091D10B13
:1002D0007091D20B8091D30B9091D40B681B790B4A
:1002E00080913609815021E030E0823010F030E01A
:1002F00020E0621B730B8BE59EE00F948F528AE027
:100300000F94514F83E59EE00F94DC4F8091D50B05
:100310009091D60BA091D70BB091D80B8C8F9D8F5D
:10032000AE8FBF8FBE016F5F7F4FCE014C960E9494
:100330003F63BE016F5F7F4F86E49EE00F94E853FA
:100340008091D90B9091DA0BA091DB0BB091DC0B73
:100350008C8F9D8FAE8FBF8FBE016F5F7F4FCE01A1
:100360004C960E943F63BE016F5F7F4F86E39EE025
:100370000F94E85320E030E04AE754E46091DD0B4D
:100380007091DE0B8091DF0B9091E00B0F94FAC51A
:10039000AB01BC018EE19EE00F9499528DE60F9463
:1003A000514F8AE00F94514F0C94607680918814DD
:1003B00083FF02C00C9460760E94883B87FF02C0D6
:1003C0000C94607689E40F94D642882311F40C943F
:1003D0008E8A0F94304290E01816190614F481E0CA
:1003E00090E026E0289FF001299FF00D1124E55DA3
:1003F000F34F808191810E94CBF661E080E00F9401
:1004000048B10F9462B10C9460768091881483FF98
:1004100002C00C9460760E94883BF82E87FF02C0D1
:100420000C94607689E40F94D642882311F40C94DE
:10043000998A0F94304290E01816190614F481E05E
:1004400090E026E0289FF001299FF00D1124E55D42
:10045000F34F8081918110E00E94CBF661E081E052
:100460000F9448B12091FB193091FC198091F91932
:100470009091FA1982179307F4F48FE89EE09F9306
:100480008F938AE99EE09F938F931F920E947C46F0
:100490000F900F900F900F900F9001E00F9462B1AA
:1004A000002311F40C94607640E0612F8F2D0F949F
:1004B000E2300C94607684E89EE0112301F3012F72
:1004C000EDCF10E0EBCF60E080E50E94353BF82EE9
:1004D00031E0381710F40C94607681E40F94884270
:1004E0006091C40D062F10E0811102C00FEF10E0E3
:1004F00089E40F94D642882311F40C94AB8A0F94AC
:10050000304290E01816190614F481E090E026E0DD
:10051000289FF001299FF00D1124E55DF34F048120
:100520001581EF2DF0E0EC53F24F0F3F110519F05C
:1005300010F00FEF10E000830C94607660E080E52F
:100540000E94353B823010F00C946076E82FF0E08A
:10055000EC53F24F10820C9460768EE40F94D642E6
:10056000882311F40C9460760F9420426093551503
:100570007093561580935715909358150C94607688
:1005800082EA9EE00DCE83E50F94D642882369F07F
:100590000F9430428D3320F480930C020C946076DB
:1005A0008CE380930C020C9460760F94FD5B1091A9
:1005B0000C0287EB9EE00F94DC4F812F0F94D1AC9F
:1005C0008AE00F94514F0C9460768091881483FFD9
:1005D00002C00C94607689E40F94D642882309F413
:1005E000C6C70F94304290E01816190614F481E043
:1005F00090E026E0289FF001299FF00D1124E55D91
:10060000F34F828193810F94484061E080E00F9422
:1006100048B10C9460768091881483FF02C00C94DA
:10062000607689E40F94D642882309F4AAC70F9410
:10063000304290E01816190614F481E090E026E0AC
:10064000289FF001299FF00D1124E55DF34F828171
:10065000938110E00F94484060E081E00F9448B12E
:1006600020919D0C30919E0C80919B0C90919C0C44
:10067000821793071CF48DEC9EE002C08EEB9EE087
:1006800060E00E94974660E0812F0F945B2F0C94EE
:10069000607683E50F94D642882311F40C9460763B
:1006A0000F943042182F8C3308F08CE38093390775
:1006B0000F94D0A26B017C01212F30E0A8EEB3E0B3
:1006C0000F94A6C4C60ED71EE81EF91EC0923507A9
:1006D000D0923607E0923707F09238070C94607694
:1006E0000E94FCEE0E945AF70F940A4D0F940D4D94
:1006F0001092900C10928F0C10928E0C68EE73E09A
:1007000080E090E00F94764C0F94124D60E08CEDF9
:100710009EE00E9497460C9460768091910C8F7EAB
:1007200080628093910C0C9460760E94AD3B0C9497
:1007300060760E94883B87FF02C00C9460768091AF
:10074000580784FD09C080915A0787FD05C0809134
:100750005B07837009F489C0FDEBCF2EF2E0DF2E3A
:10076000A9E8EA2EA4E1FA2E10E0D6018D916D01E0
:100770000F94D642882309F465C0133009F06DC088
:100780000F9458424B015C0120E030E040EA51E414
:100790000F940EBE87FF4EC0A50194016091A9146D
:1007A0007091AA148091AB149091AC140F94FAC577
:1007B0002B013C01AC019B016091B80D7091B90D0A
:1007C0008091BA0D9091BB0D0F9474BE6093B80DDB
:1007D0007093B90D8093BA0D9093BB0DA301920154
:1007E0006091B9147091BA148091BB149091BC14AB
:1007F0000F9474BE6093B9147093BA148093BB14B1
:100800009093BC146091A40D7091A50D8091A60DDC
:100810009091A70D0F9413BEA30192010F9474BE83
:100820000F9473C66093A40D7093A50D8093A60DCD
:100830009093A70D8092A9149092AA14A092AB1441
:10084000B092AC141F5FF4E0EF0EF11C143009F00D
:100850008CCF0E9425F70C9460760F945842F701D4
:10086000648B758B868B978BEDCF81E00F949C9872
:100870000C9460760E944D380C94607680917008DC
:1008800090917108009741F0DC012C91222321F016
:100890000F94B5860C94607680E00E9433470C94E8
:1008A0006076803529F4818180538A3008F42AC823
:1008B00041110F94FD5BFF2021F08DEE9EE00F941F
:1008C000DC4FC8010E94F8650C946076FF24F39415
:1008D00019C80F94C41C0C94607681E08093E20BDD
:1008E0008093E10B0F94081D0C9460768C01112706
:1008F00088E40F94D6428823C1F00F9454428A3A78
:1009000091050CF44BC00F9454428D3291400CF081
:1009100048C00F94544226E0209FF001219FF00D23
:100920001124E55DF34F9183808382E40F94D642D6
:100930008823A9F00F9454420597B4F10F945442C0
:100940008D389105A4F50F94544226E0209FF001C4
:10095000219FF00D1124E55DF34F9383828386E49C
:100960000F94D642882311F40C9460760F9454426D
:1009700097FD20C00F9454428F3F910509F0ECF48D
:100980000F94544226E0209FF001219FF00D112486
:10099000E55DF34F958384830C9460768AEA90E05A
:1009A000BACF8CE291E0B7CF85E090E0CECF8CE873
:1009B00090E0CBCF90E080E0E5CF8FEF90E0E2CF0A
:1009C00080E040C80E94883B87FF02C00C9460769C
:1009D0000DEB12E079E8E72E74E1F72EE1ECCE2E74
:1009E000E2E0DE2ED8018D918D010F94884288239C
:1009F00059F00F9458420F9473C6F70160837183C6
:100A0000828393830E94D7F6F4E0EF0EF11CC016A8
:100A1000D10641F70C9460760E94883B87FF02C0A4
:100A20000C9460766DEBE62E62E0F62E10E000E0AE
:100A3000D7018D917D010F948842882349F00F944E
:100A40005842F801E757FB4E64A375A386A397A30A
:100A50000C5F1F4F0031110559F70C94607683E548
:100A60000F94D642882391F00F9458426093BD149E
:100A70007093BE148093BF149093C0146093C514F8
:100A80007093C6148093C7149093C81480E50F9494
:100A9000D642882351F00F9458426093BD1470934E
:100AA000BE148093BF149093C01482E50F94D64275
:100AB000882351F00F9458426093C1147093C2146C
:100AC0008093C3149093C41484E50F94D642882372
:100AD00011F40C9460760F9458426093C51470938F
:100AE000C6148093C7149093C8140C9460760E9427
:100AF000263C0C9460765DEBE52E5CE0F52E10E074
:100B000088E5810F0F948842882351F00F94584252
:100B1000F7016083718382839383812F0F94E70AA7
:100B20001F5FF4E0EF0EF11C133051F780915A076C
:100B300087FF02C00C94C07980915B07837011F02D
:100B40000C94C0794091BD0C5091BE0C6091BF0CCB
:100B50007091C00C85E29FE00F9499524091C10CB6
:100B60005091C20C6091C30C7091C40C86EC9DE650
:100B70000F9499524091C50C5091C60C6091C70CCE
:100B80007091C80C83EC9DE60F9499528AE00F9403
:100B9000514F0C94607682E40F948842882341F090
:100BA00080918102909182029093120280931102AF
:100BB00082E50F948842882341F080911102909140
:100BC0001202909382028093810283E50F94D642B1
:100BD000882331F00F9454429093820280938102D3
:100BE0008091580790915907A0915A07B0915B07DF
:100BF000892B8A2B8B2B11F00C94607660918102EB
:100C0000709182028CE29FE00F94BA5285E20F94B9
:100C1000514F8AE00F94514F0C9460760E94883BAC
:100C2000082F87FF02C00C94607683E50F94D642AC
:100C3000002E000C110B7801EE0CFF1C882359F1DB
:100C40000F945442F701E75CFD4F91838083000FBE
:100C5000111F000F111F980125573D4F7901BC014D
:100C6000990F880B990B0F9415BE2AE037ED43E2DC
:100C70005CE30F9474BE025D164FD8012D913D9137
:100C80004D915C910F9474BEF701608371838283F0
:100C900093830C9460760F94FD5B85E40F94514F21
:100CA00080E3800F0F94514FF701E75CFD4F6081A7
:100CB000718180E39FE00F94BA5285E20F94514F07
:100CC0008AE00F94514F0C94607680E50F9488422F
:100CD000882311F40C9460760F9454428C01892B74
:100CE00009F082C083E50F948842882391F00F9425
:100CF00054428F3F980731F485E89AE10F94174DDD
:100D00000C946076BC0185E89AE10F94854D0C94B3
:100D100060760F94FD5B70E060E08BE39FE00F94E2
:100D2000BA528091871A08E5C02E02E0D02EC81A68
:100D3000D10887FDD394CC0CDD1CCC0CDD1C0D2C14
:100D4000000CEE08FF088091861A98E8892E912CF5
:100D5000881A910887FD9394880C991C880C991C1B
:100D6000092C000CAA08BB088091851A90E08F3FDF
:100D7000C9F1FC01EE0FFF1FE80FF91FE45CF54E0F
:100D800081819281B3E0880F991FBA95E1F7B0E0B5
:100D9000A0E014E0B595A795979587951A95D1F79A
:100DA00002969C012F5F3F4F032E000C440B550B06
:100DB000281939094A095B09A4EBB0E00F9493C4E0
:100DC000A7019601281939094A095B090F9474C4CF
:100DD000B90188E39FE00F94BA528AE00F94514F13
:100DE0000C94607680E0DDCF0F94F253B80182E579
:100DF0009FE00F94BA5283E49FE00F94DC4F0C9471
:100E000060760E94466C0C94607660E085E40E94F7
:100E1000353B811174C080E50F948842882351F0DE
:100E20000F9458426093FE197093FF198093001A33
:100E30009093011A89E40F948842882381F00F94DB
:100E400058422CEA35EC47E25EE30F9474BE60939F
:100E5000021A7093031A8093041A9093051A84E47B
:100E60000F948842882381F00F9458422CEA35EC85
:100E700047E25EE30F94FAC56093061A7093071A6F
:100E80008093081A9093091A0F94FD5B4091FE1904
:100E90005091FF196091001A7091011A81E69FE04C
:100EA0000F9499522CEA35EC47E25EE36091021A06
:100EB0007091031A8091041A9091051A0F94FAC543
:100EC000AB01BC018DE59FE00F9499522CEA35EC03
:100ED00047E25EE36091061A7091071A8091081A42
:100EE0009091091A0F9474BEAB01BC0189E59FE093
:100EF0000F9499528AE00F94514F0C9460760F949E
:100F0000F25385E69FE00F94DC4F0C94607680E509
:100F10000F948842882351F00F9458426093A00C9C
:100F20007093A10C8093A20C9093A30C89E40F946E
:100F30008842882381F00F9458422CEA35EC47E22E
:100F40005EE30F9474BE6093A40C7093A50C809321
:100F5000A60C9093A70C84E40F948842882381F018
:100F60000F9458422CEA35EC47E25EE30F94FAC541
:100F70006093A80C7093A90C8093AA0C9093AB0C6F
:100F80000F94FD5B4091A00C5091A10C6091A20CBC
:100F90007091A30C8FE79FE00F9499522CEA35ECE7
:100FA00047E25EE36091A40C7091A50C8091A60CC1
:100FB0009091A70C0F94FAC5AB01BC018BE79FE0A1
:100FC0000F9499522CEA35EC47E25EE36091A80C4D
:100FD0007091A90C8091AA0C9091AB0C0F9474BEE7
:100FE000AB01BC0187E79FE00F9499528AE00F9410
:100FF000514F0C94607683E50F948842182F882314
:1010000069F00F9454429C019093900280938F0258
:1010100091E0232B09F090E09093D60D80E50F949A
:101020008842882361F020918F0230919002232B17
:1010300011F00F9444428093D60D0C9460761111F8
:101040000C9460760F94FD5B8EEA9FE00F94DC4F6A
:101050008091D60D882391F086E99FE00F94DC4FB4
:1010600060918F02709190028DE99FE00F94BA52C7
:1010700089E99FE00F94DC4F0C94607682E99FE051
:10108000EDCF0E9449F70C9460760F941E430F94A5
:1010900030430F94E21B0C9460760E9420730C94F2
:1010A00060760E9469720C9460760F94F2538FED13
:1010B0009FE00F94DC4F61E081ED9FE00E94974636
:1010C0000E946D4468E270E088EC90E00E94D7B026
:1010D0000C94607684E50F9488428823A1F01092E6
:1010E00014091092150910921609109217091092FE
:1010F00018098FEF0F94224161E070E084E50F94AE
:101100000F438093180983E50F948842882321F0C8
:101110000F9454420F94224183E40F948842882311
:1011200031F080912002803210F40F94F64080E577
:101130000F948842882331F00F945442803210F487
:101140000F94F64085E50F948842882311F40C949F
:1011500060760F945442803210F00C94607641E037
:1011600050E060E070E0082E04C0440F551F661F79
:10117000771F0A94D2F7409550956095709500912D
:10118000140910911509209116093091170940236F
:1011900051236223732340931409509315096093DC
:1011A0001609709317099091200289130C946076A8
:1011B000109287140C9460760E9407F30C9460766A
:1011C0000F94171D0C94607661E083E50F94FA424A
:1011D00091E089270F9472320C94607680911B1BEA
:1011E00082FF05C0806480931B1B0C94607683FD96
:1011F00002C00C9460760F94F5980C9460760E946F
:10120000E8400C94607680E090E8ABE3B4E4F90148
:1012100080839183A283B3830C94427F80E090E823
:10122000ABE3B4E4F90184839583A683B7830C947C
:1012300060760E94C7440C9460760E94883B182F09
:1012400087FF02C00C9460768AE50F94D642812C09
:10125000912C90E2A92E91E4B92E882341F040E030
:1012600050E0BA018AE50F94E3424B015C01412F43
:1012700064E083E00E9486C720E030E0A901C50158
:10128000B4010F9460C718167CF580E090E0A0EAE6
:10129000B0E489839A83AB83BC8320918F0D309116
:1012A000900D4091910D5091920DC501B4010F9494
:1012B00000C56B017C0120E030E04AE753E40F9465
:1012C0000EBE87FD06C0C12CD12C8AE7E82E83E430
:1012D000F82ECC8EDD8EEE8EFF8EBE016F5F7F4FBF
:1012E000CE014C960F94121685E50F948842882300
:1012F00009F459C00F9458426B017C0120E030E0A2
:10130000A901C701B6010F9460C787FF04C0F7FAAF
:10131000F094F7F8F094F7FAF094F7F8F094C982A3
:10132000DA82EB82FC8244E061E0CE0101960F9408
:10133000C86620E030E0A901C501B4010F9460C780
:1013400018165CF580E090E0A0EAB0E489839A8307
:10135000AB83BC83A501940160918F0D7091900DBA
:101360008091910D9091920D0F94FFC46B017C01BF
:1013700020E030E0A9010F9460C718161CF0C12CC2
:10138000D12C7601CC8EDD8EEE8EFF8EBE016F5F8E
:101390007F4FCE014C960F94121610921A090E949C
:1013A0006D440C94607628E01202F0011124E5539C
:1013B000F64FC080D180E280F380A0CFA090BC0D1A
:1013C000B090BD0DC090BE0DD090BF0D8BE40F94BA
:1013D000D642882339F10F9458427B018C0120E0DA
:1013E00030E0A9010F9460C787FD0AC020E030E01B
:1013F00040E251E4B701C8010F940EBE1816A4F4E0
:101400008FE30F94514F8BE40F94514F83E190E1A0
:101410000F94DC4F8BE090E10F94DC4F88E090E17B
:101420000F94DC4F750186019701A801B501C60133
:101430000F940EBE882361F00E9449F7C701D801BE
:101440008093BC0D9093BD0DA093BE0DB093BF0DC6
:101450008091580790915907A0915A07B0915B0766
:10146000892B8A2B8B2B11F00C9460760F94FD5BEB
:101470004091BC0D5091BD0D6091BE0D7091BF0D9E
:1014800087E290E10F9499528AE00F94514F0C94A7
:10149000607681E080932A0C1092DF1760E083E58C
:1014A0000F94FA4281110C9460760F94C0870C94CB
:1014B00060760F94FD5B89E390E10F94DC4F80919F
:1014C000D309882349F086E390E10F94DC4F8AE04A
:1014D0000F94514F0C94607682E390E1F6CF0E9416
:1014E000768B0C94607610916D080F94D0A2609367
:1014F0007C0C70937D0C80937E0C90937F0C112359
:1015000011F40C946076812F0E94B2EE0C946076F8
:1015100011110C94007711E00C94FB7683E50F9485
:10152000D642882311F40C9401820F9454420C94F7
:10153000FB8183E50F94D642182F811108C082E504
:101540000F94D642082F882311F40C9461820F94D3
:1015500054420C942C8283E50F94D642882311F4D4
:101560000C9491820F9420428B010C94918283E51C
:101570000F94D642882311F40C9460760F94544251
:1015800042C883E50F94D642182F811107C082E527
:101590000F94D642882311F40C9460760F94544231
:1015A00059C8882309F4B7CF0C940377DF92EF92E0
:1015B000FF920F931F93CF93DF93EC01E090870C82
:1015C000F090880C8AE0D82E6AE070E0CE010F948B
:1015D000A1C98C01009711F0FC011082CE010E947C
:1015E000806481E00E948B740115110519F0E801F7
:1015F000D992EACFC701DF91CF911F910F91FF9050
:10160000EF90DF900C9480644F925F926F927F9284
:101610008F929F92AF92BF92CF92DF92EF92FF9202
:101620000F931F93CF93DF93CDB7DEB77C014DB6F9
:101630005EB66090870C7090880C8DB69EB66AE09E
:1016400070E0C7010F940CBD6C018C010E191F09CD
:10165000892B21F4C7010F941EBD8C01C80101968E
:101660002DB73EB7281B390B0FB6F8943EBF0FBEFF
:101670002DBF8DB79EB701965C01A801B7010F94ED
:101680003FBDF501E00FF11F1082C5010E9480648B
:1016900081E00E948B74C114D10451F076019FEF58
:1016A000E91AF90A0FB6F8949EBE0FBE8DBEC5CFDB
:1016B0000FB6F8949EBE0FBE8DBEC3010E9480641B
:1016C0000FB6F8945EBE0FBE4DBEDF91CF911F9155
:1016D0000F91FF90EF90DF90CF90BF90AF909F90D1
:1016E0008F907F906F905F904F9008954F925F9290
:1016F0006F927F928F929F92AF92BF92CF92DF9222
:10170000EF92FF920F931F93CF93DF93CDB7DEB786
:10171000C059D1090FB6F894DEBF0FBECDBF0F94EC
:101720006940882369F083E50F948842882301F19A
:1017300020E040E070E060E084E492EA0E94EA4346
:10174000C057DF4F0FB6F894DEBF0FBECDBFDF919D
:10175000CF911F910F91FF90EF90DF90CF90BF90AE
:10176000AF909F908F907F906F905F904F90089573
:1017700083E40F948842882319F00E9439A2E0CFB5
:101780008090700D9090710DA090720DB090730DBF
:101790008091790D80FF05C0909188149860909396
:1017A0008814869581708093D60D8BE09DE00E9411
:1017B000048B8091FF0C9091000D9E012F5F3F4F95
:1017C0007901009799F09F938F9382E09DE09F931A
:1017D0008F933F932F930F94A5BDC7010E94D68A84
:1017E0000F900F900F900F900F900F908091FD0C25
:1017F0009091FE0C009799F09F938F9389EF9CE056
:101800009F938F93FF92EF920F94A5BDC7010E9403
:10181000D68A0F900F900F900F900F900F906E013F
:1018200031E8C30ED11C6091DC0C7091DD0C80910D
:10183000DE0C9091DF0C860123E041E00F949EB80E
:101840009F938F9387EE9CE09F938F93FF92EF92ED
:101850000F94A5BDC7010E94D68A8FED9CE00E941F
:10186000048B87E08093E40B80932D090F900F90F9
:101870000F900F900F900F908091F80C8823F9F043
:101880006091F90C7091FA0C8091FB0C9091FC0C1A
:1018900023E041E00F949EB89F938F9386ED9CE0E8
:1018A0009F938F93FF92EF920F94A5BDC7010E9463
:1018B000D68A0F900F900F900F900F900F908091FD
:1018C000010D8823A1F01F928F931F921F9289EC24
:1018D0009CE09F938F93FF92EF920F94A5BDC70159
:1018E0000E94D68A0FB6F894DEBF0FBECDBF80919E
:1018F000020D8823A9F01F928F931F9281E08F938E
:1019000089EC9CE09F938F93FF92EF920F94A5BD7B
:10191000C7010E94D68A0FB6F894DEBF0FBECDBFB6
:101920004090030D5090040D6090050D7090060DD1
:1019300020E030E0A901C301B2010F940EBE811175
:1019400004C08091790D82FF20C0860121E041E032
:10195000C301B2010F949EB89F938F938091790D2C
:1019600082FB882780F91F928F938CEB9CE09F93DA
:101970008F93FF92EF920F94A5BDC7010E94D68A64
:101980000FB6F894DEBF0FBECDBF6091CE0C709144
:10199000CF0C8091D00C9091D10C8E010F581F4F1D
:1019A00023E041E00F949EB8782E692E6091CA0C16
:1019B0007091CB0C8091CC0C9091CD0C860123E0E2
:1019C00041E00F949EB86F927F929F938F938BEA22
:1019D0009CE09F938F93FF92EF920F94A5BDC70158
:1019E0000E94D68A6091D20C7091D30C8091D40C55
:1019F0009091D50C23E041E00F949EB880EA9CE0E2
:101A00000E94048BDF92CF9286E99CE09F938F9394
:101A1000FF92EF920F94A5BDC7010E94D68A8091D4
:101A2000DB0C8F938091DA0C8F938FE89CE09F936F
:101A30008F93FF92EF920F94A5BDC7010E94D68AA3
:101A40006091D60C7091D70C8091D80C9091D90CE4
:101A500023E041E00F949EB89F938F9385E89CE02C
:101A60009F938F93FF92EF920F94A5BDC7010E94A1
:101A7000D68A8CE0E0EEFCE0ADEBBCE001900D928C
:101A80008A95E1F78CE0ECEEFCE0A1EBBCE0019084
:101A90000D928A95E1F780E00F94E70A81E00F94B8
:101AA000E70A82E00F94E70A8091780D8093910C09
:101AB00081E08093D3090F945B4087E09DE09F9382
:101AC0008F938BEC9DE39F938F93FF92EF920F94F4
:101AD000A5BD0FB6F894DEBF0FBECDBFC7010E94F3
:101AE000D68A8091770D8F938091760D8F93809118
:101AF000750D8F938091740D8F93BF92AF929F92CB
:101B00008F9287E79CE09F938F93FF92EF920F94C1
:101B1000A5BDC7010E94D68A0FB6F894DEBF0FBEDE
:101B2000CDBF0ECECF93DF93C091C115C093970D5B
:101B300081E6C89FE0011124CD53DA4E80918814CC
:101B400080FF05C00F94FD5BCE010E94F865CE01B9
:101B50000E94806480E0DF91CF910C948B7460913F
:101B6000390270913A02072E000C880B990B0F94E2
:101B700015BE2AE037ED43E25CE30F9474BE20917A
:101B80002E0930912F0940913009509131090F945D
:101B900074BE60938B0270938C0280938D0290933D
:101BA0008E020895E0915A0CE23030F4F0E0EC53EC
:101BB000F24F8091480C808308958091101B8823F8
:101BC000C1F081508093101BECE3FBE1882351F0BE
:101BD0008150990B2BE1289FF001299FF00D1124D2
:101BE000EE58F44E8BE1A7E5BBE101900D928A958A
:101BF000E1F72091101B211105C080911B1B806211
:101C000080931B1B81E090E0A0E0B0E0211103C0B5
